:020000040800F2
:1000000000A0002081360108E9360108B526010864
:10001000E9360108E9360108E93601080000000068
:10002000000000000000000000000000E9360108A8
:10003000E936010800000000E93601085B120108FA
:10004000E9360108E9360108E9360108E936010810
:10005000E9360108E936010877ED000875ED00087A
:10006000E9360108E9360108E9360108E9360108F0
:10007000C9560008E93601085D100108E936010893
:10008000E9360108E9360108E9360108E9360108D0
:10009000E9360108E9360108E936010873ED000880
:1000A00001EA000841EA0008F1E9000869EA0008ED
:1000B00031EA000821EA000811EA0008E9360108DF
:1000C000E9360108E9360108E9360108E936010890
:1000D000E9360108551001084D10010845100108C6
:1000E00069120108E9360108E9360108E936010814
:1000F000E9360108E9360108E9360108E936010860
:10010000000000000000000000000000E9360108C7
:10011000E9360108E9360108E9360108E93601083F
:10012000E9360108E9360108E9360108E93601082F
:10013000E9360108E936010800000000000000006F
:10014000E9360108E9360108E93601080000000037
:10015000000000000000000000000000000000009F
:100160000000000000000000E9360108E93601083F
:10017000E936010800000000000000000000000057
:0801800000000000E93601084F
:100188002DE9F04F2DED068B6A4F6B4B3B60AFB0FE
:1001980000237B600EF0E7FF18B90FF007F80CF0AA
:1001A800C7F80CF083F9654A654C137843F00103EE
:1001B8001370644B4FF47002C3F88820002309932E
:1001C8000A93236843F480332360236803F40033DD
:1001D8000A93099B013309930A9B1BB9099BB3F541
:1001E800A04FF2D1236813F4003318BF01230A93F8
:1001F8000A9B012B67D0534E534BF360636ABB6075
:10020800636ADFF874A1DFF874B1DFF8749143F022
:1002180080736362636943F4FC032EAD6361032357
:100228008DF86A3041F6FF7325F8503D4FF0904045
:10023800294605F043FB4FF6FF7350462946ADF8B3
:10024800683005F03BFB4148294605F037FB40483C
:10025800294605F033FB3F48294605F02FFB294680
:100268003D4805F02BFB284609F0BCF93B4A1A9B90
:10027800B3FBF2F33A4A3B4813600021102216F010
:100288006DFD394B394A5A60F02286F82320002246
:100298009A60374E07221A60B368C9F800309BE8A5
:1002A8000300636985E8030043F48023636108233E
:1002B800CAF818301A981BA905F000FBD9F80030C5
:1002C8001B0729D464E02B4B12221A606368636011
:1002D80063686360636843F480636360636823F4FE
:1002E8007C136360636843F4E8136360236843F036
:1002F800807323602268124B9501FBD55A6822F05F
:1003080003025A605A6842F002025A60636803F0B6
:100318000C03082BFAD16EE796F89031012B37D8E9
:10032800044B96F891219B6813F0805800F0F085F3
:100338002EE000BFF0000020DFBC000808340020D9
:100348000010024000ED00E00005FA050008004832
:10035800000C0048001000480014004840420F00FC
:10036800282E00202C2E002010E000E03F1901006C
:10037800D417002000200240000400489C6E0108A9
:10038800D41F0020BF4B002283F891210CF052FAB1
:10039800642010F054FF0021BB484FF48C7216F013
:1003A800DDFCE369B94943F00703E361A36943F45A
:1003B800E123A361636943F4C023636101F5887E87
:1003C8008B7B4868CC7B03F00702DB0800EB8303D8
:1003D8009200186A4FF00F0C94400CFA02F220EACF
:1003E80002021A62186A103144EA000271451A6260
:1003F800E6D10022A649002353540132112AF9D12B
:10040800A44AFF2199540133072BF9D1A24BD9F8FB
:100418000080A24A1A60A24800213C2216F09EFCE5
:10042800C8F3801405234FF0000E9E4A9C481EF81E
:1004380002100C2202FB0EF211543CB91E3901299C
:100448009FBFFF2103F1FF331154DBB20EF1010E00
:10045800BEF1050FE9D1944A96F805B01370934B95
:10046800934983F800B0934B7B62C0330B60924B87
:10047800924A03EBCB0318F0200F5B7818BF0123D7
:10048800936200238E4A40F2DC5122F813100133A4
:10049800082BF7D113A800211C2216F05FFCDFF807
:1004A800349218F4007A1ABF1995CDF80C90CDF84B
:1004B8000CA0BBF10E0F03D00BF0EF03082B02D1F9
:1004C80001238DF85E30022007F05AFE18B14088EB
:1004D800003018BF0120C8F340038DF85230C8F32C
:1004E80040338DF84C30C8F3C03300F001008DF86C
:1004F8004F3018F400638DF851008DF8554004D042
:1005080096F884315C1E634263418DF85030C8F31D
:1005180000438DF85630BB6AB6F84441ADF86240E6
:100528001AF1000A18BF4FF0010A003318BF01235F
:100538008DF85830C8F300538DF85930B6F8463165
:10054800ADF85C30B6F85231ADF85A30C8F3804394
:100558008DF8533096F854318DF857A0181C18BFF1
:10056800012018F4805F18BF464C8DF85400B6F887
:1005780050011CBFB4F84C41ADF8624008F00101CD
:10058800C8F3C002B0F5FA7F8DF84D108DF84E20F3
:10059800ADF8600002D90BB9ADF8623096F8D431E5
:1005A800484887F82C30002387F82D3043709DF891
:1005B8005E30002B0CBF0023022301B902B10133C6
:1005C80009EB8309D9F81430A3F1020A2033049304
:1005D8004FF000093AF8023F4FF6FF72934200F0DD
:1005E800C6819DF85110DAB21B0ADEB279B12748EC
:1005F800354C00EB02104168A14208D10189B1F5E0
:10060800806F00F0B081B1F5006F00F0AC819DF80B
:10061800551031B111011D4840582C49884200F04D
:10062800A2819DF8561079B11101184C60186458D0
:1006380027498C4200F097814168B1F1904F03D16E
:10064800817B082900F08F819DF8521051B10F4825
:1006580000EB02104168B1F1904F03D101891029D4
:1006680000F081819DF84F10B1B30848164C00EB9B
:1006780002104168A1422FD10189042900F0738139
:100688002AE000BFD4170020802E0020CC9101085A
:10069800FC0000200D010020CC210020C6190020FC
:1006A800D4210020BE990108A1170020D0080020FD
:1006B80014300020E41700204C970108F0000020B7
:1006C800081700201D010020000400480004004015
:1006D800002C0140906E01089DF8501051B1B948A6
:1006E80000EB02104168B1F1904F03D10189202934
:1006F80000F03981199C7CB1B24F216807EB0217D1
:100708007868884208D13989A088884200F02B810E
:10071800E088884200F02781022B02D19DF84C30F6
:1007280003E0012B04D19DF84D30002B00F01B8114
:100738009DF85810A34B170159B19DF85E1041B9A7
:10074800A2F10E01012904D8D9599F48814208BF56
:1007580004269DF85910DC1931B19DF85E1019B9BD
:10076800043A032A40F2E780012E49D1DFF8648277
:100778000693D919FF2291F80DE088F8742088F8BB
:1007880075204868C8F8844001F108020989ADF865
:1007980068104FF0000B02218DF86B1088F878B0C4
:1007A8001AA98DF86AE0059288F830B0C8F834B014
:1007B800C8F838B0C8F83CB0C8F870B088F876B057
:1007C80088F877B005F07AF8069B059AD859917899
:1007D8005A4604F01FFF20465946324610F07EFB69
:1007E8007A4BC8F888307A4BC8F88C30C8F890B083
:1007F800204608F1880108F18C0210F0C5FBB2E030
:10080800022E4BD15FFA89F31C2101FB03FC714BCB
:10081800CDF81CC003EB0C0B01238BF87830069342
:10082800684B8BF87990D9194FF0000891F80DE0D2
:1008380048688BF87A8001F108020989ADF86810D8
:100848008BF882801AA9CBF884408DF86AE005926B
:100858008DF86B6005F032F85A4B059AD8599178A3
:10086800424604F0D7FE069B20461A46414610F041
:1008780035FB584BDDF81CC0574ACBF8882003EBF2
:100888000C01564ACBF88C208831CBF89080204652
:100898000A1D10F079FB09F1010964E0032E48D123
:1008A8009DF853304B4E4E4FE3B19DF85430DFF86E
:1008B800408196F82EB053B14A4BBDF86020B3FB87
:1008C800F2F22046082192B2BDF8623003E02046D9
:1008D80008214FF6FF7205F01AF847F82B00C0F808
:1008E8000C8020E0BDF8602096F82E80BDF86230BC
:1008F800B2F5FA7F0BD93B49B1FBF2F22046082149
:1009080092B205F004F8384B47F828000AE0374956
:10091800B1FBF2F22046012192B204F0F8FF344B09
:1009280047F82800C36096F82E30013386F82E3039
:1009380019E0042E17D1274EBDF85A2096F82D70CD
:100948002A4B93FBF2F22046BDF85C30012192B2AB
:1009580004F0DDFF96F82D3006EB87070133C7F862
:10096800580186F82D30049B9A457FF433AE194E12
:10097800204B96F82D2086F878211F4A1778A7F182
:1009880017020024022A1C709E4639D8736A234431
:10099800D3ED007AF5EE407AF1EE10FA03D1B36A9E
:1009A800002B4CD144E0154A04EB020C0FCB8CE829
:1009B8000F009EF8003010340133C02C8EF8003040
:1009C800E4D1ECE7CC91010800400140654F0008F4
:1009D80045500008F0000020595600083D4F000817
:1009E8004C2E002000127A006550000840420F008B
:1009F800555000087C2E0020D00800200C0800204C
:100A08003A4B13F837808EF8008003EBC703D3F80E
:100A18000490B9F1000FC2D04445C0DA344A23012A
:100A280003EB020C4B440FCB01348CE80F00F3E7C7
:100A3800304B1A6812F4805F994626D11FE02E4B7E
:100A48002E4A13F83700107003EBC7035C68002CBC
:100A5800EED000238342EBDAC3EBC3016218DFF860
:100A6800A880D2F8009041F8089001EB080C918812
:100A7800ACF8041092798CF806200133EAE707F005
:100A8800EF03082B1E4B20D121E09EF80020012AFD
:100A9800F5D91C4B03EB0212103210339342EED0FF
:100AA80053ED047AB6EE007A67EE877A43ED047A5E
:100AB80053ED057A67EE877A43ED057A53ED037AAD
:100AC80067EE877A43ED037AE7E70E2F08D11A78A5
:100AD80042F010021A70182F18D110F041FE15E0DC
:100AE8001A7822F010021A70192FF5E74C970108AE
:100AF8000C080020D41F0020607D0108A02F0020D2
:100B0800F01F002014080020A12F002010F00CFE78
:100B1800D9F80030B24CB34F580358BFB24BB34862
:100B28005CBF01221A70B24A137843F004031370B1
:100B38004FF40043ADF8683063694FF0020843F49E
:100B480000234FF0010B8DF86B8029468DF86AB0B1
:100B5800636104F0B3FEA74BA74A1A60002010F0A7
:100B680095FBE36943F48043E361236943F48043DD
:100B78002361636943F4802363617B6A23F4700310
:100B88007B627B6A43F4A0037B627B6A23F0706319
:100B98007B627B6A43F0A0637B627B6A23F07043CD
:100BA8007B627B6A43F0A0437B627B6A23F47023F9
:100BB8007B627B6A43F4A0237B624FF460431A9301
:100BC8008DF86C8003234FF00008384629464FF40F
:100BD800805A8DF86D3004938DF86E808DF86F8093
:100BE80008F0C4FC049B8DF86D3038462946CDF8D2
:100BF80068A08DF86CB08DF86E808DF86F8008F065
:100C0800B5FC236943F480432361236923F48043BB
:100C180023617A4B9A8822F480521204120C9A802B
:100C28009A8892B242EA0A029A801A8802F44152D9
:100C380042F4457242F003021A809A8822F47062E4
:100C48001204120C42F4E0629A809A8B22F4006239
:100C58001204120C9A8307221A821A8892B242F05E
:100C680040021A80C7F818A0D9F8003003F41073AE
:100C7800B3F5107F00F09E80614B624F1F6063697F
:100C8800DFF8609143F480236361E36943F4001360
:100C9800E361236B23F010032363236B43F01003FA
:100CA8002363D9F8203023F07063C9F82030D9F8CD
:100CB800203043F08063C9F82030D9F8203023F081
:100CC8007043C9F82030D9F8203043F08043C9F880
:100CD80020304FF000084FF0020C402248462946C9
:100CE8004FF0030B8DF86CC0CDF818C01A928DF830
:100CF8006E808DF86F808DF86DB008F037FC80221B
:100D0800484629461A9208F031FC3A68DFF80C91F7
:100D180022F001023A6039683B4A0A403A603B4A8D
:100D28003A613A6842F001023A60C7F80880C7F8A9
:100D38000C80C7F80880BA6842F40042BA603A6882
:100D48003A607A6822F0784222F400427A603A687F
:100D580042F001023A60D9F800502D4F05F40043E3
:100D68004FF0100A0493524605F400633846414692
:100D7800059315F0F3FF4FF6FF72DDF818C00E92D9
:100D880015F002058DF83DC08DF83E808DF83F8046
:100D98008DF83CB044D02EA94FF0904041F880AD7A
:100DA80008F0E4FB012507233D7087F80180FB70FC
:100DB800BD7035E0174A1378174918F901001F2844
:100DC80002BFFF2008F8010003F1FF3308F10C0807
:100DD80008BFDBB2B8F13C0FEED113704CE700BF8F
:100DE8000010024000040048380D002000080048A8
:100DF8000834002018340020A510010800380040ED
:100E0800D416002000540040FFE0CF00300E500000
:100E18003C220020A1170020D4210020D41F00204C
:100E2800049B7BB12EA9042341F8803D914808F02A
:100E38009DFB0C233B710723FB7101237D711D442E
:100E4800BB71EDB2059B83B12EA9202341F8803DEB
:100E58004FF0904008F08AFB02233B730723FB7393
:100E680001237D731D44BB73EDB2E36A824823F40A
:100E7800F873E362E36A43F4D873E362636943F0A7
:100E8800805343F00203636108F0ECFA1AA808F0F3
:100E9800BEFA7A4B1A937A4B1B93012D4FF000033D
:100EA80094BF1A4680221F924FF48072724C20928F
:100EB8004FF4806221922022204622921AA94FF4F0
:100EC80000521C931E9323922493ADF8745008F09B
:100ED800ABFA236843F0010323606A4CA36823F04C
:100EE8004053A360A36843F08053A3600A2010F026
:100EF800A6F9A36823F08043A360A368A360A3684E
:100F080043F00043A360A2685E4B002A2FDAFAE799
:100F1800531E092B3FF63CAADBF84C0028602946F3
:100F2800504604F0CBFC4FF40063CAF818303C205C
:100F380010F085F996F891319845BFF623AADFF8A5
:100F480034A108234FF4006BCAF8183078200393B3
:100F5800AAF828B010F068F9039BAAF8283078207E
:100F6800CAF818B010F060F908F10108E2E79A68C9
:100F7800454922F040529A609A6842F000529A60BD
:100F88008868424A024042F468328A60D968404A16
:100F98000A4042F40052DA601A6B013D22F00F0257
:100FA80015431D63002101237A189078002800F06A
:100FB80084805C1C042B17F801E0D278DFF8C4C0E9
:100FC800E4B20ED803EB4303DCF830505B001F207B
:100FD800984025EA00000EFA03F30343CCF83030BA
:100FE80031E0092B0ED80620053B4343DCF834508A
:100FF8001F20984025EA00000EFA03F30343CCF8BB
:10100800343020E00E2B4FF006050ED8A3F10A006D
:101018006843DCF838801F23834028EA03050EFA6A
:1010280000F32B43CCF838300DE00F3B05FB03F001
:10103800DCF83C801F23834028EA03050EFA00F3FE
:101048002B43CCF83C30BEF1090F0E4822D98369F6
:101058008569AEF10A0303EB43034FF0070E0EFA5E
:1010680003FE25EA0E05856185699A402A43826157
:1010780022E000BF0004004808040240400100507C
:101088004C2200200001005000030050E010FCFF3B
:1010980007C0FFFD436945690EF1FF3303EB4303C6
:1010A8004FF0380E0EFA03FE25EA0E054561456934
:1010B80003339A402A4342612346043110297FF4BE
:1010C80073AFC34B9A6842F001029A601A461168DE
:1010D800BF4BC907FBD5DA68BE4C22F00202DA60C2
:1010E800DA6842F00202DA60DA6842F00102DA6095
:1010F8009A6842F004029A60B4F85831002B41F023
:10110800CD80B4F95A21002A41F0C880B4F95C2195
:10111800002A41F0C380D9F800309B031FD5C820AE
:1011280010F08DF8AE200DF05AFC08B10DF062FFFA
:10113800A94D86F87901C82010F081F8A74BC6F8A8
:101148007C3100210C22284615F008FE0223EB70A2
:101158000CF0F3FB10F04CF8A14B0344AB60A14B2F
:10116800A1481B68DFF894A2B3F85EB094F85F81D9
:1011780094F8695194F86A7100210C2215F0EEFD7B
:1011880000211422994815F0E9FD002386F88031E2
:1011980019468AF881310C220AF5C270049315F0B9
:1011A800DDFD934AC6F89021232010F048F87520F9
:1011B80001210BAA0DF0CAF9049B002862D08D4AC0
:1011C800CAF888218C4ACAF88C2143228AF88421DB
:1011D800184601210CAA0DF0B9F99DF8303003F03A
:1011E8007E038DF8303040B1682B06D101238AF890
:1011F80080311D238AF8843144E09DF82C3003F0B7
:101208007E03682B8DF82C3037D10223062086F810
:1012180080310146D6F888311AAA98479DF86D1092
:1012280001F001029DF86B1001F001014B0043EA47
:1012380082019DF8692002F001030B430AD05BB2DA
:10124800012B01D1002302E0022B0FD1012386F8E4
:10125800813117E0694B0C20D3F8883101210EAA9F
:1012680098479DF8383013F00F0303D1032010F08E
:1012780061F807E0042BE9D1E4E7702B04BF0423ED
:1012880086F8803196F880215D490023022A0B7088
:1012980013D1564B5B4818605B4858605B48D86070
:1012A8005B48186104230B705A495B4B08681A7035
:1012B80040F001020A609A4603E0012010F03AF873
:1012C80021E242460A2A28BF00220123934040F225
:1012D800B23E03EA0E0EBEF1000F17D113F04D0F08
:1012E80014D0414B4D4A1A604D4A5A6096F88121F4
:1012F800002A0CBF6F226E221A724A4B04221A70FF
:10130800032318438AF80130086006E0012A4FF0E9
:101318000008D6D8434B83F80080042F00F23981A7
:10132800DFE817F0050042019900050042010A2094
:101338000FF085FF7720A02101220EAB04F0D8FB27
:10134800002800F088801E210122772004F04CFC40
:101358004FF42F600FF068FF4FF00008A8F160010C
:101368000027C9B202221AAB77208DF868708DF871
:10137800697004F0BDFB9DF869309DF8682043EA68
:1013880002221E4B03F5CA7128F8012008F1020851
:10139800B8F1100FE2D1B3F8A22102F47F4EA3F8FE
:1013A800A2E102F00F0101203B4627F0010232447E
:1013B800B2F89421002A18BF002017F0010F03D0BB
:1013C800D2B2534008222FE083EA1223FAE700BF83
:1013D80000010050D4170020542600205C1900207A
:1013E800404B4C0018170020F82C0020182500202E
:1013F800B46E010855E500086BE30008F000002012
:101408002C25002011E90008A1E2000885E2000867
:1014180090C1793DEC1F00207C000020B1E9000854
:10142800E9E200083334002013F4004F18BF83F4B6
:10143800C053013A4FEA4303F6D10137102FB4D114
:10144800844F4EEA0102A7F8A22120B9C3F303335F
:10145800994200F0038796F8A4317E4F002B40F0A4
:101468009B8014200FF0EBFE7720D02101220EABD9
:1014780004F03EFB002800F097809DF8383087F88C
:10148800BF310322552BA7F8C82140F08D80D12108
:1014980001220EAB772004F02BFB9DF8383003F0C7
:1014A8000F021B0987F8C02187F8C13116221AAB31
:1014B8007720AA2104F01CFB9DF868209DF869306C
:1014C80043EA0223A7F8A8319DF86A209DF86B30FB
:1014D80043EA0223A7F8AA319DF86C209DF86D30E5
:1014E80043EA0223A7F8AC319DF86E209DF86F30CF
:1014F80043EA0223A7F8AE319DF870209DF87130B9
:1015080043EA0223A7F8B0319DF872209DF87330A2
:1015180043EA0223A7F8B2319DF874209DF875308C
:1015280043EA0223A7F8B4319DF876209DF8773076
:1015380043EA0223A7F8B6319DF878209DF8793060
:1015480043EA0223A7F8B8319DF87A209DF87B304A
:1015580043EA0223A7F8BA319DF87C209DF87D3034
:1015680043EA0223A7F8BC313B4B41F270721A8060
:1015780046F678125A80394A5A60394A9A60394A86
:10158800DA60394A1A61394A5A61012387F8A43165
:1015980002E0012F01D107E00227354A8AF80270DC
:1015A800136843F004031360314F3B689A0702D570
:1015B800304B1B689847002386F8CC312E4B4FF4EC
:1015C8007A721A602D4BBC201B6898472C4A00235E
:1015D800022D1370904604D0032D1DD0002D40F02D
:1015E800538600238DF86830264BC6F8D0311E206C
:1015F8000A2101221AAB04F07BFA68B19DF8683021
:10160800482B09D1204B214A1A60214A5A600423E9
:1016180088F80030022341E04FF0000C0C206146AE
:1016280001221AAB8DF868C0CDF810C004F060FA3A
:1016380068B19DF86830DDF810C0482B40F09D86F1
:10164800114B144A1A60144A5A60032326E0844650
:1016580000F093BEF00000207C0600204DE3000857
:1016680051E4000831E3000811E40008E9DF00084C
:10167800EC1F0020F82C002040170020182500201F
:1016880030340020CC6E01085806002039E60008E6
:1016980077E300086BE5000879E400088AF803306E
:1016A8003B6843F008033B6094F855310BB1B84AE6
:1016B800137094F856310BB1B64A137094F8573139
:1016C8000BB188F800303B68B34913F0080F00F0FD
:1016D800D7850FFA8BFB64229BFBF2F302FB13B254
:1016E80012B207EE902AB8EEE77A07EE903ADFEDED
:1016F800AB6AF8EEE77AE7EE267AB2EE047A67EE9E
:10170800877AC1ED007AA64A137843F00203137072
:10171800A44B08229A610A25A24EB38A9BB283F091
:101728000803B38219200FF08AFD01200FF0AEFDE7
:1017380019200FF084FD013D00200FF0A7FD15F0E2
:10174800FF05E9D10823B361974E33681B0705D518
:10175800964B1B689847964B01221A70954B9FED44
:10176800968A1B68954D1B7B00EE103AB8EEC00AAE
:1017780020EE080A0AF07AFD914B9FED927A83EDEC
:10178800000A914BD3ED047A904B67EE887AC3ED4B
:10179800007A8F4B1B8807EE903AF8EEE77A8D4B6C
:1017A800C7EE277A9FED8C7AC7EE877AC3ED007A69
:1017B80009F06AFC2846FF211B2215F0CFFA002207
:1017C8002A703268854B012112F0020F18BF697028
:1017D80019701FBF032119700221A970570748BF4C
:1017E8001978284641BF4D1C1D700325455412F039
:1017F8000A0F0CD01A7804218154511CC9B205254E
:101808004554D11C0232D2B2197006218154D9F83C
:101818000020950641BF19784D1C1D70072548BF4B
:101828004554110608D51978092545548D1C0131F0
:10183800C9B21D700A2545546579082D01D00E2DB1
:1018480004D119784F1C1F700B274754197812F4CC
:10185800803F4FF00C0E00F801E001F101071CBFBA
:10186800DFF878E10231FFB21F701FBF8EF8001059
:1018780052494FF00E0E01F807E0510741BF1978A1
:101888004F1C1F70102748BF475419784F1CFFB2D0
:101898004FF0120E12F4806F1F7000F801E00ED0A6
:1018A80094F81CE2BEF1000F09D0DFF830E10231F4
:1018B8008EF8001041494FF0130E01F807E0970524
:1018C80041BF19784F1C1F70152748BF4754182D62
:1018D8000DD11978162747544F1CFFB24FF0170E39
:1018E80000F807E0CF1C0231C9B21F70455411033C
:1018F80041BF19784D1C1D70192548BF4554D205A4
:1019080048BF1A78364D41BF511C19701A218154AD
:101918001A78511C197014238354002198223148D5
:1019280015F01CFA07F071FB2F4B30491960304B4A
:10193800B4F84E212F4829602F491A8000232F4AD6
:10194800D0F800E00B70B4F89611138093701FFA6A
:1019580081F90EF181028046294F2A483D68DFF857
:10196800ACC020F8139005F596754CF82350013358
:10197800122BF1D1244DD5F800C01CF4805F08BFAC
:10198800B4F89C91A0F806900EF1D10E40E000BF8B
:101998002C25002033340020102600208988883C1C
:1019A8000834002000040048EC1F002058060020DE
:1019B80070060020E425002035FA8E3CE116002050
:1019C800142600200AE81C411825002000260020C3
:1019D8001C0000209407002000401C46E016002050
:1019E800A433002028210020B00E00205C1900201C
:1019F800B40E002018170020EB0D0020B033002093
:101A0800A8170020F6310020D41F0020340E002033
:101A18001378F3B992F80290D378994519D2B9F1AD
:101A2800000F08D009F1FF3909EB890909EB890989
:101A380009F5617306E0013303EB830303EB8303CA
:101A480003F5617392F8019009F104099BB220F83B
:101A5800193004327245DBD11CF0080F00F0C08049
:101A680094F89031062B00F2B580DFE803F0040704
:101A78000E355070700045F2F05201E042F6F8223F
:101A8800804B1A8007F06FFBA3E07E4B42F6F822EA
:101A98001A8009010A2391FBF3F10023A1F5B06133
:101AA800794A42F823100133122BF9D1774A784941
:101AB8001160784A4020137006F03CFC002800F0C2
:101AC800898001234FF0070A90F90000724A8DE8D7
:101AD80008044021714B77E06A4B42F6F8221A80DD
:101AE8006A4B6F4A1A606B4B102240201A7006F03E
:101AF80021FC00286ED001234FF0000990F9000066
:101B0800684A8DE8080240214FF4E1335CE05D4B00
:101B180042F6F8221A805D4B634A1A605D4B082230
:101B280040201A7006F006FC002853D001234FF01D
:101B3800000C90F900005D4A8DE8081040214FF430
:101B4800E13306F0CDFA5A4BC3F8D4013EE04D4AD2
:101B5800DFF890C1DFF890E1564C574842F6F8217B
:101B680011804C490C22062B0A700FD000232370D9
:101B78008CF800308EF800301B2303704F4B1A701E
:101B88004F4B05221A704FF4E1340CE0002121700C
:101B98008CF800108EF80010212101704749494C3B
:101BA8000A70474A1370394B474A1A60402006F0BA
:101BB800C1FB78B101234FF0000E444A90F90000B0
:101BC80040218DE80840234606F08AFA003018BF05
:101BD800012028B908200AF071FB2C4B3C4A1A60F6
:101BE8002B682C4A13F4804F1FBF1221117027490C
:101BF800384818BF086042F20101194003F001009B
:101C080003F4005481B11F4944F6206EA1F800E0A6
:101C180024B1082111701D492F4C0C6020B10C21F2
:101C280011701A492D48086011781806A1F10401AD
:101C3800517040F196801E48294CDFF8B090C0F8EA
:101C4800D8914FF0000A5146152200F5EE70DFF8E2
:101C5800A0B084F801A0C4F804A0C4F808A015F046
:101C68007DF8A9F105035046CBF8003008F01CFABE
:101C78003B68E360022006F05DFBD8BB80200AF0D9
:101C88001DFB66E0A80F00209032002020000020F5
:101C9800291F0108C4210020D5200108A0860100C1
:101CA800151F010829200108011F0108DD1F01086F
:101CB800F000002000210020232100209F33002075
:101CC8002421002090D00300ED8E0008018F000829
:101CD8008D1F01085D1F01087D1F01086D1F010888
:101CE800B0070020A033002001210020C6190020E1
:101CF800D007002090F805E06378CD490C2202FB5C
:101D080003125278724504D00133DBB2042BF4D9A4
:101D180000236370DBF8003062781B7890F90000CC
:101D2800002B4FF00C0303FB021314BF4FF0030EFC
:101D38004FF0010E00225B78CDF800E001920221FD
:101D480006F0CEF9BB4B1860002897D0012008F0A8
:101D5800ABF9D8F80000B84B00F5C9721A6008F062
:101D6800BBFA2B6813F4007F0DF168085CD0DFF82C
:101D78001493039BC9F80030B04BB1485A6942F438
:101D880080225A619A6942F001029A61039B1B887A
:101D9800ADF83030012402230CA98DF833308DF8CA
:101DA800324003F08BFDD9F80030A5485B88ADF8C8
:101DB80030304FF0000A0CA98DF832A003F07EFDF8
:101DC800D9F800302046197A07F00CFBD9F8003012
:101DD800586807F0BFFBD9F800305B681A93404693
:101DE80010238DF86D308DF86CA08DF86E400FF0D3
:101DF80057FFD9F800305B7A8DF838300EA80323E6
:101E08008DF839308DF83AA08DF83B400FF02AFF55
:101E18003B688C4A3C3B1360336843F010033360E3
:101E2800894B4FF0FF321A60884A894B1360894A00
:101E3800894E803313602B680024D903347040F135
:101E4800AA800DF0CFFEDFF840C2DFF8F091CDF8A0
:101E580010C040F22A3B0127604621465A46377097
:101E680014F07CFFD9F814307C4E4FF0904043F4C6
:101E78000033C9F81430436A23F00F034362436AFE
:101E880043F006034362022203234FF4807A0CA92D
:101E98008DF8342003928DF835308DF83640CDF822
:101EA80030A08DF8377007F061FBD9F81830039A25
:101EB80043F40063C9F81830338823F45C731B04B7
:101EC8001B0C33801D23F3620EA9328560233486F0
:101ED800304677610E93ADF83E401094ADF844401B
:101EE800ADF84640ADF84840ADF84A40ADF83C7012
:101EF80007F03BFAB36943F00803B361736C43F42A
:101F080000437364D9F814303B43C9F81430A9F678
:101F1800E479484607F0A6FA404607F078FA504BAD
:101F28001A9310231C938023DDF810C01F93414699
:101F38004FF400534846CDF86CC02393ADF874B005
:101F48001E94CDF880A021942294249407F06CFA72
:101F5800F36843F40073F360D9F8003043F00203E8
:101F6800C9F800300BA80C238DF82C308DF82D7093
:101F78008DF82E408DF82F700FF074FE2146394BE6
:101F88001A68394B43F8212001312029F7D103F091
:101F9800ADFB03F0ABFB2B685A0540F18580334C51
:101FA800334BD4F81C751F60042006F0C3F90421D4
:101FB800C4F8200506F09AF92E4B84F82405082069
:101FC8001F6006F0B7F92C4B2C4E1860082106F05C
:101FD8008DF9002184F825052C22304614F0BEFE28
:101FE8008E2373704FF07C0AE0234FF07D09F37065
:101FF80086F800A086F82B90214E2C22002130462E
:1020080014F0ACFE8A2373701020A023F37086F8B6
:1020180000A086F82B90C4F8287506F08BF91021DB
:10202800C4F82C0506F062F984F830052EE000BFEC
:10203800686F010850260020040F0020001002409D
:1020480000040048A807002038170020B820002006
:10205800001A002094260020390D0020002C014091
:10206800342C0140E46E01083A0D0020F0000020F5
:10207800E01F0020382000208420002008200020B5
:102088003D200020AC070020E10200202020C4F8F9
:10209800347506F04FF92021C4F8380506F026F902
:1020A80084F83C050BF020FBB84A138823F0400362
:1020B8001B041B0C1380138823F038031B041B0C10
:1020C800138013889BB243F04003138000249F239E
:1020D80032208DF838308DF839408DF83A408DF837
:1020E8003B400FF0ACF88DF86940A94C4FF480568E
:1020F8000422268540460EA90FF07EFDA6619DF8B4
:102108006A209DF86930120242EA03429DF86B305A
:102118001A43A04B9A42A04B17D008D89F498A422D
:102128000CD001F51A4102318A4209D01CE09C49C1
:102138008A4205D001318A4207D015E0202200E00A
:1021480080221A804FF4807202E04FF480721A8065
:102158005A809A88198812029A604A43DA60914A2A
:10216800012182F83D1504E000221A805A809A6005
:10217800DA60DC680CB3E40A27464FF00009A14591
:1021880009DA09EB04067610F002414610220CF039
:102198000BFF0F2806DC08F017FB824BFF02C3F881
:1021A80040750AE0002358F82320013272D1013328
:1021B800042BF8D137463446E1E72B687A4A13F402
:1021C800002318BF012313700FF012F8774B186023
:1021D800774B5A79052A194602BF764B4FF4C872D5
:1021E8001A80754B4FF47A721A80744BC8221A8081
:1021F800734A137843F008031370724A137823F074
:10220800020313702A6840F6020313406BB16E4B49
:102218006E4818606E4B032018706E4B01201870C2
:102228006D48002303806D480380930341BF6C4BC6
:1022380004221A71DA7844BF42F00102DA708B681E
:102248002B60684B01221A70674A137863F07F038A
:1022580013702FB0BDEC068BBDE8F08F634B42F2D4
:1022680010721A805A80624A5A60624A9A60624AB8
:10227800DA60624A1A61624A5A610327FFF78DB928
:1022880000230B60FFF73FBA012D7FF60DAA1D460C
:10229800FFF79CB906F1010926468CE71BB208EE48
:1022A800103AB4F95A31DFED577A574A09EE103A25
:1022B800B4F95C31B8EEC88A08EE903A28EE278A5D
:1022C800B8EEC99AF8EEE88A0021B0EE480A29EE7D
:1022D800279A68EEA78A117009F0C8FFF0EE40AAA5
:1022E800B0EE480A09F061FFF0EE409AB0EE490AF4
:1022F80009F0BCFFB0EE40AAB0EE490A09F055FF5C
:10230800B0EE408AB0EE680A09F0B0FFB0EE409A2D
:10231800B0EE680A09F049FF60EE2A6A69EE897A28
:10232800F0EE665AE7EE885A384B29EE2A6A29EE0B
:10233800807AC3ED035AF0EE465A2AEE400AE7EED9
:10234800485AE6EE887AA6EE487A29EE0A9A83ED8C
:10235800010A69EECA9A2AEE2A0A83ED009A83EDE9
:10236800028AC3ED045AC3ED059A83ED067AC3EDDC
:10237800077A83ED080AFEF7CEBE012D7FF694A9F1
:10238800002588F800C0FFF72CB900BF00380040CE
:102398000004004818BA20000C0000201520200076
:1023A8001740EF00F000002018300020D40700206C
:1023B800D4170020B02500202E3400202834002017
:1023C800F01F002032340020D81F00204E190020B2
:1023D8003C20002078000020D00F0020D20F0020E1
:1023E80054260020380D0020083400207C060020E8
:1023F80061E3000845E5000857E3000835E50008F3
:10240800C5E0000835FA8E3C540000201822002050
:102418002DE9F04FA249A34C0A6802F59C432DED23
:10242800028B20332360A04B87B01E780091C6B181
:102438009E4909688A4240F20581013E1E7001E109
:10244800D9F800309A48072D98BF595D994B88BF35
:1024580029461B689847032D0CD904EB450501361E
:10246800A880934BDFF870921A78F5B2AA42194601
:10247800E6D820E0D9F8002005F10E0302EB83032B
:102488009988DA880028E8D04FF47A73401A5843BC
:10249800531A90FBF3F040F6C90300F57A7098429E
:1024A80005DC40F2EE239842B8BF184601E040F63A
:1024B800CA0080B2D1E7804B1B6842F2010803EAE8
:1024C80008087E4BB8FA88F84FEA58181B68B8F124
:1024D800000F06D194F8292084F82820784A5078EB
:1024E800107094F828701FB1754A177887F00107A3
:1024F80094F82BB091F800A00F220326BBFBF6F648
:1025080006EB460684F82A20C6EB0B06D9F800200D
:10251800DFF8CC91F6B20025554559DA4FEA450C5B
:102528001FB1684931F8150000E03846918ADFF894
:10253800B4E1814202D8D18A81421ED25EF82500D8
:102548005849834203D2604931F80C0019E0E8B2D7
:102558000292019303910FF02DFE032D019B029A25
:102568000FDC03994FF0010C91F82AE00CFA05FCF6
:102578002EEA0C0E81F82AE003E003F596714EF876
:102588002510B8F1000F1CD194F8BC1029F81600DA
:1025980031B9BBF1020F14D94249012081F8BC00BE
:1025A800B9F80210B9F800000844B9F80410084452
:1025B800464980B221F8150000B2032190FBF1F0E2
:1025C80080B2414909F1060921F815000135A3E750
:1025D80094F82A2039493E4BA2F10F0EDEF1000291
:1025E80042EB0E0284F8D6206AB13A4A12685701C3
:1025F80009D40A68D9689A60521AC82A1DD90122D2
:1026080083F8212019E02E4A0120507010700A68C2
:102618009968DA605B68521A9A4282BF2C4B002292
:1026280083F821200025554507DAE8B20FF0C2FDEE
:10263800254B23F815000135F5E794F82B300133C5
:1026480084F82B301C4B1A6812F4805F984605D02A
:10265800204B1B68DE0701D40FF072FA009B196843
:102668001D4B1868837A002B3ED0013B164D027B28
:1026780035F813301AB1C3F53B6308339BB21BB26C
:10268800A3F57A73B3F57A7FA8BF4FF47A7323EA78
:10269800E37307EE903A9FED117AF8EEE77A5CE083
:1026A80010340020C00D0020AC330020A8330020D7
:1026B800C421002020000020D41F0020A8170020DB
:1026C80008000020C40D0020F63100207E0E0020F6
:1026D800B0330020DC160020A433002000007A4428
:1026E800EC0D0020340E0020D8F80020150440D549
:1026F800D4F8D820934E8A1A002A3ADB01F59C4276
:102708002032C6F8D820904AC07A55798F4A32F8D4
:10271800152096F8DC50013592B292FBF0F205F0E4
:102728000F0086F8DC00304480F8DD201A4688481F
:10273800185C01330244102B92B2F8D112B292FB0A
:10274800F3F31BB2642BA8BF642323EAE37307EEF9
:10275800903A9FED807AF8EEE77AC7EE877A7E4A5C
:102768009FED7E7A67EE877AFCEEE77A17EE903A6D
:102778001380D8F800307A4F13F4807F00F0098175
:10278800784BDFF8E491994205D999F8022012B9FB
:10279800012289F8022099F80220002A00F0F98025
:1027A800714A3E7892F821506A1E554255416F4A47
:1027B8001168002DC1F38063C6F38006009392462A
:1027C80014BF4FF0000B4FF0030B99F82020052A97
:1027D80000F2D980DFE802F0034D527584A1002E83
:1027E8003AD0D4F8F000B4F8F4100EF0BCFC01288C
:1027F80009D15F495F4A09681268C988642000FBEB
:102808000122C9F81020009B6BB1594A126812794D
:102818004AB10FF02DFF032289F820204FF47A7275
:10282800C9F81C20D1E7002D40F0AD80514AD9F8F5
:10283800101010684C4A88420AD901920FF018FF0C
:10284800019A032182F8201040F6B831D161BCE723
:10285800012182F82010B8E7009B4FF4806013B183
:1028680009F01CFD01E009F009FD0022C9F810205B
:1028780089E0002D46D10FF0FBFEA6E725B1052221
:1028880089F82020012000E0284666B1D4F8F0201D
:10289800D189394A11805180918035490968498820
:1028A800D1804FF0020B334A1168D9F814209142B5
:1028B80001D8002E64D147F23052C9F81C200322F7
:1028C80021E03A7842F002023A700FF039F9294AC9
:1028D800D9F81C1012680A44C9F81820042212E01A
:1028E800244A9DB11168D9F8182091424BD9234A3E
:1028F80092781AB9DAF80020D30744D43A7822F04B
:1029080002023A70052289F820205EE71268D9F899
:102918001C100A44C9F8182035E01549154A0968F9
:102928001268C988642000FB0122C9F810204FF4FE
:102938008060002289F8202089F8032009F09EFC95
:1029480043E700BFC00D00203C2200204C2200209D
:102958009D0E00200000C8423C17002000C07F44A4
:1029680032340020404B4C00B0330020DC160020ED
:1029780004340020A8170020F631002008000020A9
:1029880000287FF422AFBBF1000F02D058460EF0AA
:1029980097FC984D05F5C470B5F84E110EF0E3FBA1
:1029A800834668B90FF05AFE934BC3F800B0C3F8DA
:1029B80004B0C3F808B0914B00221A605A609A60BC
:1029C8003B785E0736D5D8F80030D80632D58C4B20
:1029D8001B78D9062ED48B4B9B7893B195F8E031B0
:1029E800BBF1000F15D17BB1874B1A68D4F8F830CA
:1029F8009B1A002B08DA0FF0A3F8844B83F8FCB07D
:102A080018E0BBF1000F0DD110200EF059FC012386
:102A18000EE03BB17C4A12684FF47A7101FB032344
:102A2800C4F8F83094F8FC3023B10EF035FC0023DC
:102A380084F8FC30002295F8DEA195F8DF11B5F88E
:102A480098E1B5F89AC113467148009030F91260C0
:102A58009B087645C4BF63F07F03DBB2013266454D
:102A6800B8BF43F04003042AEED194F8FD2067482C
:102A78009A4205D190F8FE20F92A04D8013200E0E4
:102A8800002280F8FE2084F8FD305E4B614E9A7873
:102A98009946E2B93368DA0708D5BBF1000F16D1B9
:102AA8003B78DB0713D50EF09DFE10E03B78580706
:102AB8000DD5564B93F828304BB1574BDB7833B9CB
:102AC80011B10FF03DF802E0BBF1000FF9D094F816
:102AD800FE304E4ADFF85CB1142B40F0B48099F810
:102AE80002301AF1000A18BF4FF0010A6BB392F8CE
:102AF800FD305F2B11D13B7803F0040303F0FF0195
:102B080013B10FF01DF808E00B20029101920EF0AE
:102B1800D7FB019A029982F8FE10BAF1000F14D07F
:102B280094F8FD307D2B10D13B7803F0040303F0BB
:102B3800FF0213B10FF004F807E00B2001920EF02A
:102B4800BFFB324B019A83F8FE203B7803F0040365
:102B580003F0FF01002B76D194F8FD302B4A572B58
:102B680010D12E4B4FF47A721A80D8F800301A061A
:102B780001D507F013FC2A4B1B685B0763D50A22B3
:102B8800284B34E0D8F80000400716D55A2B14D14A
:102B9800254B187820B11970244B01221A7052E085
:102BA80092F8FF3083F0010382F8FF300BB10C205C
:102BB80000E00D200EF084FB45E05D2B00F0318530
:102BC8005B2B00F030855E2B02D1032000F02CBD7A
:102BD800562B01D109F02EFE99F8023063BB94F808
:102BE800FD30972B40F03885114B4FF4C8721A808E
:102BF80029E000BFD41700208C240020DC330020FB
:102C0800F01F002008000020A8170020C00D002099
:102C1800F6310020DC160020B03300202E340020CE
:102C2800EC1F002028340020DD250020DE250020B0
:102C3800B02500201817002094F8FD306F2B40F0C5
:102C480002850EF0CFFDD8F80030580732D594F839
:102C5800FF30A3B13B78590711D5009BB3F9062083
:102C6800B5F898319A420ADD336813F0010301BFC1
:102C7800AD4A32211180AD4A08BF82F8FF3033686F
:102C8800DA030AD5AA4B1A782AB9AA4A127812B9CD
:102C9800A54A3221118001220BE0A64A13784BB1D4
:102CA8003B7803F0040303F0FF011BB9A24B11703A
:102CB80001221A70DBF800A0002333600AF18309AF
:102CC8000AF1D30B99F8002099F8013019F8010C92
:102CD8009A420BD249460EF00FFA38B119F8022C75
:102CE800012303FA02F233681343336009F104093C
:102CF800D945E7D1914B1B7843B1914B914E1A6856
:102D080012F0020F994640F03F8336E30AF1D206EB
:102D18000AF58D793278737816F8010C9A4225D223
:102D280031460EF0E9F908B3B37896F804C0864A3C
:102D380096F803A07D480C21013B01FB0C4103EBF5
:102D480043031344D1F804219A420FD0C1F8043147
:102D5800002390F83021C1F80831012303FA0CF35D
:102D680022EA030381F800A180F8303106364E4587
:102D7800D0D1764B1E68764B1B68029394F82830A6
:102D88000393744B019300230093019B1B68002B52
:102D980000F0E88293F800A0BAF1000F00F0E28298
:102DA800019A029952688A1A002A0CDB01F5FA7214
:102DB80001994A60009901228A4094F8301121EA69
:102DC800020284F83021039A002A00F0CB82019A8B
:102DD800597812F8042C0432D2B2002940F08182CA
:102DE8005D4931F91210B5F8962102F1C800814207
:102DF80002DD93F802B015E0C83A914203DA9978F7
:102E0800C1F1000B0EE0009A0123934094F83021A1
:102E180022EA030384F83031029B019A03F5FA731E
:102E280053609FE294F83031009A1341DB0700F1B8
:102E38009982BBF1000FCCBF022001200EF062FA8C
:102E48000AF1FF33DFF8E490132B00F28382DFE806
:102E580013F01400250037004B0064008B00EE00CF
:102E68005101B801E601160281024B005A008B009D
:102E7800EE005101C0002301880196F80090D94462
:102E8800B9F1FA0FA8BF4FF0FA0929EAE9793046F3
:102E980086F800900EF016F901200FE096F80190E0
:102EA800D944B9F1640FA8BF4FF0640929EAE97958
:102EB800304686F801900EF005F902204946DBE11C
:102EC80096F803A0DA44BAF1640FA8BF4FF0640A79
:102ED8002AEAEA7A86F803A03046D9F8341105F0D0
:102EE8002FFA03205146C7E1717959446429A8BFD4
:102EF800642121EAE17171710D200EF065F9BAF1D2
:102F08000D0F00F02782317959446429A8BF642144
:102F180021EAE17131710E20AEE1B179594481F3B2
:102F28000801B1710520A7E1C4250020C00D0020CB
:102F3800DC250020DD250020DE250020343400209B
:102F4800DC160020EC1F00206073010844170020E5
:102F5800A8170020C40E0020F631002000007A4493
:102F68000000C84200000000D9F838311A78022A57
:102F780020D107EE90BAB8EEE70A5FED077A93ED35
:102F8800097A80EE270A30EE070AB5EEC00AF1EE9C
:102F980010FA07D4B4EE670AF1EE10FAC8BFB0EE23
:102FA800670A01E01FED110A83ED090A0F200EF0F0
:102FB800F5F80AE099785944C829A8BFC82121EA38
:102FC800E17199700F200EF0FFF8BAF10F0F00F0C1
:102FD800C181D9F838311A78022A1ED107EE90BA81
:102FE800B8EEE78A5FED227A93ED080A88EE278A21
:102FF80038EE000AB5EEC00AF1EE10FA07D4B4EEC6
:10300800670AF1EE10FAC8BFB0EE670A01E01FEDDB
:103018002B0A83ED080A122056E159785944C82929
:10302800A8BFC82121EAE1715970122024E1D9F81A
:1030380038311A78022A20D107EE90BAB8EEE70A9A
:103048005FED397A93ED0C7A80EE270A30EE070AA5
:10305800B5EEC00AF1EE10FA07D4B4EE670AF1EE45
:1030680010FAC8BFB0EE670A01E01FED420A83ED0F
:103078000C0A10200EF092F80AE0197B5944C8296E
:10308800A8BFC82121EAE171197310200EF09CF83D
:10309800BAF1100F00F05E81D9F838311A78022A97
:1030A8001ED107EE90BAB8EEE78A5FED537A93ED3A
:1030B8000B0A88EE278A38EE000AB5EEC00AF1EE50
:1030C80010FA07D4B4EE670AF1EE10FAC8BFB0EEF2
:1030D800670A01E01FED5D0A83ED0B0A1320F3E098
:1030E800D97A5944C829A8BFC82121EAE171D972FF
:1030F8001320C1E0D9F838311A78022A22D107EE14
:1031080090BA1FED6A0AF8EEE77A87EE800AD3EDE7
:103118000F7A30EE270AB5EEC00AF1EE10FA09D49C
:103128005FED717AB4EE670AF1EE10FAC8BFB0EE3F
:10313800670A01E01FED750A83ED0F0A11200EF0F2
:103148002DF80AE0997D5944C829A8BFC82121EA69
:10315800E171997511200EF037F8BAF1110F00F0EE
:10316800F980D9F838311A78022A20D107EE90BAB6
:103178001FED860AB8EEE78A88EE008A93ED0E0AFC
:1031880038EE000AB5EEC00AF1EE10FA09D45FED88
:103198008C7AB4EE670AF1EE10FAC8BFB0EE670A8F
:1031A80001E01FED900A83ED0E0A14208CE0597D92
:1031B8005944C829A8BFC82121EAE17159751420CA
:1031C8005AE0D9F838311A78022A1ED107EE90BA97
:1031D800B8EEE78A5FED9E7A93ED0A0A88EE278AB1
:1031E80038EE000AB5EEC00AF1EE10FA07D4B4EED4
:1031F800670AF1EE10FAC8BFB0EE670A01E01FEDEA
:10320800A70A83ED0A0A09205EE0D9785944C8293B
:10321800A8BFC82121EAE171D97009202CE0D9F8AA
:1032280038311A78022A1ED107EE90BAB8EEE78A2A
:103238005FEDB57A93ED0D0A88EE278A38EE000A1D
:10324800B5EEC00AF1EE10FA07D4B4EE670AF1EE53
:1032580010FAC8BFB0EE670A01E01FEDBE0A83EDA1
:103268000D0A0A2030E0597B5944C829A8BFC82153
:1032780021EAE17159730A200DF0A6FF6AE0D9F836
:1032880038311A78022A22D107EE90BA1FEDCD0AFA
:10329800B8EEE78A88EE008A93ED100A38EE000A45
:1032A800B5EEC00AF1EE10FA09D45FEDD37AB4EEA8
:1032B800670AF1EE10FAC8BFB0EE670A01E01FED29
:1032C800D70A83ED100A0B200DF068FF42E0D97D84
:1032D8005944C829A8BFC82121EAE171D9750B2032
:1032E800CAE7012936D19878BA4B33F91230B3F5C9
:1032F800617F05DB40F633029342A8BF134601E025
:103308004FF46173BAF10C0F24D14FF4966292FB1B
:10331800F0F0B14AA3F5617393FBF0F35FFA83F918
:1033280013784B4516D0B9F1040F34BF4B4602232E
:103338001370AA4A0AFB035303F2CE73136009F011
:1033480091F8504649460DF03FFF09F10100C0B21F
:103358000DF0D8FF009A0123934094F830211343CD
:1033680084F83031009B01330093019B0C330193A7
:10337800009B042B7FF409ADBFE4D8F80030D805D2
:1033880010D5974BDB786BB1336899070AD5954B05
:103398001B8813F0010A0AD10FF060F9012008F028
:1033A8007DFF04E0012008F069FF012300E000230D
:1033B800D9F8002052070DD563B1012008F05EFF4F
:1033C800884B1B88980708D40FF048F9022008F0AA
:1033D80065FF02E0022008F051FF336813F00A0F7E
:1033E80032D0D9F80030D9060FD57E4B1B885A0742
:1033F8000ED4042008F052FF7B4B0A22B3F90430A4
:1034080093FBF2F3A4F83C3102E0042008F036FF05
:10341800D9F800309B0607D5724B1B88580606D48E
:10342800402008F03BFF02E0402008F027FFD9F8D1
:103438000030590641BF6C4BB3F904300A2293FBA4
:10344800F2F348BFA4F83E3133689A0609D4D9F894
:1034580000301B0540F194804FF4807008F01EFF87
:1034680092E0624BDFF87CA11B7813F0020F53D077
:103478005F4B1B78042B4FD9D9F8003013F4007B2D
:103488000FD0BAF80030DE063AD4102008F006FF54
:10349800202008F0F3FE5748011D06F0D3FE022352
:1034A8002AE0BAF8006006F01006B6B22EB1102075
:1034B80008F0E4FE012684F840B1D9F80030580538
:1034C80012D5D4F844314C495A89B1F90030002B4F
:1034D800B8BF5B42934207DAB1F90230002BB8BF9C
:1034E8005B429342C0F20081BAF80030990608D5D1
:1034F800202008F0C3FE002384F84031012600E0B4
:10350800002694F84831BBB90E200DF0D9FE3B4B8C
:10351800012283F848210FE0BAF8003003F03003A5
:10352800002B94D0102008F0A9FE202008F0A6FE59
:10353800002384F8403101E0002E88D0304B002071
:1035480003F1280603F150042E4A002122F8101036
:103558002D4A596022F810100432716022F81010B8
:1035680000221A609A603260B26022606160A260D4
:1035780014331436143400287FF469AF0120E3E7CC
:103588004FF4807008F07AFE6B79082B01D00E2B6F
:1035980002D1402008F072FED8F800305A0540F1F8
:1035A800B98095F81C321BB93B7813F0040F03E07F
:1035B800D9F8003013F4002F2AD0144B00221A70C7
:1035C8003C2005F019FE002800F0A4800DF010F84A
:1035D800F6E700BFF6310020D82C00204417002061
:1035E800B0330020B4200020C0170020F01F0020B6
:1035F800F61F00204C170020CC170020C00D00201B
:103608000C0F00202A340020840F0020D021002035
:103618000AF06AF807B0BDEC028BBDE8F04F05F080
:10362800F4BC012000E002205FFA80F909F1FF33C1
:1036380085F8CC3708F07CFE08F038FF48460DF0D6
:1036480061FEFFF700BBBAF1000F3FF4C8AA7E2B5A
:103658007FF4C5AAFFF7F5BAA72B06D1304A13782D
:1036680043F004031370FFF7EEBA0022BB2B059258
:1036780001D1022303E0B72B04D14FF6FE73ADF856
:10368800163009E0BE2B01D1022303E0BD2B1AD16D
:103698004FF6FE73ADF81430DBF80030BDF81410A7
:1036A800B3F860200A44A3F86020BDF81610B3F8F8
:1036B80062200A44A3F8622009F0BCF8002384F8C9
:1036C800FE30FFF7C0BA792B04D1164AD37823F01D
:1036D800010306E07A2B7FF4B6AA124AD37843F0A6
:1036E8000103D370FFF7AFBABAF800309B063FF575
:1036F80008AF202008F0D2FD0B480C4B011D1A68BA
:103708005B684360026006F09DFD094B012683F863
:103718004061F6E607B0BDEC028BBDE8F08F00BF54
:10372800F01F00205426002054170020F81F002006
:10373800C00D00202DE9F04FBB4BB3F90610BB4B71
:103748002DED028B1E6872898FB0914201930EDBBA
:10375800B1F5FA6FF479BDBF8B1A6343A2F5FA6429
:10376800C4F16404BCBF93FBF4F4643400E0642443
:10377800AF4BB04AB3F896B193F95E311268029232
:103788009BB2154603930022A74B33F912E0CBEB0B
:103798000E0303F2F31740F2E63087424FEA420C79
:1037A80003D8002BB8BF5B4201E04FF4FA73022A3A
:1037B80000934FF06400029B2FD093F819712FB13A
:1037C800009BBB42CCBFDB1B00230093009B9A4F9E
:1037D80093FBF0F86FF0630A37F818900AFB083A81
:1037E80008F10108954B37F918700FFA89F8C8EBFA
:1037F800070707FB0AF797FBF0F74F4423F80C700D
:10380800B718009B3F797B438D4F93FBF7F36433E5
:103818009BB2634393FBF0F02EE093F81A712FB13B
:10382800009BBB42CCBFDB1B00230093009BDFF84F
:10383800309293FBF0F06FF0630839F9107008FBD1
:10384800003A0130BDF80C3039F91000C01B00FBFC
:103858000AFA9AFBF8FAC7EB0A0A1AFB03FA774B3B
:10386800A3F804A0009BB079002BB8BF5B42434388
:10387800734893FBF0F064306F78724B4FF0640834
:10388800474397FBF8F79F5403F10309EF7A47433F
:1038980097FBF8F709F8027006336F7D022A00FBE0
:1038A80007F0664F90FBF8F09854674B0ED1DE4551
:1038B80083F802800DDB5E4CB4F89821914214DB4A
:1038C800B1F5FA6FA8BF4FF4FA610FE0DE459C54DA
:1038D80004DA37F80C305B4227F80C300132032A3F
:1038E80005F101057FF450AFE5E71146DFF878E10F
:1038F800524D891A4FF47A736FF063065943C2F533
:10390800FA626423B1FBF2F191FBF3F23EF8120084
:1039180006FB0211013206B23EF91220921B5143F6
:1039280091FBF3F30344FB80484B1B88590639D5B8
:10393800474BDFED487AB3F904300A2293FBF2F3E0
:10394800454A12889B1A1BB208EE103AB8EEC88A8C
:1039580028EE278AB0EE480A08F088FCF0EE408A84
:10396800B0EE480A08F021FCB5F9023006EE903AAC
:10397800B5F90030F8EEE66A07EE903A20EE667A7E
:10398800F8EEE77AA7EEA87A67EE807ABDEEC77AF6
:10399800E6EEA87A17EE103AFDEEE77A2B8017EEDE
:1039A800903A6B802D4B2E4E1B88DFED2E0A358BFF
:1039B80000EE103A06F11C00B8EE400A012108F0AA
:1039C80091F9BCEEC00A96F826308DED000ABDF8D4
:1039D8000000B5FBF0F0451CADB2B584002B45D016
:1039E800B6F828B000231E4937F8138001F1320CCD
:1039F80001F12A093CF813E039F813202CF8138058
:103A0800CEEB080E12FB0BF20FFA85FA92FBFAF2D4
:103A1800964429F813E00133042BE4D1002381F8FC
:103A28002630088525E000BFF63100204417002025
:103A3800D417002018170020182E0020CC170020BB
:103A48000CFEFFFF9E0F002080240020B4200020E1
:103A5800C017002035FA8E3CFE0E0020D01600203C
:103A6800900F00206F12833ABE200020338D013B57
:103A78003385A54D288D03B2002B4FF0000312DDCE
:103A8800B5F924E0A14931F81320083112FB00F2FE
:103A980031F8131092FBFEF28A1A27F8132001332B
:103AA800042BEFD100E02B85994B1A6812F0020F16
:103AB800984678D0974BDFF850B21A68EB6B45F20E
:103AC8000721D31A8B426EDDCBF83C2005F0D6FFD8
:103AD800914BDFF880A21A78032A9946BAF8003089
:103AE80024D10A2B2ED90023282089F800300DF084
:103AF800A6FB05F0C3FF894B188805F0A9FF884B82
:103B08001A68D37890FBF3F001300828854BA8BFDA
:103B180008201870537980B213FB00F3A5F84030E1
:103B2800137913FB00F0A5F842000BE00A2B09D823
:103B380003237C4A89F8003000231370ABF8403027
:103B4800ABF8423099F80030734A012B0DD002D3FC
:103B5800022B1ED027E0B5F84020BAF800309A4270
:103B680021DD012389F8003011E0BAF80010B5F81A
:103B780042308B4202DD0223137011E0624BB3F82E
:103B880040300133994202DD002313700BE0082016
:103B980007E0B5F84230BAF8002001339A42E0DC79
:103BA80007200DF08DFBD8F8008018F4006F7DD049
:103BB800584B6A6C1B685448C2EB030945F207224C
:103BC800914573DD564AB7F906C0D2F800A04364A0
:103BD8009AF80A20544B554FB3F84E11012AACF508
:103BE8007A7C03D049D3022A22D048E0504B816C1A
:103BF8005A7B504B33F812204FF0080E92B291FBCB
:103C0800FEF3C91A8B18A0F84C20836440F6E442EE
:103C180093FBFEF39BB25343BAF80820C2EB13336D
:103C28004FF47A725343BAF9062093FBF2F325E076
:103C3800414ABAF808B01278C7F800B052071ED542
:103C480003F5C470CDF800C00DF08DFADDF800C0A2
:103C580020B918F0100F18BF4FF0000C32220CFBDF
:103C68000CF393FBF2F3BAF9062063445A434FF47A
:103C78007A7392FBF3F35B4400E000233B60D6E9E0
:103C880014013B6803FB09F94FF47A7399FBF3F9C4
:103C980010EB090241EBE973C6E9142310461946F3
:103CA800264A00230FF0BEF9254B1860254F0097D0
:103CB8003B6813F4805F52D018F0800F4CD0224B31
:103CC8001B789E0748D5214B1878042844D9002230
:103CD8001F4B02EB030E0521961C4FF00A0C122A0B
:103CE800D154F1B28EF801C004D0B0EB510F324676
:103CF800EED800E014215A18322002F8010CFF22F5
:103D08005A540F2029E000BF900F0020BA0F00205E
:103D1800D41F0020103400203C2000205422002012
:103D2800D81F002078000020D4170020E41F0020AE
:103D38003C2200204C22002032340020407E050026
:103D4800E81F0020DC160020F01F0020F61F0020CE
:103D5800042D0020DC1F00200A200DF0B1FAA74E28
:103D68003268002A58D0A649A64B08681F688742BF
:103D78008946984650D8A44BDFF89CA21878516819
:103D880010BB01201870BAF80030CB5C63B313780D
:103D9800013B00FA03F29D4BD3F8F8371A4201D1E0
:103DA8000DF074FA9A4B01221A700EF059FABAF80B
:103DB8000030CBB933681B78053B012B14D80DF0C4
:103DC80017FA944B18600FE04FF0000B83F800B01F
:103DD800BAF80030CB5C3BB158460DF057FA8C4B23
:103DE80083F800B00EF03CFA3268BAF80030526836
:103DF8008948D25CFE2A01D100230CE0FF2A02D1B7
:103E08000DF04AFA08E0D9F800600A2111FB0262B5
:103E1800C8F8002001330380804E3378580703D553
:103E28007F4B08221A8538E0009A1268D1075CBFD8
:103E380043F0010333707B4B1B781A0758BF337864
:103E4800734A5CBF23F001033370774B1B6813F090
:103E5800040F02D07549098851B97549098809B113
:103E68009B0705D4734B1B88003318BF012333B15C
:103E780002231370337823F00103337004E03178A0
:103E8800CF0758BF022313700DF0B2F96A4B1B68B5
:103E9800C01A002801DB0EF0E3F909F025FC674A97
:103EA80002921378002B78D0654F3B68002B00F006
:103EB800758738680DF0A6FA002800F06F87604B08
:103EC800604C18680DF09BFA092801D03F2858D19A
:103ED8004FF0000AD4F80080DFF888915646B8F110
:103EE800000F06D05848D9F80010424612F07EFF5D
:103EF80010B9CA4606B94E46544B09F110099945FE
:103F0800EDD3EEB1D6F800C0DAF8009023681CF8BB
:103F180003E019F80300704512D15A1C4A4958B9F0
:103F28002D2B09D8DFF81CE1CEF800204FF0200E29
:103F380001F803E0885403E001F803E02260E5E7B4
:103F480023680BB1564511D041480CF04BFC56453F
:103F580007D856F8100B0CF045FC09200CF03AFC79
:103F6800F5E73C480CF03EFC4FF000082368984504
:103F78009FD2354B13F808000CF02CFC08F101080F
:103F8800F4E72368002B40F02E87042840F02587AB
:103F98002D4808F0EBFD00F001BF00932E4B009A6E
:103FA8001A4492F84A10012940F0F2862B4F0099E2
:103FB8003A602B4ACB581360B9469046D8F80000AF
:103FC800DFF89CA00DF01EFA002800F0CD86DAF884
:103FD80000000DF014FAD9F8003093F84820834611
:103FE8001AB9242872D1012205E0012A3CD14D28B2
:103FF80014BF0022022283F848208DE0482E0020BA
:10400800A8170020402E00203C2E0020D4170020A6
:10401800D4330020D0310020442E00203234002038
:1040280000040048F01F0020EC1F00202834002066
:10403800B02500202E340020D8330020343400204E
:10404800F42C00209026002060260020A07C010887
:10405800DC950108E1950108282100209420002022
:1040680098200020C07A0108022A04D13C2814BFF5
:1040780000220322BFE7032A0AD140284FF000029A
:104088009FBF1A71DA715871987198BF0422B2E70C
:10409800042A08D19A7983F8490080EA020B83F848
:1040A80006B00522A7E7052A36D159791A7991422F
:1040B800997906D941409971511C197113441872A4
:1040C8002AE081420CBF0622002294E73378C34AD3
:1040D800590721D42328DAF8003011D10392029A23
:1040E800BF48AB6501211170BE490B600CF07AFB2B
:1040F800BD480CF077FB039A137843F00203137062
:10410800BA4B1B681B785B4501BFB94BB94A1A60AB
:10411800B94B04BFB94ADA60D9F80030DFF8FCA21D
:1041280093F848B0BBF1060F7FF448AF93F8490005
:1041380001F0C8FD002840F01186DAF8002092F856
:1041480049304C2B00F0DE8400F29280352B00F0D1
:10415800A6823CD82B2B00F0AC8422D8252B00F06B
:104168007F8404D8232B00F05F8200F033BE272B16
:1041780000F07D84292B40F02D860CF063FADFF8DF
:104188008082A8F880010CF05DFAA8F882010CF092
:104198004FFA88F884010CF055FAA8F8860100F067
:1041A800DABD2F2B00F04E8504D82D2B00F0868425
:1041B80000F010BE312B00F05A85332B40F00A86F0
:1041C8000CF036FA8E4B83F8920100F0C4BD412BF7
:1041D80000F0F2841AD8392B00F0588404D8372B11
:1041E80000F0F78400F0F6BD3C2B00F0DE803E2B9B
:1041F80040F0F0850CF01CFADFF8048288F8E00142
:104208000CF016FA88F8DF0100F0A5BD442B00F089
:10421800628525D8432B40F0DD850CF009FA002390
:10422800A36060710CF018FA08F050F80CF000FA6E
:1042380084F890010CF006FAA4F858010CF002FA80
:10424800A4F85A010CF0FEF9A4F85C010CF0FAF994
:10425800A4F880010CF0F6F9A4F8820100F07BBD07
:10426800482B00F092834A2B00F0758500F0B2BD10
:10427800D12B00F0B48320D8CC2B00F037820FD894
:10428800C82B62D004D84E2B00F0688400F0A2BD81
:10429800C92B00F07D83CA2B00F0C28000F09ABDC4
:1042A800CE2B00F06583C0F05A83CF2B00F08482B8
:1042B800D02B00F0498300F08DBDD82B00F045814C
:1042C8000BD8D32B3BD027D3D42B00F0CA82D62BC4
:1042D80040F080854FF00008B8E2F22B00F0098327
:1042E80012D8EF2B40F07685DFF82C81D8F80090B3
:1042F8000CF0A8F9A9F86200D8F800800CF0A2F92F
:10430800A8F8600000F027BDF32B00F0E884FA2B32
:1043180000F0378300F05EBD337803F0040303F048
:10432800FF08002B40F017850CF082F9344B022867
:1043380083F8CC0740F20E8383F8CC870AE30CF0AD
:1043480081F9304B188000F006BD92F805804FEADD
:104358005808B8F1120F03D904F04AFF00F0FBBC6B
:104368004FF00009C14507D20CF06CF905AB23F8F2
:10437800190009F10109F5E742460023434507DA28
:1043880005A931F81300204921F813000133F5E796
:10439800122A05D01C4B002123F812100132F7E72E
:1043A800012385F85C3000F0D6BCDFF86C90D9F8B2
:1043B80000800CF03DF918B10228A8BF022000E0E7
:1043C800012088F80000D9F800301B78022B0F4B29
:1043D80014BF0F4A0F4A1A6000F0BDBC32340020E7
:1043E80011960108F42C0020E1950108CC21002049
:1043F800FC9F0020EFBEADDE00ED00E00400FA05F2
:10440800D4170020FC0E0020D832002074000020B1
:1044180025AE0008B52201081817002094200020B6
:10442800DC4B1A681278022A4FF00009984670D1BE
:10443800D8F800A00CF0FCF807EE900AF8EE677ABE
:10444800B2EE048AC7EE887A0AEB890ACAED087ABE
:10445800D8F800A00CF0ECF807EE900A9FEDCE7AA1
:10446800F8EE677A0AEB890AC7EE877ACAED0B7A03
:10447800D8F800A00CF0DCF807EE900A9FEDC77A98
:10448800F8EE677A0AEB890AC7EE877A09F101091B
:10449800B9F1030FCAED0E7ACAD1B9F1070FD8F8EE
:1044A80000A01CD10CF0C4F807EE900AF8EE677A69
:1044B800C7EE887ACAED117AD8F800A00CF0B8F8DF
:1044C80007EE900AF8EE677AC7EE887ACAED127A94
:1044D800D8F800A00CF0ACF88AF84C0012E00CF008
:1044E800A7F8CA448AF80100D8F800A00CF0A0F890
:1044F800CA448AF80B00D8F800A00CF099F8CA440E
:104508008AF8150009F10109B9F10A0FC5D100F0BF
:1045180022BCD8F800A00CF08BF8CA448AF8010035
:10452800D8F800A00CF084F8CA448AF80B00D8F830
:1045380000A00CF07DF8CA4409F10109B9F10A0F8D
:104548008AF81500E5D100F006BC8146DFF8448200
:104558009FED928AD8F800A00CF074F807EE900A44
:10456800F8EE677A0AEB890AC7EE887ACAED087A04
:10457800D8F800A00CF066F807EE900AF8EE677A13
:104588000AEB890AC7EE887ACAED0B7AD8F800A038
:104598000CF058F807EE900AF8EE677A0AEB890AE9
:1045A800C7EE887A09F10109B9F1030FCAED0E7A4D
:1045B800CCD1B9F1070FD8F800A01CD10CF042F803
:1045C80007EE900AF8EE677AC7EE887ACAED117A94
:1045D800D8F800A00CF036F807EE900AF8EE677AE3
:1045E800C7EE887ACAED127AD8F800A00CF02AF83B
:1045F8008AF84C0012E00CF025F8CA448AF8010049
:10460800D8F800A00CF01EF8CA448AF80B00D8F8B5
:1046180000A00CF017F8CA448AF8150009F101093E
:10462800B9F10A0FC5D196E30CF002F813288246B7
:104638003FF692AEDFF85C91D9F800B00BF0F8FFC6
:104648000023574A0C2101FB0322117A814222D10F
:104658000FFA8AF80BEB8808137888F881300BF08A
:10466800E7FF88F882000BF0E3FF88F883000BF07F
:10467800DFFF4C4B4C4A1A6088F884004B4BD9F842
:1046880000001860002181300CF05CFD484B80F080
:10469800010018705FE301331C2BD2D15CE60BF0EC
:1046A800C7FF0B2880463FF657AE3A4BD3F8009029
:1046B8000BF0BEFF03283FF64FAE0BFB089B8BF8B1
:1046C800D6000BF0B5FF8BF8D1000BF0B1FF8BF8DB
:1046D800D2000BF0ADFF8BF8D3000BF0A9FF8BF8DD
:1046E800D4000BF0A5FF8BF8D50034E35379092BE0
:1046F8007FF632AE019BD3F800800BF099FF019B47
:1047080088F80000D3F800800BF092FF88F80100C9
:104718000BF08EFF019B64281B68A8BF64201871EA
:104728000BF086FF019B64281B68A8BF64205871A2
:104738000BF07EFF019BFF281B68A8BFFF20987124
:104748000BF076FF019B6428D3F8008028BF642013
:1047580088F807000BF06CFF019B88F80200D3F87B
:1047680000800BF065FF019B88F80300D3F80080F8
:104778000BF068FFDAF80030A8F80A005B790A2B1A
:1047880040F2E9820B4BD3F800800BF051FF88F818
:104798000800E0E2181700200000C84200007A4430
:1047A800F0730108F40E002014190020F80E002000
:1047B8000A000020441700200BF044FF6FF4AF629A
:1047C80083189BB2C62B9CBFD64BA3F896010BF05F
:1047D80039FFA4F840010BF035FFA4F842010BF0B3
:1047E80031FFA4F844010BF02DFFA4F8D8010BF019
:1047F8001FFF84F8ED010BF01BFF0BF019FF84F885
:10480800EE010BF015FF84F885010BF011FF84F819
:1048180092010BF00DFFC44BD3F800800BF012FF90
:1048280000EB80004000A8F85E000BF001FF84F860
:104838007A010BF0FDFE84F87E010BF0F9FE84F896
:104848007D010BF0F5FE84F87F0184E20BF0FAFE9F
:10485800B64B23F8180008F10108B8F1080FF5D194
:1048680079E253790F2B7FF477AD0BF0E1FE07283F
:1048780080463FF671ADDFF8B092D9F800A00BF092
:10488800E1FE0E2303FB08F8C244AAF82101D9F877
:1048980000A00BF0D7FEC244AAF82301D9F800A063
:1048A8000BF0D0FEC244AAF82501D9F800A00BF0FD
:1048B800BFFEC2448AF82701D9F800A00BF0B8FE61
:1048C800C2448AF82801D9F800A00BF0B1FEC2440E
:1048D8008AF82901D9F800A00BF0AAFEC244D9F839
:1048E80000908AF82A010BF0B7FEC844C8F82B01DB
:1048F80031E20BF09DFE0F2880463FF62DADC8EB48
:10490800C8080BF095FE04EB080303F1D00883F800
:10491800D0000BF08DFE88F801000BF089FE88F8B6
:1049280002000BF085FE88F803000BF081FE88F882
:1049380004000BF07DFE88F805000BF079FE88F87E
:1049480006000CF00DFF06E233785B0700F10382E6
:104958000AF02CFC07F0ECFC07F0A8FDFBE133782B
:10496800580700F1F881724B4FF4C8721A80F2E1CF
:104978003378590700F1EF816E4A137843F0040346
:104988002BE033785A07E5D524E20AF0E5FAE2E1AC
:104998000BF04EFE674B1A7810B142F0020201E0AC
:1049A80022F002021A700BF043FE634BDFF8A88175
:1049B80018700BF051FEC8F800000BF04DFEC8F857
:1049C80004000BF03FFE5D4B18800BF03BFE5C4B88
:1049D8005C4A1880137843F002031370BBE10BF0B4
:1049E80027FE83460BF038FE82460BF035FE8146E3
:1049F8000BF032FE80460BF025FE0BF023FE0BF089
:104A080017FEBBF1000F14D14F4B1020C3F800A0C4
:104A1800C3F8049007F032FC464A137843F00103C8
:104A28001370B8F1000F00F09681484BC3F800806E
:104A380091E1BBF1100F40F08E81454BC3F800A007
:104A4800C3F80490B8F1000F02D0404BC3F80080BF
:104A58003F48404B0222011D1A7005F0F3FB7AE132
:104A6800304B98600BF0F8FD07F030FC73E10BF069
:104A7800E9FDDFF8B080A8F858010BF0E3FDA8F8CD
:104A88005A010BF0DFFDA8F85C0164E10BF0D0FDE2
:104A9800DFF8908088F87A010BF0CAFD88F87E016B
:104AA8000BF0C6FD88F87D010BF0C2FD88F87F0188
:104AB80051E10BF0BDFD1B4B58714CE10BF0B8FDFB
:104AC80084F890010BF0BEFDA4F89A010BF0BAFD32
:104AD800A4F896010BF0B6FDA4F898010BF0A8FD18
:104AE8003B6884F891015B79DFF83880082B40F245
:104AF80032810BF0A7FDA8F89C010BF0A3FDA8F8E4
:104B08009E0128E10BF094FDDFF8188088F8D601A3
:104B18000BF08EFD88F8D7010BF094FDA8F8D801AA
:104B280019E100BFD417002018170020DA2C002044
:104B3800B0250020F01F0020F61F0020F41F0020E1
:104B4800F21F00204A1700204C1700205C17002095
:104B580054170020000F0020F81F002092F805804D
:104B68000323B8FBF3F8B8F1120F3FF6F5ABDFF803
:104B78004C934FF0000AC24580F0ED800BF058FDD1
:104B880089F8A0010BF05EFD40F2ED23984205DDA7
:104B980040F6CA039842A8BF184601E040F2EE204A
:104BA800A0F2EE2019230AF1010A90FBF3F009F1B3
:104BB800020989F89F01DEE781460BF039FDBF4BFA
:104BC8004B4409F10109B9F1080F83F88801F4D1C0
:104BD800C1E053794FF00709B3FBF9F9C9EBC902F2
:104BE8009B1A13F0FF0F7FF4B7AB5FFA89F909F14D
:104BF800FF395FFA89F9B9F1FF0F00F0AC800BF0CB
:104C080017FD5FFA80FA4FFA8AF003F0B9FA804686
:104C180000283FF4A1AB80F800A00BF013FDA8F822
:104C280002000BF005FD88F804000BF001FD88F880
:104C380005000BF0FDFC88F807000BF0F9FC88F87C
:104C48000600D4E7DFF8748208F140090BF0FAFC9B
:104C5800A8F8AC020BF0ECFC88F8AE020BF0E8FC0C
:104C680008F1040888F8AB02C845EFD173E00BF0EF
:104C7800DFFC1F2880463FF66FAB3B685B79082B4B
:104C88007FF46AAB0BF0DEFC08F18A0804EB8808B5
:104C980000F03F00A8F806000BF0D4FCB8F8063086
:104CA800800100F4FE501843A8F806000BF0C0FC81
:104CB800000188F804000BF0BBFC98F8043000F001
:104CC8000F00184388F804000BF0B2FC88F80500C0
:104CD8000AF088FF3FE0012385F85D303BE00BF0E8
:104CE800A7FCFF28814622D100238DF813309DF8B8
:104CF8001330072B14D89DF81300714A9DF8133010
:104D080052F8300002EBC30301215B68994089B275
:104D1800042203F047F99DF813300133DBB2E4E7CE
:104D280068484FF40041002203F03CF913E00728DB
:104D38003FF612AB00200BF0CDFC0BF0A7FCD8F827
:104D480000000CF056FB18B932200CF078FAF6E7A0
:104D5800484603F035F900200BF0BCFC0BF096FC3C
:104D68003B68002283F8482095F85D3083B1564BA4
:104D7800009A98580CF03DFB18B932200CF05FFAF5
:104D8800F5E70CF0ADFC07F0A9FA504B504ADA6091
:104D9800009B4C33982B00937FF400A94D4B1B6864
:104DA8009B060FD54C4B2A6E1B689A1A002A09DB02
:104DB8004A4A1278042A81BF03F51233484A03F598
:104DC800F8731366474B9B68002B00F0AC8046488D
:104DD8009847A8E004F00CFAC0E70C2820D1434813
:104DE8000BF000FD1AE00C28F9D00A281CD1404E1F
:104DF80040480BF0F7FC3046232111F0E2FF08B1E0
:104E0800801B2060236893BB39482360002130222F
:104E180011F0A4FF029B1B78002BBFD036480DE091
:104E28007F2812D1FFF745B80D28E0D07F2809D197
:104E3800013B2F4A314823600021D1540BF0D2FCAA
:104E4800FFF737B82F2B3FF634A8A0F12002D2B2D3
:104E58005E2A3FF62EA813B920283FF42AA85A1C28
:104E68002260234AD0540BF0B5FCFFF722B85A1E33
:104E7800B15C202901D11346C5E71D4A23600021F2
:104E8800D1541F4B1F4ED3F800A0D6F800B0DFF85E
:104E98006090584611F0A2FF80464246484659465F
:104EA80011F0A4FF184A28B919F8083053445B7860
:104EB80058072BD010369642E7D32FE0D41700209E
:104EC80040990108000800482821002000ED00E072
:104ED8000400FA05EC1F002010340020F61F002003
:104EE800900F002018250020F40F0020E6950108F7
:104EF800602600204CA50108E19501080D960108DF
:104F080080000020C07A0108A07C0108964205D2E2
:104F180008F10100F3684844984702E004480BF0A0
:104F280061FC002370E70FB0BDEC028BBDE8F08F89
:104F3800F195010810F80A3C0133DBB20A2B84BF53
:104F480010F8131C044A00F80A3C82BF002322F818
:104F5800113000F80A3C7047FC320020334A136CC9
:104F680090681944081A40F68C23984270B5134685
:104F78009160D06051603BD9127893F945108A420C
:104F880010460BD1111F082908D893F84610182984
:104F980001D8013103E083F8442002E0002183F8BE
:104FA800461093F944402149A24219D191F847404B
:104FB800B4B10C310024944206DA1D4D51F8046F47
:104FC80025F814600134F6E70C2805D018490024A8
:104FD80021F810400130F7E71648017801310170D7
:104FE80083F84520002201211A7083F8471070BD0C
:104FF80092F84710C9B1A0F2EF2440F2DA518C427E
:1050080008D811780B2905D80B1D0131117042F809
:10501800230070BD002283F84720074B03F13002BC
:10502800002143F8041F9342FAD170BD20010020EB
:10503800FC3200203D0600202C010020024A136C9F
:10504800013319441164704720010020024B53F8C2
:1050580020301B68196070474C2E0020064B53F80F
:1050680020301A681B89A1F57A7159434FF47A7375
:1050780091FBF3F1116070474C2E0020054B9842CC
:105088000CBF054A054A138801339BB213800020E0
:10509800704700BF00540040D8160020DA160020E0
:1050A800F0B5046D8668236823F0010323608379D3
:1050B800054613F0020F40790CBF4FF0000E4FF475
:1050C800005E13F0040F14BF4FF48067002710F040
:1050D800010F14BF042100218307206820F001007C
:1050E8002060626822F440524EEA0202626022683E
:1050F80022F4B05323F00C0348BF41F008013B43AE
:105108000B432360A36895B023F44073A3606846FB
:1051180004F068FA284B9C4201D10C9B0EE0274B07
:105128009C4201D10D9B09E0254B9C4201D10E9B6D
:1051380004E0244B9C420CBF0F9B109B2268A8796B
:10514800170448BF5B00B3FBF6F206FB1233B3EB60
:10515800560F236828BF01321E0441BF4FF6F07373
:10516800C2F34201134041EA03026B7992B213F091
:10517800020FA28100F0010114BF4FF40032002297
:10518800DC0748BF42F480322B6D11B159680A43DD
:1051980002E0596821EA02025A609A6801074CBF86
:1051A80042F0080222F008029A601A6842F00102EE
:1051B8001A6015B0F0BD00BF00380140004400403F
:1051C80000480040004C00402DE9F0471E46A64B21
:1051D8008CB09842894690469DF8505040F08580A2
:1051E800A24BA34A1A60A34A5A6102F580729A61D7
:1051F8004FF48072DA601A619F4A1A63143A5A634C
:10520800A2F54842203ADA6404329A64C3F8088066
:1052180018659A4B9A6942F480429A615A6942F039
:1052280001025A6102238DF80830032315F0010AA0
:105238008DF809304FF000038DF80A3014BF0223AF
:1052480001232C078DF80B3019D54FF090444FF4FB
:10525800007701978AF001038DF80A30636A23F01A
:10526800F0036362636A43F070036362204601A936
:1052780004F07CF9BAF1000F27D1A76125E0B00747
:1052880010D50CA94FF4007341F82C3D4FF0904015
:10529800436A23F0F0034362436A43F070034362B6
:1052A80004F064F9F10710D50CA94FF4806341F8B4
:1052B8002C3D4FF09040436A23F470634362436A85
:1052C80043F4E063436204F051F90E238DF8003093
:1052D8000022012368468DF801308DF802208DF8F0
:1052E8000330624C0CF0BEFC0BE1654B984276D162
:1052F800644B5F4A1A604FF48072DA601A61624A3E
:105308005A6102F580729A615C4AC3F80880186590
:10531800D36943F40033D36102238DF808300323A3
:1053280015F0010A8DF809304FF000038DF80A30A6
:1053380014BF022301232A078DF80B3019D54FF02B
:1053480090444FF4804701978AF001038DF80A30A2
:10535800636A23F070636362636A43F0E0636362C5
:10536800204601A904F002F9BAF1000F27D1A7617C
:1053780025E0B30710D50CA94FF4804341F82C3D24
:105388004FF09040436A23F070634362436A43F0EE
:10539800E063436204F0EAF8F70710D50CA94FF46C
:1053A800004341F82C3D4FF09040436A23F070438E
:1053B8004362436A43F0E043436204F0D7F826238C
:1053C8008DF800300022012368468DF801308DF8F1
:1053D80002208DF803302B4C0CF044FC91E02B4B51
:1053E800984240F00F812A4B214A1A604FF480728C
:1053F800DA601A61274A5A6102F580729A611F4A77
:10540800C3F808801865D36943F48023D361022365
:105418008DF80830032315F0010A8DF809304FF094
:1054280000038DF80A3014BF022301232C078DF8DE
:105438000B3033D5184C4FF4806701978AF001037D
:105448008DF80A30636A23F470636362636A43F415
:10545800E0636362204601A904F088F8BAF1000FFE
:1054680040D1A7613EE000BF00380140C42D0020B4
:105478009C730108F80F00205800024000100240F9
:1054880000440040702D0020F81100200048004022
:105498001C2D0020F813002000040048B0070FD589
:1054A8000CA94FF4806341F82C3D5848436A23F413
:1054B80070634362436A43F4E063436204F056F85E
:1054C800F1070FD50CA94FF4006341F82C3D4F4864
:1054D800436A23F470434362436A43F4E0434362FC
:1054E80004F044F827238DF8003000220123684691
:1054F8008DF801308DF802208DF803300CF0B2FBE6
:10550800434CC4F82C900027012384F844302762C8
:10551800E761A76267626671C4F80880A5712046D2
:10552800FFF7BEFDF20734D5236B002B2AD001A864
:1055380003F06DFFE36C01934FF480530A938023CB
:105548000693E368ADF8103020230993206B636954
:1055580002930B97059707970897039703F082FF25
:1055680001A9206B03F060FF236B216D1A6842F0DC
:1055780001021A608A6842F040028A605B689BB246
:10558800236406E0236D20221A621A6842F0200282
:105598001A60B3072FD5636B43B301A803F037FF35
:1055A800A36C01934FF480530A93802306932369D5
:1055B800ADF8103000251023606B03930B9505950B
:1055C80007950895099503F04DFF606B01A903F055
:1055D8002BFF636B1A6842F002021A60226D5D604D
:1055E8005D60936843F08003936004E0226D136864
:1055F80043F080031360226D136843F001031360C6
:10560800204600E000200CB0BDE8F0870004004808
:105618001C2D00201FB50123ADF808300023ADF87C
:105628000C30ADF80A30094BADF804101B78ADF812
:105638000620012B08BF032301A908BFADF80C30D1
:1056480003F00EFE05B05DF804FB00BF1C0100204E
:1056580038B510F80E2C50F8043C044652B9012213
:1056680000F80E2C20F80C1C997A18680222BDE864
:105678003840CFE730F80C2C20F80A1C891A89B278
:1056880020F8081C074A10F80F0C002522F8101003
:1056980004F80E5C1868997A2A46FFF7BBFF04F8ED
:1056A800065C38BDFC320020044B53F820301BB197
:1056B80007289CBF1B681960704700BF480200207C
:1056C800074A13689B060AD5064B0021197006493C
:1056D80008684FF6FE7303400B6020235360704741
:1056E80000000240313400201C0002402DE9F04740
:1056F8006B4DD5F800366B490A78581C02F0FF0646
:105708008E460AB10346F6E7C5F8003695F80886CE
:1057180095F8090695F80A26D5F80C36374639B2B1
:10572800202900F09B80DFF88CC10CEB81033CF84A
:105738002110DC789B78C3F1FF039BB2002B65D066
:10574800C3F1FF0363434FF03C0C1B12B1FBFCF9A0
:10575800B9F1050F5DD8DFE809F0030B1A293A4AB9
:10576800E01ADAB24143B1FBFCF01044C0B251E098
:10577800B1FBFCF00CFB101189B2DAB2C1F13C01AB
:10578800E31A4B432046B3FBFCFC94442CE0B1FBEA
:10579800FCF00CFB10115FFA83F8E21A89B24A4355
:1057A800B2FBFCF24244D2B2204632E0B1FBFCF933
:1057B8000CFB191189B25FFA83F8E01AC1F13C01B8
:1057C8004843B0FBFCF04044C0B2224621E0B1FBA4
:1057D800FCF80CFB1811D8B289B2E31A01FB03F2EA
:1057E800B2FBFCFC224684445FFA8CF412E0B1FB65
:1057F800FCF80CFB181189B2D8B2C1F13C01E31ACC
:105808004B43B3FBFCF20244D2B203E022462046EB
:1058180000E044464FEA042C4CEA004C4CEA020CE7
:10582800172306F117014FF0010808FA03F8C91AFF
:1058380018EA0C0F89B2DFF8808014BF4FF0110905
:105848004FF0090913F1FF3308F80190E9D218362F
:105858000137B6B2BFB2144BA04660E785F80A26F6
:10586800C5F80C36114AA5F8061601238EF8003043
:105878000F4985F8088640F22A3385F80906A5F805
:105888000466536000234B620B889BB243F001030C
:105898000B80136843F001031360BDE8F08700BF75
:1058A800F80F002031340020001600201C000240B0
:1058B800002C01403A0D0020E102002073B5064695
:1058C8000D46002401232A88A34013421AD0AA783F
:1058D800009302F003038DF80430EB78022B03D019
:1058E800032B0CBF032301238DF805303046C2F388
:1058F80001136946C2F381028DF806308DF807203E
:1059080003F034FE0134102CDCD102B070BD2DE957
:10591800F04F754E96F8105607460C4687B011465C
:105928009A4600686B1C914622464FF0020B86F897
:1059380010360BF085FA3B897868ADF8043001A978
:105948008DF806B08DF807B0FFF7B8FF0023ADF863
:105958000A30ADF81230ADF8163070230193BA7AD8
:105968003C68CDF80CA0012306F214682D01ADF8AF
:1059780008304FF48073A844ADF810B0ADF8143077
:105988000C2A7ED8DFE802F0077D7D7D0F7D7D7DC6
:10599800387D7D7D5E00204601A903F0E6FCA36901
:1059A80043F0080326E0236A504823F010032362DB
:1059B800236A6168A26922F0807222F4E642844276
:1059C80042F4E04206D000F50060844202D043F081
:1059D800300307E023F0E00321F4406143F0300393
:1059E80041F480616160A261C4F838A02362A369B0
:1059F80043F40063A36144E0236A3C4823F48073C2
:105A08002362226A6168E369844223F0730343F0E6
:105A1800700306D000F50060844202D042F4407260
:105A280007E022F4606221F4405142F4407241F4EC
:105A380080516160E361C4F83CA02262E36943F0ED
:105A480008031DE0236A294823F480532362226A4D
:105A58006168E369844223F4E64343F4E04342F493
:105A6800405203D000F50060844201D141F48041E6
:105A78006160E361C4F840A02262E36943F4006313
:105A8800E3613A7B3B681AB15A6C42F400425A64AB
:105A98001A8892B242F001021A80BA7A0C2A19D8EE
:105AA800DFE802F0071818180B1818180F1818183C
:105AB8001300721903F134010AE0721903F1380175
:105AC80006E0721903F13C0102E0721903F140018A
:105AD800C2F8141635444046A5F81C96C5F8183681
:105AE80007B0BDE8F08F00BFF80F0020002C014080
:105AF800F8B53A4E3A4C4000C7B24FF420453068EA
:105B0800C4F8D456D0F818E01EF4004F05D0AE46BD
:105B1800013DBEF1000FF5D116E0D0F804E0314D9B
:105B28000EEA050545F490353D4345604FF42045A0
:105B3800C4F8D456D0F818E01EF0020F2DD1AE46A6
:105B4800013DBEF1000FF5D1C4F8D4561FE0294637
:105B5800013D0029F8D081694906F8D5C4F8D45622
:105B680020494568294041F0007141F4105141EA4B
:105B78000241394341604FF42041A2B13068856940
:105B88006D071ED411F1FF31F9D2C4F8D416FFF70E
:105B980075FA003018BF0120F8BD4FF42045816226
:105BA800C4F8D456D7E73068C4F8D4160B468269CF
:105BB80092060CD41A46013B002AF8D1C4F8D43610
:105BC800E5E7416A03F8011B013AD2B2D3E7C4F80A
:105BD800D4362023C3610120F8BD00BFD4160020AD
:105BE800F80F0020009800FC400070B5C5B232489C
:105BF800324B00684FF42044C3F8D4468669360413
:105C080004D52646013C002EF8D113E046682C4CFA
:105C1800344044F0807444F490342C4344604FF48E
:105C28002044C3F8D4468669B60729D42646013CE1
:105C3800002EF8D1C3F8D4461CE02146013C0029C7
:105C4800F8D081690E06F8D544681D49214041F015
:105C5800007141F48031294341604FF42041C3F879
:105C6800D4168469A40711D40C460139002CF8D144
:105C7800C3F8D416FFF702FA003018BF012070BD30
:105C88004FF420448162C3F8D446DAE782624FF4C5
:105C98002042C3F8D4268169890606D41146013A00
:105CA8000029F8D1C3F8D426E4E7C3F8D426202382
:105CB800C361012070BD00BFD4160020F80F00207A
:105CC800009800FC2DE9F0472DED028B4B28A0B081
:105CD800044600F04E8600F2B580302800F0DA86DF
:105CE80051D8222800F0978423D8032800F0638134
:105CF80014D8012800F05381022840F03687042088
:105D08000AF0E8FC42200AF0B0FC54200AF0ADFC8E
:105D180046200AF0AAFC4C2000F060BE042800F0DF
:105D28005581052840F021871A200AF0D3FC002469
:105D38005DE1282800F0EB8515D8242800F0D285ED
:105D4800262840F01287B64C06200AF0C3FCB4F8A7
:105D580058010AF0C2FCB4F85A010AF0BEFCB4F8C3
:105D68005C0100F0BCBD2C2800F0E4852E2800F072
:105D780060862A2840F0F98601200AF0ABFCA84B7F
:105D8800587900F02BBE3D2800F020831ED8362815
:105D980000F035860BD8322800F01A86342840F0F7
:105DA800E48648200AF096FC002500F056BC3A2804
:105DB80000F0C0823B2800F02784382840F0D586C0
:105DC80004200AF087FC964C00F092BD452800F0AC
:105DD800B98627D8402800F00486422840F0C586B6
:105DE8008F4C10200AF076FC60790AF03EFCA0681F
:105DF8000AF07CFC94F890010AF037FCB4F85801DA
:105E08000AF06BFCB4F85A010AF067FCB4F85C01BC
:105E18000AF063FCB4F880010AF05FFCB4F8820170
:105E280000F05DBD472800F06B86C0F05886492811
:105E380040F09B8602200AF04DFC7A4BB3F87000C4
:105E480000F04DBD702800F0F4825AD8692800F09F
:105E58004E822AD8652800F0FD8015D84D2800F01C
:105E68009785642840F0818607200AF033FCE720F4
:105E78000AF0FBFB6A4B58790AF0F7FB00200AF09E
:105E8800F4FB042000F06DBE672800F0B38100F237
:105E9800218212200AF01EFC634B1B88B3F5806F29
:105EA8008CBF08250125002487E16C2800F0328288
:105EB80017D86A2800F096846B2840F0568605208B
:105EC8000AF008FC594B18880AF007FC584B188848
:105ED8000AF003FC534B93F87A0000F0010000F03D
:105EE8007DBD6E284F4D00F02C8200F27A8206208C
:105EF8000AF0F0FB686E0AF0F9FB4E4B188800F0C8
:105F0800EEBC782800F0838119D8742800F0C68385
:105F18000BD8722800F02684732840F026860820C3
:105F28000AF0D8FB012400F056BC762800F07A84E9
:105F380000F2F8832F200AF0CDFB3F4C5CE3A42845
:105F480000F0998414D87B2800F0FC82A02840F047
:105F58000C860C200AF0BEFB384B18680AF0C6FB0A
:105F6800374B18680AF0C2FB364B186800F0F9BDC9
:105F7800F12800F08881FE2800F0A484F02840F081
:105F8800F485284C04200AF0A5FBA36CB3F8620042
:105F98000AF0A3FBA36CB3F8600000F0A0BC0320D8
:105FA8000AF098FB00200AF060FB20460AF05DFB2F
:105FB8000D2000F013BD0AF08DFB02200AF055FBFE
:105FC80001200AF052FB012000F008BD06200AF06B
:105FD80081FB49200AF049FB52200AF046FB432086
:105FE8000AF043FB46200AF040FB00F077BC164B52
:105FF800185D01340AF039FB0B2CF8D10024134B3F
:10600800185D01340AF031FB082CF8D10024104B3C
:10601800185D01340AF029FB072CF8D100F0A3BD64
:10602800D4170020D01600201C0000206A20002071
:106038006C200020B8170020BF730108ACF7FF1FC1
:10604800B0F7FF1FB4F7FF1F2B9301083793010820
:106058000F930108CD4C0B200AF03CFB20880AF076
:106068003CFB6268CA4B9A420CBF2089608980B2A7
:106078000AF033FBC74B1B68C3F3C000C3F38002AD
:10608800800040EA4200C3F340021043C3F34012C9
:1060980040EAC20003F0100318430AF01EFBBE4B8F
:1060A8001A88E368247C02F0080103F4475949EA96
:1060B800010903F4804149EA010903F4004149EA6E
:1060C800010903F4803149EA010903F4003149EA7E
:1060D800010903F4802149EA010903F4002149EA8E
:1060E800010903F4801149EA010903F0007349EA40
:1060F8000303DFF8D49299F8009012F0010FC9F366
:10610800800914BF4FF002084FF0000843EA090362
:1061180012F0020F43EA080314BF4FF0040C4FF0CB
:10612800000C12F0040F43EA0C0C14BF4FF0100ED1
:106138004FF0000E12F0400F14BF202700274CEA42
:106148000E0E12F0100F14BF4FF4007600264EEA20
:10615800070712F0200F14BF4FF4806500253E4357
:1061680012F4807F14BF4FF400600020354312F40E
:10617800007F14BF4FF400110021284312F4806FF0
:1061880041EA000114BF4FF0806300230020194347
:106198000346A3420AD2814A9D5C012202FA05F510
:1061A8000D421CBF9A4010430133F2E70AF09EFAF1
:1061B8007B4B93F8CC0700F011BC7A4B33F91400F1
:1061C80090FBF5F0013480B20AF087FA032CF4D181
:1061D8006E4CA08D0AF081FAE08D0AF07EFA208ECE
:1061E8000AF07BFA608E0AF078FAA08E0AF075FA47
:1061F800E08E74E310200AF06DFA00246A4B185DF3
:1062080001340AF032FA102CF8D100F0ACBC70203E
:106218000AF060FA00265D4D0E24AB6C74432344EB
:106228000136B3F821010AF058FAAB6C2344B3F8ED
:1062380023010AF052FAAB6C2344B3F825010AF0A3
:106248004CFAAB6C234493F827010AF00EFAAB6CB6
:10625800234493F828010AF008FAAB6C234493F816
:1062680029010AF002FAAB6C234493F82A010AF0D8
:10627800FCF9AB6C1C44D4F82B010AF037FA082E51
:10628800C9D100F070BC7020454C0AF023FA04F123
:10629800700594F8D0000AF0E8F994F8D1000AF0F3
:1062A800E4F994F8D2000AF0E0F994F8D3000AF07F
:1062B800DCF994F8D4000AF0D8F994F8D5000AF07B
:1062C800D4F9073494F8CF000AF0CFF9AC42E0D102
:1062D80000F049BC10200AF0FDF90024334B185D8A
:1062E80001340AF0C2F9102CF8D100F03CBC304D52
:1062F8002878400000F0FE000AF0ECF900242B7822
:106308009C4280F030842B4B33F814000AF0E5F9F6
:106318000134F4E7284C06200AF0DCF920880AF05A
:10632800DCF960880AF0D9F9B4F904300A2093FB43
:10633800F0F029E004200AF0CDF9144B986E00F033
:1063480010BC07200AF0C6F91C4B1888FF28A8BF04
:10635800FF20C0B20AF089F9194B186880F31000C1
:1063680080B20AF0BAF9B5F86C000AF0B6F90C4B2D
:1063780093F88521134B186822B10A23584380F3F8
:10638800100001E000F30F0080B2A8E2D016002050
:1063980000540040EC1F0020B4200020E11600202B
:1063A800D4170020B2170020081700201C1700205F
:1063B800C4210020F6310020C0170020DC1F002077
:1063C800E81F0020E41F002032340020C44C0220C3
:1063D8000AF080F994F8E0010AF047F994F8DF012F
:1063E800FCE20B200AF076F96B6F18780AF03DF999
:1063F8006B6F58780AF039F900266B6FB94C334443
:10640800013618790AF031F9032EF6D1636FD8797D
:106418000AF02BF9636F98780AF027F9636FD87838
:106428000AF023F9636F58890AF057F9636F187AED
:10643800D4E2AC4C1E200AF04DF9A36C1B78022B59
:106448004FF000056BD1A36C03EB850393ED080AAD
:10645800B2EE048A20EE080A0FF08AFA80F30800E8
:10646800C0B20AF002F9A36CDFED9F7A03EB850353
:1064780093ED0B0A20EE270A0FF07AFA80F3080052
:10648800C0B20AF0F2F8A36CDFED987A03EB85034B
:1064980093ED0E0A20EE270A0FF06AFA80F308003F
:1064A800C0B201350AF0E1F8032DCCD1072DA36C59
:1064B80023D193ED110A20EE080A0FF059FA80F360
:1064C8000800C0B20AF0D1F8A36C93ED120A20EECE
:1064D800080A0FF04DFA80F30800C0B20AF0C5F8B8
:1064E800A36C93F84C3000EE103AB8EE400A0FF067
:1064F8003FFA80F30800C0B20BE02B4458780AF04A
:10650800B4F8A36C2B44D87A0AF0AFF8A36C2B44E8
:10651800587D01350AF0A9F80A2DC7D123E3A36CE9
:106528002B4458780AF0A1F8A36C2B44D87A0AF0C7
:106538009CF8A36C2B440135587D0AF096F80A2D77
:10654800EDD110E33C200AF0C5F80024654D9FED1D
:10655800678AAB6C03EB840393ED080A20EE080A04
:106568000FF006FA80B20AF0B8F8AB6C03EB8403BC
:1065780093ED0B0A20EE080A0FF0FAF980B20AF040
:10658800ACF8AB6C03EB840393ED0E0A20EE080A1B
:106598000FF0EEF9013480B20AF09FF8032CD5D140
:1065A800072CAB6C16D193ED110A20EE080A0FF0F8
:1065B800DFF980B20AF091F8AB6C93ED120A20EE85
:1065C800080A0FF0D5F980B20AF087F8AB6C93F897
:1065D8004C000BE0234458780AF07FF8AB6C234456
:1065E800D87A0AF07AF8AB6C2344587D01340AF063
:1065F80074F80A2CD4D1B6E214F8010F002800F080
:10660800B2820AF032F8F7E701200AF063F8354B56
:106618009B6C1878E2E150200AF05CF80025314BB9
:106628009C6C334B04EB85040C2194F8812001FB0E
:106638000233013593F838000AF017F894F882000D
:106648000AF013F894F883000AF00FF894F884001D
:106658000AF00BF8142DE2D185E2224B9C6C06233C
:1066680003FB0544013594F8D60009F0FEFF94F8C1
:10667800D10009F0FAFF94F8D20009F0F6FF94F877
:10668800D30009F0F2FF94F8D40009F0EEFF94F873
:10669800D50009F0EAFF0C2DDFD164E24FF00008C5
:1066A800012600270F4B1A7C974232DA1133002457
:1066B800FA5C0F4D0C2305F130016343595C91429C
:1066C80007D12B44586B10F089FB82462EB9B1468E
:1066D80010E001341C2CECD119E0804417E000BF15
:1066E800D4170020D01600200000C84200007A44C9
:1066F800C0730108D1450ADA0C2303FB04535B6B12
:1067080013F8090009F0B1FF09F10109F2E70137AF
:10671800C8E7002E00F027825FFA88F009F0DAFF58
:106728000026BEE7CE4D287C09F0D4FF00242B7C40
:106738009C4280F01882CB4BE65C0021CA480C22B0
:1067480000F1300702FB01F3DA5DB24205D10344E0
:1067580093F8380009F089FF02E001311C29EDD1D6
:106768000134E4E7C14C162009F0B4FFB4F89601EF
:1067780009F0B3FFB4F8400109F0AFFFB4F84201E3
:1067880009F0ABFFB4F8440109F0A7FFB4F8D80149
:1067980009F0A3FF94F8ED0109F067FF002009F064
:1067A80064FF94F8EE0109F060FF94F8850109F0A0
:1067B8005CFF94F8920109F058FF002009F055FF9A
:1067C800A74B9B6C0A20B3F95E3093FBF0F080B2C4
:1067D80009F083FF8CE0E0B2013409F046FF092C90
:1067E800F9D1C0E1102009F075FFA14BA14C187830
:1067F80000F0020009F039FF9F4B187809F035FFC7
:10680800206809F073FF606809F070FF9B4B1888D7
:1068180009F063FF9A4B188809F05FFF904BB3F8B3
:1068280078005CE009F004FF0746122009F052FFE7
:106838008B4C1FB9E66FD4F8805007E0102F13BFB8
:106848000025D4F88460D4F888502E46384609F0DC
:106858000CFF304609F04AFF284609F047FFD4F8F4
:106868008C0009F043FF002009F037FF002009F0F1
:1068780034FF0020B2E07A4D95F890008000013096
:10688800C0B209F027FF95F8900009F0EEFE002449
:106898002E4696F890309C4280F06581794D285DAF
:1068A80009F0E3FE05F11003185D09F0DEFE05F1BD
:1068B80020033035185D09F0D8FE285D09F0D5FEB3
:1068C8000134E6E7082009F005FF002009F005FF7C
:1068D800002009F002FF002009F0FFFE002009F067
:1068E800FCFE40E1042009F0F5FE604B986838E1B1
:1068F80094F87A0109F0B9FE94F87E0109F0B5FE22
:1069080094F87D0109F0B1FE94F87F0166E0574CD8
:10691800072009F0DFFEB4F8800109F0DEFEB4F8C4
:10692800820109F0DAFE94F8840109F09EFEB4F8B9
:106938008601D4E74D4C0C2009F0CCFE94F8900168
:1069480009F093FEB4F89A0109F0C7FEB4F896016D
:1069580009F0C3FEB4F8980109F0BFFE94F891015C
:1069680009F083FEB4F89C0109F0B7FEB4F89E0163
:10697800B5E73E4C042009F0ADFE94F8D60109F0C5
:1069880074FE94F8D70109F070FEB4F8D801A6E7B0
:106998003D4C3E4D207800EB4000C0B209F09AFE15
:1069A800002623789E4205F1020580F0DC8015F868
:1069B800020C09F05AFE15F8010C00EB800000EB00
:1069C800800000F2EE2080B209F087FE0136E8E789
:1069D800012009F07FFE254B93F8920109F045FE4E
:1069E800C1E0082009F076FE0024204B234401343E
:1069F80093F8880109F039FE082CF6D1B3E0184B5A
:106A08001A4C93F8D100C0EBC000C0B209F062FE86
:106A180004F1280594F8F40100231D4AD25C904241
:106A280000F0A5800C333C2BF7D10834AC42F1D1EF
:106A380099E040200D4C09F04DFE04F14005B4F8F2
:106A4800AC0209F04AFE94F8AE0209F00EFE0434D6
:106A580094F8AB0209F009FEAC42F0D183E000BF24
:106A6800D0160020E1160020C0730108D4170020BA
:106A7800F01F0020F81F0020F61F0020F41F002040
:106A8800F21F002061170020C42100207419002083
:106A9800D4210020E020444C09F01CFE04F18005BC
:106AA800B4F82E0200F03F0009F017FEB4F82E02E9
:106AB800C0F3861009F011FE94F82C02000909F0C1
:106AC800D4FD94F82C0200F00F0009F0CEFD043438
:106AD80094F8290209F0C9FDAC42E1D143E0334CF6
:106AE8000D2009F0F7FD08F002FA09F0BEFD208834
:106AF80009F0FCFDE06809F0F9FD03F0ADFD30E0B8
:106B080009F0AAFD0546842009F0E4FD284609F0AD
:106B1800EDFD264BDC6805F18003A3428CBF641BA6
:106B2800802403F051FE28462246694608F03CFAC4
:106B380000240546AC4216DA1DF8040009F095FD5C
:106B48000134F7E7132009F0C5FD0024184B185D40
:106B5800013409F08AFD0B2CF8D1002009F0C6FD9C
:106B6800002009F0C3FD012018E0002016E009F01C
:106B78007CFDB4F8F60109F0B0FD94F8F80109F0CD
:106B880074FD94F8F90109F070FD94F8FB0109F01F
:106B98006CFD94F8FA0109F068FD46E720B0BDECF9
:106BA800028BBDE8F08700BFD41700200C0000203E
:106BB8002B9301082DE9F043CD4C237887B0074685
:106BC800002B00F0ED816268A368D31A7C2B40F299
:106BD800E781237BA26001332373002606F124009A
:106BE800C34DC0B206F034FD05F10E0333F916307B
:106BF80007EE903ABF4B1B88B8EEE77A07EE903A5B
:106C0800F8EEE77A0136C7EE277A9FEDBB7A67EE92
:106C1800877AFDEEE77ACDED037ABDF90C0006F030
:106C280005FD032EDAD1302006F012FDB5F9140067
:106C380006F0FCFC06F004FD2B7B9E072ED1AA680B
:106C480041F288339A4217D9102006F001FD6426D4
:106C5800A86990FBF6F000B206F0E8FC212006F0E7
:106C6800F7FCA86990FBF6F306FB13000028B8BFF1
:106C7800404200B206F0DAFC142006F0E9FC0A23D0
:106C8800B4F9200090FBF3F006F0D0FC1C2006F0CD
:106C9800DFFC002006F0CAFC06F0D2FC237B944EF1
:106CA800580740F05A81022006F0D2FC706A64232B
:106CB800323090FBF3F000B206F0B8FC0320B6F9CE
:106CC8002E5006F0C5FC8D4B1B7859074FF0050870
:106CD80095FBF8F5ADB20DD506F5DC7039460AF02E
:106CE80042FA28B9D6F8303813F0100F18BF00252B
:106CF80028B205E0D6F834389889B0FBF8F000B22D
:106D080006F094FCD4F83038794D9A076CD5DFF842
:106D18000082B5F83A6898F80030B5F83828360196
:106D28006427B6B207FB02325B00B2FBF3F346EA14
:106D38000326B6B2C3F303231E43062006F088FCDD
:106D480030B206F073FCB5F83A3898F80010013301
:106D58009BB293FBF1F201FB1233A5F83A38D5F850
:106D68003C389B7B012B05D1392006F071FCB5F925
:106D780038081AE0B5F838586E233A205D431526CE
:106D880006F066FC95FBF6F5AEB2B6FBF7F528B251
:106D980006F04CFC07FB15653B2006F059FCA8B231
:106DA800451D0A2095FBF0F000B206F03FFC2820B4
:106DB80006F04EFCD4F840380A2093FBF0F000B2FD
:106DC80006F034FC042006F043FCD4F834389B89E0
:106DD80013B102F015FE04E0454BD3F8440880F3E4
:106DE800100000B206F022FCD4F84838404E9B064A
:106DF80040F1A88096F84C389F071DD5112006F061
:106E080027FCB6F84E083E4B4FF4F365684390FBF9
:106E1800F3F000B206F00AFC192006F019FCB6F8E7
:106E28004E084543642095FBF0F595FBF0F300FB15
:106E3800135000B206F0FAFB94F84C38B4F85058E6
:106E480013F0020F08BF0025012006F001FC28B24C
:106E580006F0ECFB092006F0FBFB002006F0E6FB41
:106E6800284B94F852581A88B2F5967F0AD9204BC5
:106E78001B7B03F00F03072B04D842F20F759542D2
:106E880028BF1546052006F0E3FBD4F83C385B7BA9
:106E98000BB928B21CE0A5F1200307EE903A9FED4C
:106EA8001A7AF8EEE77AF6EE006AC7EE877ABEEE4F
:106EB800007AF5EEC07AF1EE10FA58BFB0EE667AB5
:106EC80077EE877AFDEEE77ACDED037ABDF90C000F
:106ED80006F0ACFB94F84C28054B950703D493F8BF
:106EE8005328012A18D1012384F85338074830E081
:106EF800A41700201C00002000007A44323400202F
:106F0800A08601007A0000206666E63FF81F002090
:106F1800780000208096184BD3F83C385FED036A60
:106F280093ED017AD3ED027A27EE267A67EEA67AF8
:106F3800BDEEC77AFDEEE77A8DED047ACDED057AE0
:106F480004A806E0B74A92E8030004AB83E803000C
:106F5800184606F08DFB06F073FB227BB24B282AFD
:106F68001ED100221A733C265B684FF47A70B3FB7B
:106F7800F0F7172006F06CFBB7FBF6F5B5FBF6F05B
:106F880006FB1050000200B206F050FB182006F075
:106F98005FFB06FB157000B206F048FB06F050FBDD
:106FA80094F85C38A04D002B00F05B810AF020F9C2
:106FB800D5F860389D4AC31A9342064640F2C58008
:106FC800002385F8663885F86838B5F83838DAB2B5
:106FD8001B0A85F8822885F8833885F8782885F88B
:106FE8007938D5F890286B689A1AD5F89438D97BEF
:106FF8004FF47A734B439A420DD36B68C5F89038B7
:1070080095F89838013B012B9FBF102385F8663807
:10701800022385F868380A20D4F8402892FBF0F259
:1070280084F88028121284F8812894F84C28D4F81F
:10703800443893FBF0F384F884381B1284F88538BD
:10704800900794F85238784984F8B33803D42D233C
:1070580081F8B43877E0042BD4F85498D4F85878E9
:10706800DFF8D881724A8CBF3323322381F8B438D1
:107078004FF0060C6F4B99FBF3F097FBF3F308FB0B
:10708800009108FB037803EB83030CFB01F103EB8E
:10709800830391FBF2FE642502FB1E119B0091FB0A
:1070A800F5F184F8A51809120CFB08FC84F8A61859
:1070B8009CFBF2F143FA81F39BB202FB11C292FBF3
:1070C800F5F284F8AA28121284F8A83884F8AB28B4
:1070D8001B0AB4F84E2884F8A9382423534393FB99
:1070E800F5F5B4F8C63884F8AC3800EB80001B0A14
:1070F80000EB8000800084F8AD380A22B4F85038DC
:10710800B3FBF2F303F5FA739BB240FA8EF080B248
:1071180084F8AE381B0A4FEAD97984F8A308FF0F20
:10712800000A84F8A05884F8AF38C5F30725B4F8E6
:10713800C83884F8A29884F8A40884F8A77884F852
:10714800A15884F8B538C4F8606894F8CA88364DF0
:10715800B8F1000F0DD1D5F8D0080AF053F901287D
:1071680007D90228344F00F05B8206F051FA012358
:10717800BB70D4F8D4282C4D002A72D095F8CA7860
:107188003FB1D5F8DC3840F6B731F31A8B4219D83D
:1071980067E00123D5F8D00885F8CA3800F08DFFDC
:1071A800D5F8E03893F9000002238DE8880008211B
:1071B8003A464FF4964300F093FF85F8E478C5F813
:1071C800D0084CE095F8D878CFB9D5F8D008C5F8EC
:1071D800D47885F8CA7800F070FFD5F8E03893F9CC
:1071E800000001238DE8880008213A464FF49643B1
:1071F80000F076FFC5F8D00806F00AFA2FE0013F44
:10720800FFB285F8D87895F8E41895F8E538BFB94D
:107218004A1C013385F8E42885F8E538D5F8D00804
:107228001BE000BF4C750108A41700203F0D0300A8
:1072380040420F00809698001C000020806967FF7C
:1072480012F8017BC5F8D428781885F8E4080133CA
:10725800D5F8D00885F8E53839460AF0D6F8C4F8E4
:10726800DC6894F8E638A44DDBB1D5F8E838C3B14A
:10727800D5F8EC38ABB1C5F8F0381B689F4AC5F8AB
:10728800F438D5F8F8381344187AFEF71BFD09F0DE
:10729800FDF9D5F8F8380133092B88BF0023C5F864
:1072A800F83894F8FC28944B6568002A00F0F381BC
:1072B800D3F80029002A00F0EE8193F80439013B45
:1072C800012B00F2E881D4F800098B4E0AF09AF8F5
:1072D800E0B1D6F800090AF092F896F80539D6F820
:1072E80004807E2B07460ED102231B2886F804391A
:1072F80009D1D6F800090AF085F820B90123C6F8A3
:10730800088986F80C3984F80579DCE7D6F8082965
:1073180073689B1A41F6583293421FD9032386F8A3
:107328000439B8E1764A32F8130010B903464FF42D
:1073380003600133B0F5C06FDBB27ED020D9B0F561
:10734800006F00F0848033D9B0F5036F40D184F822
:107358000D39D4F84838684E9B0640D494F80C6927
:1073680094F80D39002E00F0588162686249521B6A
:10737800012AD7D981F80D39002381F80C398AE11F
:10738800B0F5007F43D007D8B0F5807F4CD0B0F57A
:10739800887F00F09180E5E7B0F5806F00F0B2805B
:1073A800B0F5826F00F0F780B0F5047FDAD123E002
:1073B800B0F5E26F00F09280B0F5E46F00F09380D2
:1073C800B0F5E06FCED184F80D39B4F90E108EE027
:1073D800B0F5046F7AD0B0F5026FC3D106E196F824
:1073E8004C389F07BAD5B6F84E1824234B431233AE
:1073F800642193FBF1F10AE184F80D39D4F83038AF
:107408003D4E9907AAD5B6F838380A21FEE084F827
:107418000D39D4F83038384E1A059FD5D6F84018AB
:107428000A2391FBF3F1F2E084F80D39D4F84838D7
:10743800314E5B0792D5B169E9E084F80D39D4F88B
:1074480030382D4E1F0589D5D6F84418DFE0D4F81A
:107458004818294A84F80D3988067FF57FAF92F8D5
:107468004C1889077FF57AAFDB0712D5D2F8583860
:1074780083EAE371002BA1EBE37101EB51014FF0BB
:107488001902B1FBF2F1ACBF41F0004141F04041BB
:107498000FE0D2F8543883EAE371A1EBE371002BD3
:1074A80001EB51014FF01902B1FBF2F1B8BF41F005
:1074B80080414FF4006088E084F80D39D4F84838EA
:1074C8000D4E5F077FF54AAF7169A0E0B4F920104F
:1074D80084F80D3901EB8101490076E084F80D3913
:1074E800B4F9101003E0B4F9121084F80D392C2304
:1074F80091FBF3F169E000BFA41700204C75010867
:107508002C97010884F80D3994F80E39634A013331
:10751800DBB2032B88BF012382F80E3994F80E19C9
:1075280042F2107359435E4B1B78D80748BF0131AC
:107538009A0748BF02315F07B4F8103948BF0431D1
:10754800DE0748BF0A31980748BF14311A0648BFFA
:107558002831DF0548BF28315E0748BF6431180766
:1075680048BFC8319A0548BF01F5C8719F0648BF92
:1075780001F57A71DE0648BF01F5FA61580648BF81
:1075880001F57A614FF4806001F064FC434B0022FE
:1075980083F80C29E2E6D4F84818404F84F80D39EE
:1075A80011F0200617D097F84C2812F0020F14BFDC
:1075B8004FF47A71002112F0010F14BF4FF4FA63EF
:1075C80000230B4494F85218194401F043FC00239B
:1075D80084F80C39C2E6D7F8303819067FF5BEAE04
:1075E800314601F037FC87F80C69B7E684F80D39A5
:1075F800D4F84838294E9A067FF5B0AE96F84C383C
:107608009B077FF5ABAEB6F850386421594301F0BB
:1076180021FC002386F80C39A0E684F80D393AE0FD
:10762800BB7823B1C5F8CC6887F80280A1E5D5F806
:10763800CC38F31AB3F57A6FFFF49BAD0123D5F874
:10764800D008BB7009F0DBFE0746D5F8D00809F072
:10765800D6FE79067FF48DAD8A2802D08E280DD00B
:1076680087E5D5F848389A067FF583AD95F8CA3886
:10767800002B7FF47EAD05F6990306E095F8CA382D
:10768800002B7FF476AD05F66403C5F8D4382D23B6
:1076980085F8D8386DE507B0BDE8F083A417002059
:1076A80032340020F8B504460E4617460025204619
:1076B80020210FF086FB0446D0B1013420460DF09E
:1076C800E7FFB0F5617F05DB40F634039842A8BFB9
:1076D800184601E04FF46170A0F56170192390FB22
:1076E800F3F00DB9307000E070703B7801333B70F7
:1076F8000DB90125DBE72046F8BD30B505460C4637
:107708001346294622460248BDE8304004F01EBD13
:107718001C9801087FB504780646E4B9354B1B6808
:1077280003EB8403192193F8830093F8846093F89A
:10773800812093F882304FF4617511FB005011FBE2
:107748000651009001912C482146013404F0FEFCBA
:10775800142CE3D14BE00DF09BFF1328054641DCC8
:10776800244B701C1C68202100238DF80F300FF06B
:1077780028FB2035064670B1013630460DF088FFEB
:107788001A289FBF04EB850358709DF80F3001330A
:1077980098BF8DF80F30304620210FF012FB0646B7
:1077A80070B1013630460DF073FF0D289FBF04EB12
:1077B800850398709DF80F30013398BF8DF80F300E
:1077C80004EB85043046E11C0DF10F02FFF76AFF58
:1077D8009DF80F30042B0AD0601C002104220FF002
:1077E800BDFA04E0054800211322FFF786FF04B024
:1077F80070BD00BF181700203B9801085098010879
:10780800014808F0EFBF00BF569801082DE9F04382
:1078180004788FB00546002C59D17B4B00211422E7
:1078280009A807AED3F800800FF098FA072230466F
:1078380000210FF093FA05A80023A700059308EB91
:10784800070583801A467149B5F802E031F813C07C
:107858001CEA0E0F0AD00DF1380C0E3102F1010EA0
:107868006244595C02F81C1C5FFA8EF20133072B44
:10787800E9D100210B46664AB5F802E011F802C0CA
:107888001CEA0E0F0AD00DF1380C063203F1010E76
:1078980063448A5C03F8242C5FFA8EF301310629CD
:1078A800E9D118F807305B498DE841006A780292FF
:1078B80009A81A0903F00F0304F033FC21465648BF
:1078C80009AA013404F042FC202CA6D198E00DF05E
:1078D800DFFE1F28044600F3868028462021E4B2F4
:1078E8000FF06FFA1F2C02D9FFF78AFF88E0464B8A
:1078F8001B6803EB8404451C0021204604220FF07A
:107908002DFA0027454B09AE304600210A2217F808
:1079180003905FFA87F80FF021FA002315F8012B7E
:1079280032B10A2B04D04A4502D0F2540133F5E7AC
:107938004A455ED108F1FF33032B09D8DFE803F08D
:107948001005023F0DF1230134E00DF123011EE083
:1079580030460DF09DFE2378C0B243EA001006E0E1
:1079680030460DF095FE237800F00F001843207084
:1079780031E00133062B0AD0244800F11B069E5D36
:107988009642F6D103445A7D63881343638011F805
:10799800012F02B30023EFE70133072B0AD01B485E
:1079A80000F10E069E5D9642F6D130F813206388EA
:1079B8001343638011F8012F6AB10023EFE73046C3
:1079C8000DF066FE0F2804DC30460DF061FE607095
:1079D80001E0002363700137052F93D1012408F0DB
:1079E80001F96CB980E70E4800211F22FFF785FED8
:1079F80006E02046002104220FF0B0F90024EEE74B
:107A08000FB0BDE8F08300BFB82000206075010802
:107A18007575010864980108739801088175010853
:107A280050980108F8B50478064674B9304DB5F891
:107A3800C421B5F8C6312F482146013404F086FB2D
:107A4800042C05F10405F2D1F8BD2B490FF08EF98D
:107A5800A8B9274B4FF47A714FF4FA62A3F8C4110E
:107A6800A3F8C621A3F8C811A3F8CA21A3F8CC111A
:107A7800A3F8CE21A3F8D011A3F8D221F8BD30463F
:107A88000DF006FE032805462BD8304620210FF0BE
:107A980098F9044630B1013420460DF0F9FD01266D
:107AA800074600E00646204620210FF08AF910B963
:107AB800BDE8F840A4E601300DF0EAFD012EF7D14B
:107AC800A7F2EE2240F2DC539A42F1D8A0F2EE225D
:107AD8009A42EDD8064B703503EB85039F80D8801A
:107AE800F8BD064800210322BDE8F84005E600BFBE
:107AF800D41700207F98010892980108B9A60108B8
:107B08002DE9FF4104780546002C39D17348744D9E
:107B180008F068FED5ED047AF5EE407AF1EE10FA39
:107B280000F0D88021466F4804F010FB95ED040A58
:107B3800684604F08BF901466B4804F007FB95EDA5
:107B4800050A684604F082F90146674804F0FEFA1F
:107B580095ED060A684604F079F90146624804F092
:107B6800F5FA95ED070A684604F070F90134014604
:107B78005E4804F0EBFA0C2C05F11005CAD1A9E017
:107B88005B4905220FF032F940B9554B03F1C002A9
:107B9800002143F8101F9342FAD19BE0284655492B
:107BA80004220FF023F904462846002C40D1202156
:107BB8000FF007F9002800F08D80451C28460FF0CB
:107BC8000DF907464C4B53F824601EB94B4808F092
:107BD80009FE7FE028463146FAB20FF007F9013472
:107BE8000028EFD13E4B03F1C0029E46002143F826
:107BF800101F9342FAD1424B03EBC4029846D2F8C5
:107C080004C0BCF1000F04D131463E4804F09EFA8E
:107C180057E0002718F834309F42F5DA3B010EEBA5
:107C2800030563440FCB103585E80F000137F1E7F2
:107C38000DF02EFD0B28064647DC284620210FF0C4
:107C4800C0F8054650B10135284604F075F8244BB4
:107C580003EB061383ED040A012400E004462846DA
:107C680020210FF0AEF8054648B10135284604F04A
:107C780063F81B4B03EB061383ED050A0134284612
:107C880020210FF09EF8054648B10135284604F03A
:107C980053F8134B03EB061383ED060A0134284609
:107CA80020210FF08EF810B9FFF7AAFD12E001307D
:107CB80004F042F80A4B032C03EB061686ED070A7C
:107CC800F2D11148FFF71CFF04E0104801210C22F3
:107CD800FFF713FD04B0BDE8F08100BF98980108D4
:107CE800D4170020B3980108B9980108F0A3010837
:107CF80092980108BD980108A07C0108C298010863
:107D08004C970108D198010810960108509801086D
:107D1800F0B5047887B006461CBB514B196806239A
:107D280003FB0411192091F8D25091F8D37091F8FF
:107D3800D62091F8D1304FF4617610FB056510FB21
:107D480007600095019091F8D4000290D031454821
:107D5800497903912146013404F0F8F90C2CDCD15F
:107D68007CE00DF095FC0B28044672DC3C4B701C43
:107D78001D68202100238DF817300FF022F80646E1
:107D880080B1013630460DF083FC03289FBF0623DF
:107D980003FB045383F8D6009DF817309CBF0133CA
:107DA8008DF81730304620210FF00BF8074680B1C8
:107DB800013738460DF06CFC0D289FBF062303FBE6
:107DC800045383F8D1009DF817309CBF01338DF818
:107DD800173006266643A9193846D2310DF1170225
:107DE800FFF760FC20210EF0ECFF074670B1013769
:107DF80038460DF04DFC14289FBF9DF817307619B2
:107E0800013386F8D40098BF8DF817303846202102
:107E18000EF0D7FF78B101300DF03AFC0D289FBF66
:107E2800062303FB045383F8D5009DF817309CBF45
:107E380001338DF817309DF81730062B0ED0062227
:107E480002FB04500021D1300EF088FFFFF7D8FC68
:107E580004E0054800210B22FFF74FFC07B0F0BDF6
:107E680018170020DD980108509801082DE9F347FC
:107E7800047807464CB9204601A901F063F901349A
:107E8800FFF7F4FF122CF6D17EE00DF001FCC5B22D
:107E9800112D74D8781C20210EF093FF3C4C3D4FD7
:107EA80005F1D006034614F8168030B9A8F102028D
:107EB800D2F1000848EB020846E007F1260800F175
:107EC800010A597840460EF07CFF68B1032D8CBF3B
:107ED80003230023C8EB00003B4453FA80F090F8DA
:107EE8002A90B9F1030F02D1FFF78AFC4CE0A9F1FF
:107EF8000203D3F1000850464FF0200148EB030875
:107F08000EF05FFFD8B1B8F1000FEDD001300DF0E1
:107F1800BFFB40F2ED2380B2984205DD40F6CA036C
:107F28009842A8BF184601E040F2EE2004EB460351
:107F3800A0F2EE20192290FBF2F0587002E0B8F19E
:107F4800000FD1D104F8169014F816301F4497F892
:107F58002620B8F1000F0DD00D4B0F4803EB460655
:107F68002946737840F2EE24192505FB034304F0F3
:107F7800EDF809E02946094804F0E8F804E0084863
:107F880000211122FFF7B9FB02B0BDE8F08700BF5E
:107F9800D417002060750108FD9801080F990108A1
:107FA800B9A6010807B50123ADF8041001A98DF899
:107FB80006208DF80730FDF781FC03B05DF804FB5F
:107FC8002DE9F041054672B64FF090464FF48061B6
:107FD8004FF400773185304604223785FFF7E2FFFA
:107FE800304639460122FFF7DDFF2C4850F835406E
:107FF80000EBC500236842680125510005FA01F825
:1080080048EA030395402360A561B7614FF09043A8
:108018001B8A5E05FAD4236848EA030323604FF0FD
:1080280090434FF40072A9B221851A850822C3F83B
:10803800182440F605564FF090473B8A580503D45C
:10804800002EF8D0013EF6E7A56120460422FFF78E
:10805800A9FF96B14FF090431A8A5205DBD5228AC0
:1080680092B215420E4A4FF400704FF0080115BF46
:108078009861188591611185ECE7094B4FF40071FF
:108088000822B96138469A610222FFF78BFF62B66F
:108098000A20BDE8F04109F0D2B800BF40990108B4
:1080A8000004004810B50446204609F0A2F918B9A2
:1080B8000A2009F0C4F8F7E710BD002207490C238D
:1080C80003FB02135968814204D10022C2621A726A
:1080D8005A6070470132052AF0D17047D421002038
:1080E8002DE9F74389469DF8288011461A469DF8E0
:1080F8002C30064600250C2068431D4FC419C05774
:10810800B04202D1207A20B12BE00135052DF2D101
:1081180027E0022E0FD005DC56B1012E21D10093A5
:1081280014480AE01E2E0DD01F2E1AD1012009E096
:108138000093114801E0114800934346FDF744F8C5
:10814800044605E006F014FE4146044609F04EF9DF
:108158004CB10C2303FB0575267185F808906C60FB
:1081680001E0002000E0204603B0BDE8F08300BF36
:10817800D42100200044004000380140004800405D
:1081880010B5084B1968002201EBC20393F90240AD
:10819800844201D1981C10BD0132052AF4D1002077
:1081A80010BD00BFCC210020F0B5027887B08AB995
:1081B8004A4C04F1280694F8F421002348495956FA
:1081C80050B281426ED00C333C2BF7D10834B44204
:1081D800F1D181E0002204920592451C0DF058FA75
:1081E800C4B260B2FFF7CCFF074618B18DF8104053
:1081F800012400E00446284620210EF0E2FD054651
:1082080038B1013528460DF043FA0134ADF81200B3
:10821800E4B20026284620210EF0D3FDB0B3451C59
:1082280028460DF035FA00222E4951F822308342B3
:108238005FFA82FE04D00132082AF5D1002300E05B
:10824800734651F82320824220D1022E0FD0032EEC
:1082580012D05A1E012ED2B204D0042A13D88DF897
:1082680014300EE0042A0ED88DF8153009E0052BDD
:1082780009D88DF8173004E09A1E052A03D88DF81E
:1082880016300134E4B20136042EC3D1052C04D8CB
:1082980007B0BDE8F040FFF7B3BA04AB03CB3860D2
:1082A800796019E094F8F9010E4B94F8F85153F8F5
:1082B8002000B4F8F621009094F8FB0153F8200050
:1082C800019094F8FA0153F82000029053F82530F1
:1082D800054803F03BFF79E707B0F0BDD41700204D
:1082E800D4210020687A01081E99010838B1438812
:1082F80011EA030003D08B420CBF01200220704713
:1083080030B50A4B0A491C680A79042A0AD8134668
:1083180004EBC303551CEAB29D882842F5D00A71C4
:10832800981C30BD0A71002030BD00BFCC21002050
:10833800B8200020014B00221A71E1E7B820002084
:108348002DE9F047877890F803C0214DBBB2C7F1FB
:10835800640E03EB83065C42C3F178005FFA8EFE7D
:108368007600CCF16408A4B280B2A3B20FFA83F904
:10837800B9F1000F05DC002B14BFBA464FF0010A13
:1083880000E0F24613FB03F303FB0CF21AFB0AF3BB
:1083980092FBF3F3434403FB09F30A2293FBF2F342
:1083A80033449BB225F8023FB1F800904A880A345A
:1083B800C9EB020AA4B21AB202FB0AF24FF47A73AA
:1083C800844292FBF3F34B442B80CED1BDE8F08777
:1083D800BC200020344B354A1B68126810B51A605F
:1083E800334A1168596051689268DA60314A996075
:1083F80011681961516892689A612F4A5961116828
:10840800D961516892685A622C4A19621188198593
:10841800518859859188D288DA85294A99851188A1
:1084280019865188598692889A86264A1188D9864B
:10843800518819871946928821F83A2F224A1078CC
:108448000022824206DA214C34F8124021F8024F09
:108458000132F6E71E4A1288A3F864201D4A1288E2
:10846800A3F866201C4A1188A3F86C1051889288DA
:10847800A3F87020194AA3F86E1012689A66184A71
:108488003B21126892FBF1F2B2F5967FC8BF4FF01C
:10849800FF325A67134A1288A3F87820124A528981
:1084A800A3F85E2010BD00BF383000201034002033
:1084B800C4240020D0240020DC240020CC17002075
:1084C800FC160020B21700207C2E00201C1700206C
:1084D80054220020DC0F002002170020BC170020C7
:1084E800000000203C170020081700202DE9F84361
:1084F8000E4B93E8800305460E460024B44213DA77
:108508007B1933F9140008EB050333F9142009EB40
:10851800050333F914301344022293FBF2F3C01A13
:1085280007F047FA0134E9E7BDE8F883383000205E
:1085380010B5104B93F8F437012B014612D10E4AAF
:108548000E4C1078431CDBB213701B0644BF00238B
:108558001370215402F076F93F2809D9BDE810407C
:1085680002F04EB9064BBDE81040186808F04DBF40
:1085780010BD00BFD4170020882B00208A2B0020B4
:108588001C30002070B54720FFF7D2FF174B1B683F
:108598001B0307D5164B174A5B6810681B68C01A7F
:1085A80007F0F7F9144E154C154D307807F0F1F92E
:1085B80023682868C01A07F0FCF963686868C01A5D
:1085C80007F0F7F90F4B188807F0E3F90E4B1888F6
:1085D80007F0DFF90D4B188807F0DBF933782374BF
:1085E8002B68A3606B68E36070BD00BFBC310020DE
:1085F8003830002010340020F61F002024300020DE
:10860800F81F0020F41F0020F21F00204817002048
:108618007FB5264C264E274D2749284A284B20B19E
:1086280028480088B0F5805F31D23088ADF8040062
:1086380028781E4D91F8201012788DF806008DF8D4
:1086480007108DF808201B788DF8093001A82946F5
:1086580006220EF06BFB30B30198BDF80830286095
:10866800AB805320FFF764FF208807F092F9A078C9
:1086780007F08FF9E37801932379029301A86379CE
:10868800039307F0F5F80F4B00221A800BE03088AF
:10869800208091F82010287812781B78A070E1705B
:1086A80022716371DDE704B070BD00BFD8200020DF
:1086B800B4200020F01F0020B0330020E80D002077
:1086C800960E0020E03100200A4A138801331380F7
:1086D800094A136801331360084A138801339BB2AF
:1086E800202B01BF00231380054A138808BF0133DC
:1086F80013807047E0310020C4310020C8310020C9
:10870800CA31002038B5294B1B78083B012B054698
:108718000C464AD84520FFF70BFF2846FFF708FF0D
:108728000E2D33D003D83DB10D2D07D038BD142DF3
:1087380020D0FF2D32D038BD20682BE06378207818
:108748009BB180F08000FFF7F3FEA568E8B2FFF761
:10875800EFFEC5F30720FFF7EBFEC5F30740FFF771
:10876800E7FE280EFFF7E4FE04E0FFF7E1FE60688D
:1087780007F01FF92078FFF7DBFE606807F019F9AA
:108788002489E0B2FFF7D4FE200A0BE0206807F046
:1087980000F96068BDE8384007F0FBB8044807F006
:1087A8000CF90020BDE83840C2E638BD183000207A
:1087B800809901082DE9F04FBE4BBF4F1A888BB046
:1087C8000193002A40F0A980B7F8F207BB4E42F2A5
:1087D8000103C21A50425041FFF71AFFFFF7FAFD92
:1087E80034684920FFF7A4FEB54B2546186807F002
:1087F800D0F855F8040B07F0CCF8284600F0F8FB41
:1088080004F1100000F0F4FB04F11C094FF010080B
:10881800AC4D01232A6803FA08F3134203D0D9F8B0
:10882800000007F0C6F808F10108B8F1130F09F1C4
:108838000409EDD104F1280000F0CAFBB7F8403173
:10884800B4F92E00C01A07F0A4F82B68DB0408D589
:108858009D4BB4F864001B88181AC0F30D0007F08C
:1088680098F82B68980403D5B4F8660007F091F8D7
:108878002B68590503D504F16C0000F0A9FB2B689F
:108888001A0502D5A06E07F094F82B685B0402D590
:10889800606F07F08EF82B68180403D5B4F87800D9
:1088A80007F077F804F13000A04600F091FB04F1DE
:1088B800360000F08DFBB7F8403138F93C0FC01A8C
:1088C80007F067F80127814B1B789F4208DA38F9CF
:1088D800020FB4F93C30C01A07F06BF80137F2E721
:1088E8002B68990505D5B4F95E00A0F2DC5007F0B5
:1088F80060F8326876487260B260121A9110754A50
:108908004A43531C032293FBF2F202EB42029A1AE7
:108918007C2303FB02033360D6E16F4B6F4A1B686D
:1089280011688B4206D00AA9002041F8203D136047
:10893800FFF7E8FE019B97F8F2171B8897F8F307F3
:108948000B44013BB3FBF0F200FB12338B4280F087
:1089580086815A4F0120FFF75BFEFFF73BFD502051
:108968003E687D68FFF7E4FDBA683B6810681B68DD
:108978007A6803441068A3EB400007F01AF86A68A5
:1089880073689B1A0293AA68B3689B1A0393EA68F0
:10899800F36802A89B1A049300F02AFB2A6933693A
:1089A8009B1A02936A6973699B1A0393B369AA694C
:1089B80002A89B1A049306F05BFF06F11C0B05F155
:1089C8001C0810243F4901220B68A2401A428A461B
:1089D80006D0DBF80000D8F80030C01A06F0E9FF2E
:1089E8000134132C0BF1040B08F10408EAD106F149
:1089F800260005F12601002331F9024F30F9022F34
:108A0800121B02AC44F823200133042BF4D10321B8
:108A18004FF000094FEA89035FFA83F902AB53F874
:108A280021206AB102F108000F2802D849F0010993
:108A380006E08032FF2A94BF49F0020949F0030991
:108A480011F1FF31E6D24846FFF772FD00240DF11F
:108A5800080BA04609F00302022A16D0032A1DD0EB
:108A6800012A4ED1B8F1000F05D1DBF800402401EE
:108A7800E4B2904645E0DBF8000000F00F00204328
:108A8800FFF756FD4FF000083BE0B8F1000F0CD09F
:108A9800DBF80000C0F3031020432CE0B8F1000F0E
:108AA8001ED19BF80100FFF743FD9BF80000FFF77C
:108AB8003FFD26E0C8310020D417002038300020C0
:108AC800C4310020BC310020B83100207C2E0020A9
:108AD80044300020DF7BEFBDD0310020CC310020B6
:108AE800DBF80000C0F303302043FFF721FDDBF87B
:108AF8000000C0F30710FFF71BFDDBF8004024015E
:108B0800E4B20BF1040B06AB9B454FEA9909A1D1DE
:108B1800B8F1010F02D12046FFF70AFDDAF800305C
:108B280013F480541FBFB6F86420B5F86410521AC5
:108B3800029218BF01249A040AD50AAA02EB8401FA
:108B4800B5F86600B6F86620121A41F8202C0134F0
:108B5800580513D502AA02EB840C06F16A0E05F13A
:108B68006A0000223EF9021F30F9028FC8EB0101AA
:108B78004CF822100132032AF4D10334190508D520
:108B88000AAA02EB8400A96EB26E521A40F8202C91
:108B980001345A0408D50AAA02EB8400696F726F7F
:108BA800521A40F8202C013418040BD50AAB03EBF9
:108BB8008402B5F87810B6F878305B1A42F8203C91
:108BC800013400E0FCB1012C03D1029806F0F1FE5B
:108BD80019E0631E002002AA400052F82320C0B208
:108BE8000AB140F00100013BF5D5FFF7A1FC4FF0B9
:108BF800000802AB53F8280008B106F0DAFE08F1C5
:108C08000108A045F5DB30200321FFF76FFC362073
:108C18000321FFF76BFC2F4B3C201978FFF766FC0C
:108C2800DAF80030990506D5B6F95E00B5F95E3078
:108C3800C01A06F0BEFE3A6827487B687A60121AA6
:108C48009110264ABB604A43531C032293FBF2F25D
:108C580002EB42029A1A7C2303FB02033B60204B7F
:108C68001B681A0630D51F4C1F4D22682B689A4284
:108C78000BD162686B689A4207D1019B1B88102B45
:108C880011D11A4B1B885B060DD14820FFF750FC09
:108C9800206806F08EFE606806F08BFE23682B6065
:108CA80063686B600EE0124A0F4B11782A7C914280
:108CB80008D1104A99681068884203D15268DB6865
:108CC8009A4201D0FFF75EFC06F0C0FD0BB0BDE88C
:108CD800F08F00BF7C2E002044300020DF7BEFBDEA
:108CE800D41F00204C17002024300020CA31002057
:108CF800F61F0020F81F00202DE9F74F0E9F4D4C5E
:108D0800C2EB030B0D9BFF1A6368002914BF4FF0D9
:108D180006094FF0040901338246164634D1226809
:108D28004A4580F08280DFF82881019158F82200B6
:108D38000EF054F80B3006F029FD0199054608B1EC
:108D4800012073E022683C48032A98BF514658F82E
:108D5800222006F0C5FE394A1368181A63681060A5
:108D680001336360364B9D710EE00D9A92B103FB9F
:108D780007F20D99895C01228A40324909680A4242
:108D880008D163680133636063680C9A294D934284
:108D9800EBDB32E003FB0BF5236806EB050A2BB986
:108DA80070590EF01BF800F1050801E04FF00308B8
:108DB800404606F0EBFC0028C2D1204A204B106840
:108DC800C8EB000010609A791AB12C20FFF7B0FBAD
:108DD80001E001229A71236843B9705906F0EDFD4C
:108DE8009AF904104B1CCCD0174803E09A44174852
:108DF8009AF8041006F074FEC3E710D1012006F0BB
:108E0800C5FC60B90D4A13680A20013B1360FFF7DF
:108E18008FFB2B6801332B604FF0FF336B602068AA
:108E280048452CBF0020012000E0002003B0BDE829
:108E3800F08F00BFD83100208B990108D431002071
:108E4800D8200020BC3100209A99010827A30108E6
:108E5800507A010830B585B004AC002524F8025DCD
:108E68000091ADF806002146102004F0B3FB9DF8F0
:108E78000600214604F0AEFB9DF80700214604F0E9
:108E8800A9FB9DF80000214604F0A4FB9DF8010011
:108E9800214604F09FFB9DF80200214604F09AFB4E
:108EA8009DF80300214604F095FB9DF80E00C04391
:108EB800C0B2294604F08EFB05B030BD084BDA6815
:108EC800D10709D4DA68D20608D4DB6813F0040F96
:108ED80014BF032004207047012070470220704708
:108EE8000020024003788B4286BF024B33F8110002
:108EF80000207047E020002070B5344C054608F08B
:108F080077F9A369A061C31AB3F5FA5FE36182BF79
:108F1800002384F8203084F8213094F820302BB9CD
:108F2800A12D02BF294A012182F8211094F82110AD
:108F3800264A31B1D118EDB2013381F8225082F8B6
:108F4800203094F8205094F84330AB423CD11F4B6A
:108F580093F84430052B02D0062B03D02FE00020D5
:108F680009F0DCF894F823301E2B28D100200246A3
:108F7800C1B26B1E99421ADA214491F822300821B5
:108F8800DBB283EA0206F60744BF83F01803C3F393
:108F9800460301F1FF3154BF5B0843F0800311F031
:108FA800FF01C2F34702ECD101301A46E0E723443F
:108FB80093F822309A4202D1032009F0AFF8002337
:108FC80084F8213084F8203070BD00BFE0200020F4
:108FD80010B50446B0F9000006F0EBFCB4F9020045
:108FE80006F0E7FCB4F90400BDE8104006F0E1BC67
:108FF80010B50446006806F0DCFC606806F0D9FC91
:10900800A068BDE8104006F0D4BC2DE9F74F012058
:10901800FFF790F9002488B3012C2FD8194E4FF090
:109028004C0909FB04FA06EB0A0808F19007BD7819
:1090380015B10134E4B2EEE790F9003090F804E09D
:109048001846114B03228DE8240001212A4653F8C3
:109058002E30FFF745F8834660B106F148005044CA
:1090680029464A460DF07AFE01231C44C8F848B048
:10907800BB70E4B20120FFF743F9CCE703B0BDE8C9
:10908800F08F00BFE0200020687A010800212A2222
:1090980010B511480DF062FE104B00221946104819
:1090A800105C83F8F40104240520013283F8F941A7
:1090B80082424FF0000483F8F80183F8FB4183F8FB
:1090C800FA0103F10803EAD10123A1F8F63152238A
:1090D80081F8F23110BD00BFC6190020D417002056
:1090E800BE99010810B5FFF7E9FE4FF430240128B6
:1090F80006D11CB1FFF7E2FE013CF8E7052010BDE0
:10910800002C08BF052010BD70B50646441E14F893
:10911800011F89B1094D28460DF053FE0028F6D0ED
:1091280005F1080398423FBF054B401BC018A31B1D
:1091380038BF80F88831EAE770BD00BF3BB001084E
:10914800D4170020031EB8BF2D2210B5B8BF58424F
:109158000C46B8BF01F8012B0A2202F0E1FE0023F9
:109168000370204610BD07B51C4B03F1E402C3F899
:10917800E0201B4A92F890215AB1012A14D1032108
:1091880083F8E610072183F8E82083F8E7100C221B
:1091980008E0022183F8E610032183F8E82083F829
:1091A800E710072283F8E4200E4B0F4A1A6040208C
:1091B800FFF7C0F870B10122002390F900004021A8
:1091C8008DE80C00094A4FF4E133FEF789FF0030BF
:1091D80018BF012003B05DF804FB00BFE0200020A9
:1091E800D417002020000020D91E0108911F010873
:1091F8000120002107F050BAF0B5184AD2F8EC70F7
:1092080092F8F0301546042B11D807EBC3025E1C08
:10921800941CF6B209D013469288D10705D510429E
:1092280003D008E00131052908D13346EBE785F87A
:10923800F0300020F0BD93F802E00021074C0C222A
:1092480004F1F40C02FB01F31CF803209645E9D164
:10925800234484F8F060D3F8F800F0BDE020002043
:109268000A888B88F0B54C880E89CD88C2B9026A05
:1092780022F0010202628269016A22F0F3021A43B3
:1092880042EA061344F0010421F00A021443836100
:109298000462836923F00C03836183691D431FE023
:1092A800042A016A1ED14FF6EF720A4002628269EF
:1092B800016A1B0222F4734243EA06332401134372
:1092C80044F010044FF65F720A40A4B2224383614F
:1092D8000262836923F440638361836943EA052555
:1092E8008561F0BD082A1DD14FF6FF620A4002626F
:1092F800C269076A4FF60C7111404FF2FF523A40AB
:1093080042EA042443EA06130B4344F480749BB2F4
:10931800A4B2C3610462C2694FF6F3731340C36118
:10932800C3691FE04EF6FF720A400262C169026A11
:1093380040F6FF470F4045F6FF7111401A0242EA16
:10934800063341EA04343B4344F480549BB2A4B24C
:10935800C3610462C2694FF2FF331340C3612D0237
:10936800C369ADB21D43C561F0BD036A23F00103B3
:109378000362036A70B5446882690D6822F480321A
:1093880022F0730215438A8923F0020313438A8863
:109398001343134A90420FD002F5006290420BD05B
:1093A80002F54062904207D002F58062904203D0F5
:1093B80002F5806290420DD1CA89CE8823F0080355
:1093C80013430A8A24F4407414434A8A23F004039A
:1093D800334314438A68446085614263036270BD05
:1093E800002C014001F0030301F0FC0101F1804170
:1093F80001F5803110B59B008C680F229A4024EA51
:1094080002028A608A68984002438A6010BD00237D
:109418000360436083608381036143618361C36147
:1094280003624362836270478A68036810B50C6AF6
:1094380014430A6914434A6914438A691443CA697C
:1094480014434A6A14438A6A23F4FF4323F07003DF
:109458002243134303608B8943600B6883604B6826
:10946800C36010BD02684FF6FE731340036000230B
:10947800036043608360C360284B984201D1284A47
:1094880027E0284B984201D1254A2AE0264B9842EA
:1094980001D1234A2DE0254B984201D1204A30E0E2
:1094A800234B984201D11E4A33E0224B984204D103
:1094B8001B4A536843F470032EE01F4B984204D1B3
:1094C800174A536843F0706326E01C4B984204D156
:1094D8001B4A536843F00F031EE01A4B984204D10D
:1094E800174A536843F0F00316E0174B984204D12B
:1094F800134A536843F470630EE0144B984204D146
:109508000F4A536843F4704306E0114B984204D164
:109518000B4A536843F470235360704708000240B5
:10952800000002401C00024030000240440002409B
:10953800580002406C0002408000024008040240CB
:10954800000402401C04024030040240440402406B
:109558005804024020F01F01012300F01F00024AB6
:1095680083408B50704700BF14040140F0B50023BE
:109578000E681C460125A54005EA060EAE452BD10E
:109588000F797A1E012A15D8856803229A4025EAA0
:10959800020282604D7982689D4015438560828809
:1095A80092B222EA0E0282808A798588A2402A43F2
:1095B80092B28280032205689A40D2431540056022
:1095C80005689F402F430760C7681740CA7902FAA9
:1095D80003F547EA0502C2600134102C03F10203C7
:1095E800C8D1F0BD9B4A536803F00C03042B2DE946
:1095F800F04105D0082B06D097490160B3B916E0B1
:10960800954B036012E053685468C3F38343991C75
:10961800E30349BFD36A914B8F4C03F00F0344BF58
:109628000133B4FBF3F34B43036000E000235168BC
:109638008B4FC1F3031139440D790168EDB221FA5A
:1096480005F444605668C6F302263E44367924FA87
:1096580006FEC0F808E05668C6F3C2263E443679CE
:10966800F6B2F440C460D2F82C80C8F3041808F0AD
:109678000F0C07EB4C0C18F0100FBCF814C01FFAB5
:109688008CFC07D0BCF1000F04D0B3FBFCFCC0F885
:1096980010C000E00161D2F82CC0CCF3442C0CF0CF
:1096A8000F0807EB48071CF0100FBF8ABFB204D0A1
:1096B8001FB1B3FBF7F7476100E04161176BFF0685
:1096C8005ABF654F87618161176BBF065ABF624FEA
:1096D800C761C161176B7F065ABF5F4F076201629E
:1096E800176BFF0506D5994204D1AE4202D14F004F
:1096F800476200E04462176BFF0406D5994204D123
:10970800AE4202D14F00876200E08462176BBF054A
:1097180006D5994204D1AE4202D14F00C76200E09B
:10972800C462176B7F0506D5994204D1AE4202D1B7
:109738004F00476400E04464176B3F0506D5994223
:1097480004D1AE4202D14F00876400E08464176BF5
:10975800BF0406D5994204D1AE4202D14B00C3647E
:1097680000E08464156B3B4BAD0701D1046315E041
:109778001C6B04F00304012C01D101630EE01C6B87
:1097880004F00304022C02D14FF4004305E01B6BE4
:1097980003F00303032B01D12F4B0363146B2D4BF1
:1097A80014F4403F02D1C0F834E018E01C6B04F414
:1097B8004034B4F5803F01D1416310E01C6B04F4E0
:1097C8004034B4F5003F02D14FF4004306E01B6B70
:1097D80003F44033B3F5403F01D11F4B4363146B8F
:1097E8001C4B14F4402F02D1C0F838E018E01C6B71
:1097F80004F44024B4F5802F01D1816310E01C6B80
:1098080004F44024B4F5002F02D14FF4004306E0DD
:109818001B6B03F44023B3F5402F01D10E4B836338
:10982800146B0C4B14F4401F02D1C0F83CE021E04B
:109838001C6B04F44014B4F5801F01D1C16319E016
:109848001C6B04F44014B4F5001F0BD14FF4004313
:109858000FE000BF0010024000127A0000093D002E
:10986800200000201B6B03F44013B3F5401F01D107
:10987800134BC363126B134B12F4400F03D1C0F8A0
:1098880040E0BDE8F0811A6B02F44002B2F5800FA7
:1098980002D10164BDE8F0811A6B02F44002B2F50E
:1098A800000F02D14FF4004306E01B6B03F44003A2
:1098B800B3F5400F01D1024B0364BDE8F08100BF4E
:1098C80000127A000010024038B52DED048B4A4C86
:1098D8000368C4F830318388A4F83431023A0D465D
:1098E800062A05D8DFE802F00A101822292F3500C9
:1098F800B4F830310B80B4F8323113E0B4F83231B7
:109908000B80B4F8303105E0B4F830315B420B809D
:10991800B4F832315B4205E0B4F832315B420B8077
:10992800B4F830316B80B4F834311DE0B4F830311C
:109938005B420B80B4F8323112E0B4F832310B805C
:10994800B4F830310CE0B4F830310B80B4F832316F
:1099580005E0B4F832315B420B80B4F830315B4239
:109968006B80B4F834315B42AB80244B93F83430CD
:10997800002B3ED1B5F9003094ED510AD4ED4E7A62
:1099880009EE103AB5F9023008EE103AB8EEC88A76
:10999800B5F90430B8EEC99A28EE000A08EE903AF4
:1099A800A7EE890AF8EEE88AD4ED547AA7EEA80A59
:1099B8000BF0DEFF94ED520AD4ED4F7A288028EEA2
:1099C800000AA7EE890AD4ED557AA7EEA80A0BF08B
:1099D800CFFF94ED530AD4ED507A688028EE000A40
:1099E800A7EE890AD4ED567AA7EEA80A0BF0C0FFB5
:1099F800A880BDEC048B38BDE020002020000020AA
:109A0800104BDFED117A1B689A89104B1B6883F3A2
:109A18001003D31A07EE103AB8EEC77A27EE277A62
:109A280007EE902AF8EEE77AC7EE277AFDEEE77A96
:109A380017EE900A6428A8BF642020EAE070C0B23C
:109A4800704700BFD81F00200000C842E81F002050
:109A5800094B1A68137844F6FB7103EB431300FBB8
:109A680003135078C0EB0030B3FBF0F39078B3FBEE
:109A7800F0F080B2704700BFD81F002008B50A4830
:109A880090F85D3100EB43030A22B3F86C1189B2F8
:109A9800A0F8741100F5BC7007F0BAFC80B2FFF7AB
:109AA800D7FF024B188008BDE0200020DC1F0020F3
:109AB80007EE900AF8EEE77ADFED0C6A9FED0C0AE4
:109AC800F5EEC07AF1EE10FAD4BFB1EE677AC7EEC0
:109AD800A67A08B5D8BFC7EE267A27EE800A02F024
:109AE800C5FB044B83ED000A08BD00BF8096184BE8
:109AF80035FA8E3C6C000020F8B59B4B1B68044679
:109B0800187818B1012800F068819BE2242C974D41
:109B18000CD006D80A2C00F0D9800D2C00F0D68085
:109B280046E12A2C06D02C2C04D041E1287068701C
:109B3800A8704EE18E4B69782F788C4A00205854D3
:109B48002FBB1978D770472921D1597850291ED1B0
:109B58009978472907D1D978472904D11979412912
:109B680001D10121D1709978814A522903D1D17844
:109B78004D2900F0918299787D4A472907D1D178FB
:109B8800532904D11279562A04BF0322EA70EA78CD
:109B9800764E022A39D0032A4CD0012A40F085801B
:109BA800BA1E072A00F28180DFE802F004080F13CA
:109BB8001A257F2A08F0E2F8686076E01B78532BB4
:109BC80073D16B685B426B606FE008F0D7F8A860F0
:109BD8006BE01B78572B68D1AB685B42AB6064E0E5
:109BE8001B78302B634B1A788CBF42F0020222F0AC
:109BF80002021A7059E0002008F020F9287354E096
:109C0800002008F01BF9E8814FE0072F06D0082F45
:109C18004BD1012008F012F9708246E0012008F0CB
:109C28000DF941F2184358434FF47A73B0FBF3F03F
:109C380030823AE0022F07D0032F0AD1002008F023
:109C4800FDF84D4B187030E0002008F0F7F830753B
:109C58002BE02AD93A1F9210337D0132D2B2013B50
:109C680002EB8303DBB2102B1FD8F91EC2F10102ED
:109C780001EB8202D2B2012A0BD0042A11D10020B2
:109C88005E1E08F0DBF83D4B98553D4B00229A5577
:109C980007E05E1E3B4A0020935508F0CFF83A4B88
:109CA80098553A4A136801331360304B2A2C18BF71
:109CB8009A7807F101074FF000000CBF01225440C9
:109CC8002F7068700CBF5A759C7082E0687D002800
:109CD80047D02F4B13F8012D2E495A708B42F9D1DA
:109CE800234A224C13785278402B85BF373B1B01FF
:109CF8001B01DBB298BF03F0F003402A8CBF373A50
:109D0800303AD2B21344AA78DBB29A4226D1212340
:109D18000B702149E0780B681E4A013301280B605B
:109D28000AD002281CD1722313701C4B228A1A8075
:109D38001B4B628A1A8013E0672313700D4B1B7844
:109D48009F070ED5174B62681A60A2685A60164BB7
:109D5800227B1A70154BE2891A8002E03F230B70B0
:109D6800002000236B7534E0D0070020E02200209B
:109D7800E6310020F01F0020601700209117002016
:109D8800811700206117002071170020BC260020D1
:109D9800E0020020CC020020C8260020F21F00208C
:109DA80048170020F81F0020F61F0020F41F00208D
:109DB8006B78687D0E2B9FBFA34A591C5170A34A2C
:109DC80098BFD454A04A18B993785C40947000E0C6
:109DD8000020003018BF0120F8BD9B4B997D002260
:109DE800082900F22F81DFE801F0050B0F15202B61
:109DF80048606A00B52C40F02581DA7501223AE006
:109E0800622C08BF022236E003229A751C765C7623
:109E18009C7617E104229A755A7E997EDC76224454
:109E2800D2B25A760A449A760CE105229A755A7E7D
:109E3800997E9C832244D2B25A760A449A7601E1EA
:109E480006229A755A7E997E2244D2B25A760A44DC
:109E58009A769A8B02EB0424A4B2B4F5AC7F88BF3F
:109E6800794A9C8384BF0121D1750022DA83002CB2
:109E780040F0E88007229A75E4E05A7E997E2244F1
:109E8800D2B25A760A449A76DA8BB2F5AC7F3CBFE6
:109E98006D49891802F1010238BF81F82040998B79
:109EA80092B29142DA83E5D9CCE008229A755B7EBA
:109EB800A34200F0C780644B0122DA750DE0644DBF
:109EC8009A7515F8012D6A70624A9542F9D1997E02
:109ED8005D4AA14206D03F232B705F4A5368013385
:109EE8005360AFE05D48016801310160D07D10B179
:109EF8003E232B70A6E021212970D17E062941D06E
:109F080004D8022907D0032923D0F8BD122959D033
:109F1800302967D0F8BD502129705149546A4C60E6
:109F2800946A0C60116B4FF47A7491FBF4F14D4C08
:109F3800218092F878114C4A19B1117841F0020148
:109F480002E0117821F002011170012283F87921D1
:109F580069E05321297092F82510CE0705D592F8AB
:109F68002420D51E6A426A4100E0024602F001013F
:109F780083F87811002A56D13B490A7822F0020268
:109F88000A7050E04F21297092F82B10CC0705D5A4
:109F980092F82A20D11E4A424A4100E0024602F0C5
:109FA800010183F8781122B92F490A7822F00202B8
:109FB8000A702E4A93F84F1011702D4AB3F84C10BE
:109FC800118030E0562129702A49546B0C8042F2E6
:109FD8001074916B91FBF4F1274C2180012182F8D8
:109FE8007A1120E04921297092F82410234A102977
:109FF80088BF10211170224914780022A2420ED283
:10A00800204D0E7A5655204D4E7A56551F4DCE7A14
:10A0180056551F4D11F80C6F56550132EEE71D4984
:10A028000A6801320A6093F87931074A002B3AD05E
:10A0380092F87A31BBB3002182F8791182F87A114B
:10A048001846F8BD0020F8BDE0220020E6310020C7
:10A05800E0020020CC020020B0070020C826002023
:10A06800F81F0020F41F0020F01F0020F61F00201A
:10A078007A000020F21F00204817002060170020F7
:10A08800002300206117002071170020811700208D
:10A0980091170020BC2600201279432A7FF46BAD6B
:10A0A8000222EA7067E5F8BD0449054B0968187093
:10A0B80000225A6199611A77704700BFA8170020DB
:10A0C800B007002010B5121A07EE902A5B1A2DED82
:10A0D800028BB8EEE78A07EE903A434B059CF8EE00
:10A0E800E78AD3ED007A68EEA78A28EEA80AA8EED8
:10A0F800080A0BF08BFEB1EE488AB0EEE86AF0EE83
:10A10800C85ADFED3A7A049BB4EEE56AF1EE10FA2C
:10A1180020EE270AD4BFF0EE656AF0EE466ABCEE80
:10A12800C00AF5EE406AF1EE10FA83ED000A0BD092
:10A13800B4EEE56AF1EE10FA54BFF0EE657AF0EE8F
:10A14800467AC7EEA66A01E0DFED296ADFED297AD3
:10A158009FED297A9FED295AA6EEA77ADFED287A96
:10A16800E7EE267A9FED277AA7EEA67ADFED267A24
:10A17800E7EE267AF4EEC65AB1EE677ADFED237A77
:10A18800A6EEA75AF7EE007AE5EE267AF1EE10FA77
:10A19800C7EE277AC8BF9FED1E7ADFED1E6AF5EE7F
:10A1A800C08AC8BF77EE677AF1EE10FA48BF9FED14
:10A1B8001A7AB5EEC08A48BF77EE677AF1EE10FAE0
:10A1C8009FED167A48BFF1EE677AA7EEA67ABDEC46
:10A1D800028BFDEEC77A17EE903A002BBCBF03F551
:10A1E8000C43A033236010BD6C0000202C7D8E3FF3
:10A1F8000000000039094E3DE3B59EBE69A2163E37
:10A2080088FA16BE45FE7FBFA7DFA8B499FB243F96
:10A21800DB0FC93FA00CB345DB0F494000A00C463B
:10A2280044F25063984203DDA0F50C40A038704713
:10A23800034B9842BCBF00F50C40A030704700BFEC
:10A24800B0B9FFFF73B51A4C036823600B686360ED
:10A25800184D0068184EFFF72BFC184B009395E833
:10A26800030094E80C000196FFF72CFF144B3268AA
:10A278001A606868636813491B1A07EE903A124B14
:10A28800286893ED007A23681B1A0B600F4BF8EED1
:10A29800E77A1A600E4B67EE877A1B68FDEEE77A5D
:10A2A800DA880C4BC1ED017A1A8002B070BD00BF8C
:10A2B800782C0020F81F0020842C0020802C0020FF
:10A2C800C02C0020882C00206C000020B82C002016
:10A2D800040F0020B42C00204279DFED2A5A2A4BC3
:10A2E8009FED2A5A07EE902AF8EE677AC27BC7EEEE
:10A2F800A57AB2EE047AC3ED007A07EE902AF8EE5A
:10A30800677A234ADA60C7EEA57AC3ED017A8179C4
:10A31800204B07EE901AF8EE677A017CDA60C7EEF8
:10A32800877AC3ED007A07EE901A817E06EE101A3E
:10A33800F8EE677AB8EE466AC7EEA57A86EE056A41
:10A34800C3ED017A83ED026AC179134B06EE901AC8
:10A35800417CDA60F8EE666AC6EE876A07EE101A84
:10A36800C17EC3ED006A07EE901AB8EE477AF8EEA0
:10A37800677A87EE257AC7EE857A83ED017AC3ED91
:10A38800027A70470000C842902C002000007A44EE
:10A398000000FA44A02C0020C42C002010B50E4C5C
:10A3A80023789B0717D50D4B1B78042B13D90C4A20
:10A3B8000C4B106852685A601860FFF779FB0A4B1B
:10A3C8000A22B3F9043093FBF2F3084A1380237886
:10A3D80043F00103237010BDF01F0020F61F00207A
:10A3E800F81F00204C170020C0170020D42C002094
:10A3F8002DE9FF47734B744933F9103004462BB9E4
:10A4080002280CD0714B1B88980708D0704B00228B
:10A4180023F814206F4B1B8821F81430CFE031F853
:10A42800143023B96C4A02EB8402C2F87C31013340
:10A438009BB221F814301BB2002B1CDD022C664A9B
:10A4480066480BD1D2F88461B0F90450202095FBFE
:10A45800F0F505FB0060C2F884010CE002EB840211
:10A4680030F91450D2F87C61802095FBF0F505FB9B
:10A478000060C2F87C015A4F386890F8582093421F
:10A4880040F09D80544ADFF8488102EB840200EBDB
:10A49800040E022CD2F87C5195FBF3F39EF8515030
:10A4A800C2F87C3108BF5E424FF0000221F8142048
:10A4B80007BFB6B214219EB20A21002D7DD0002E0E
:10A4C8007BD038F81420002A77D00FFA86F90FFAD3
:10A4D80082FCE14571D089EAE9728CEAEC7AA2EB58
:10A4E800E972AAEBEC7ACAEB0202B9F1000F12B2D8
:10A4F80009B2DFF8F89003DDBCF1000F03DC20E0BF
:10A50800BCF1000F1DDA8A420BDD022C90F85420B2
:10A5180002D102F580720EE039F8141040320A4474
:10A5280019E049428A4218DA022C11D190F85420D5
:10A53800C2F57F42C032B9F804100A44A9F80420D1
:10A548000BE0002AB8BF52428A4206DD022C04D032
:10A5580039F81420203A29F8142039F914209EF8E3
:10A568004E9092114A4503DBAA42A8BF2A4691465B
:10A578001C4A126812031FFA89F508D5142001A98C
:10A588008DF804400293ADF80C50FEF7BBF8164B5B
:10A598001B7873B12AB207EE902AF8EEE77AB2EE8A
:10A5A800047AC7EE877A3B6803EB8403C3ED087A25
:10A5B80003E03B68234483F8019028F8146004B052
:10A5C800BDE8F087CC170020EC070020B42000205D
:10A5D800E6070020DE070020E0220020FC1600200D
:10A5E800D8070020D41F0020DC070020E007002047
:10A5F800094A13781844C0B210F0800F18BF803889
:10A6080010701346054A19781378994201BF002340
:10A618001370014A13707047892B0020882B002083
:10A6280010B50A4B0A4A1B7842609C18094A046014
:10A6380012789A4225BFD31A0B60C3F18003002316
:10A648002EBF4B600B604A6010BD00BF892B0020F5
:10A658008A2B0020882B00201FB5684602A9FFF727
:10A66800DFFF044B02981B6803440398184405B0A5
:10A678005DF804FB300600202DE9F04F89B08246D2
:10A6880001930023029103929946039A934205DAB3
:10A69800029A52F8232001339144F6E7019B4D4674
:10A6A800002B56D104F023FC002852D101987CE0FD
:10A6B80002223F4E8DF81C201A0C4FF480578DF85B
:10A6C8001D2006201A0A8DF81E208DF81F3004F070
:10A6D80033FC3785062007F067FA364BB76101224D
:10A6E8001A700020378507A9042207F085FA029F0F
:10A6F800D04626464FF0000B039B9B451EDABC460E
:10A7080057F8042B4FEA8B03002A47D0B24235D3BF
:10A7180032465AF80310CDF814C00020049307F00D
:10A728006BFA049BDDF814C05AF8032032444AF847
:10A738000320DCF800309E1BCCF800601C4B4FF463
:10A7480080529A611C4A13682D1B1C44019B14609B
:10A758004BB345B3184B1B68DCB22A19B2F5807F9E
:10A76800164AD2688CBFC4F580742C4693429FD396
:10A77800134A00231370134A137014E00020D8F80A
:10A78800001007F039FA57F8043CD8F80020F61AF8
:10A798001344C8F80030002347F8043C0BF1010BC0
:10A7A80008F10408A8E7C5EB090009B0BDE8F08F77
:10A7B800000400482D060020300600200C00002070
:10A7C800882B0020892B002030B50B4C0B4D2278AC
:10A7D8002B789A4285B00CD0684602A9FFF720FF73
:10A7E8000123684602A90222FFF746FF00232B70C7
:10A7F800237005B030BD00BF892B0020882B0020B6
:10A8080030B50E4D0E4C2A7823789A4285B011D077
:10A81800684602A9FFF704FF002302A9022268463E
:10A82800FFF72AFFFFF7E4FE20782B781B1A58421F
:10A83800584100E0012005B030BD00BF892B002041
:10A84800882B0020054A064B10781B7883422EBFC0
:10A85800181AC0F18000C018704700BF892B00206B
:10A86800882B002008B508480CF0B8FAC0B20928AF
:10A878000246054B04DC01302021C0B29954F6E7AA
:10A8880000221A5408BD00BFA526002008B50748B5
:10A898000CF0A4FAC0B21428044B04D8421C20219E
:10A8A8001954D0B2F7E700221A5408BDA526002093
:10A8B8002DE9F74FA74C06F09BFC26686568A7684A
:10A8C800861BF643451BC71BED43FF43F60F804627
:10A8D800ED0FFF0F2EB93FB9002D00F08682B94663
:10A8E8002CE04FF0000929E0B14627E003EB8A0B82
:10A8F800BBF802301A050ED413F4805F1DBF964AC8
:10A908009BF801101268954A954B14BF52F8212004
:10A91800126843F82A20BBF80230D80516D49905E6
:10A928000AD5904B1B7813F0040F0CBF8E4A8F4A40
:10A938008B4B126843F82A2009F10109207B8C49C6
:10A948005FFA89FA82450B68D0D326E0894A5046D7
:10A95800594605F0D7F8884B1B885A0603D5504648
:10A968005946864A16E0580703D550465946844A40
:10A9780010E0190703D550465946824A0AE09A075B
:10A9880003D550465946804A04E0DB07D4D57F4AB0
:10A998005046594605F0B6F8CEE7DFF808E20093CE
:10A9A800BEF906307822A3F57A7353434FF47A72CE
:10A9B80093FBF2F303F22B1301930022F3465FFAA1
:10A9C80082FE864517D2009B03EB820EBEF802E09A
:10A9D8001EF4806F0DD0DFF88891019B39F822E0D2
:10A9E80040F2671A9E449EFBFAFC0AFB1CEE29F80B
:10A9F80022E00132E3E74DB308F5C333A0336360C7
:10AA0800637B544A13BB9373614B1B6813F0020FAB
:10AA18000AD0DFF894E19EF800E0BEF1000F03D001
:10AA28004FF0010E82F80EE0DA0506D5594BDB78B7
:10AA38001BB1A37B43F00203A3734A4B1B7813F0AB
:10AA4800050F02BFA37B43F00403A37394F80EE041
:10AA5800BEF1000F03D13F4B5B7B002B4FD094F826
:10AA68000DC01CF0010FACF10C031DD1BCF1030F9C
:10AA780007D8DFF8E8903C4A1EF0040F08BF4A46A2
:10AA880000E0364AACF1040CBCF1070F05D8DFF83A
:10AA98001CC11EF0010F18BF6246DBB2032B0ED893
:10AAA8001EF0020F3C4B06E0DBB2032B06D82F4BFF
:10AAB8002A4A1EF0020F18BF1A4600E0274A4FF034
:10AAC800000C5FFA8CF383420DD20B6803EB8C0306
:10AAD8005B881B0642BF224BD2F8009043F82C90AB
:10AAE8000CF1010CEDE785B1BEF1000F08D0637BD6
:10AAF800184A0133DBB2142B06D1002304E025B138
:10AB0800637B002BF3D100E05373002E52D0234A0D
:10AB1800B2F90250B2F90020002DB8BF6D42002AE8
:10AB28004FF03203B8BF524295FBF3F592FBF3F2B4
:10AB3800EDB2D3B2AB4238BF2B46194A13B192FBE0
:10AB4800F3F300E0134643442360E37B014A7BBBF5
:10AB580001232EE06824002094260020DC920108BE
:10AB68003A0D002032340020A082010890820108AA
:10AB7800B8200020887A0108B42000208E7A0108C5
:10AB8800947A01089A7A0108A07A0108A67A01083D
:10AB9800D41F0020B0330020A8820108CC17002061
:10ABA800400D0300F63100203C200020B08201084F
:10ABB8000023D3738E4D8F4B2D78E27BADB9002FD8
:10ABC80000F00E818C4B267B1A788C4B8C4D93F8B9
:10ABD80000C08C4BD3F800E00B6802F0040200219F
:10ABE800D2B203EB86060F46B5E01AB9864A1A6157
:10ABF800002508E0854AFAE70A68AB00D618768887
:10AC0800760604D40135EBB28342F5D3D7E7804EFC
:10AC1800B6F90060192E25DD12F803E094F814C087
:10AC280026690EF00F09E1450CDCDFF8C8C19CF875
:10AC380015C0BCEB1E1FDEBFDFF8D8E1D6F800C098
:10AC480043F80EC012F803E094F816C00EF00F098E
:10AC5800E14533DBDFF89CC19CF815C0BCEB1E1F37
:10AC68002CDC26E0193629DA12F803E094F814C02F
:10AC780026690EF00F09E1450CDCDFF878C19CF875
:10AC880017C0BCEB1E1FA2BFDFF888E1D6F800C0D2
:10AC980043F80EC012F803E094F816C00EF00F093E
:10ACA800E1450BDBDFF84CC19CF817C0BCEB1E1F5D
:10ACB80004DBD6F800E0574E43F806E0544EB6F9E8
:10ACC8000260192E1BDD12F803C094F814E02669FF
:10ACD8000CF00F09F1450CDCDFF8189199F8159084
:10ACE800B9EB1C1FDEBFDFF82CC1D6F8009043F883
:10ACF8000C90D25C02F00F0CF4451EDD82E7193689
:10AD080080DA12F803C094F816E026690CF00F09EF
:10AD1800F1450CDBDFF8DC9099F81590B9EB1C1FB6
:10AD2800DEBFDFF8F0C0D6F8009043F80C90D25C94
:10AD380002F00F0CF445FFF665AF94F817E0BEEB90
:10AD4800121FA2BF334A36689E505BE75888000539
:10AD580004D404330435B342F8D122E04AB101EBFC
:10AD68000C0A06209AFBF0F900FB19A001280DDC5B
:10AD780001E057B9012793F801900EEB89003EF8DE
:10AD880029A090F80290C07803E017460020814679
:10AD98008246013125F802AC85F800906870C9B286
:10ADA800D7E7164A1378013B13F0FF0308BF0623C1
:10ADB8001370114B1B785B0741BFBBF90630A3F535
:10ADC8007A7303EBC3034FF47A7243BF93FBF2F336
:10ADD8000133DBB20123104A92FBF3F34344A3602F
:10ADE80003B0BDE8F04FFAF781BC03B0BDE8F08FBF
:10ADF800E80D00206824002032340020580000208C
:10AE08003C0D002094260020AC820108DC92010849
:10AE1800CC1700203A0D0020400D03002DE9F04F1B
:10AE28002DED028B85B083460393894B02921B88D4
:10AE38009D0737D5109B8748DC89B0F900301B1B6C
:10AE480003F2F31540F2E632954203D8002BB8BF5F
:10AE58005B4201E04FF4FA73B0F90220121B02F2D0
:10AE6800F31440F2E630844203D8002AB8BF5242B5
:10AE780001E04FF4FA729342B8BF1346C3F5FA7370
:10AE8800052293FBF2F30A22643B53439BF81C20F0
:10AE9800D2105343642293FBF2F3134423EAE3737F
:10AEA800DBB200E064230093CB1C0193D846002555
:10AEB800019B694813F8011F0193022D4FEA450AC7
:10AEC80006D1B0F9040001F11B044443631131E0D9
:10AED80030F81530614830F91500022413FB0400DE
:10AEE8001AB2029B5B42984203DB029B8342A8BFD3
:10AEF80003465B4830F90A40039830F915001B1BDC
:10AF08001844534B1E88F40710D41B3151430B11BE
:10AF1800B1070FD59BF812409DF9001044434C43EC
:10AF2800642294FBF2F203EB221303E09BF808304F
:10AF380043431B114B4A4C4832F90A202F5C042426
:10AF480092FBF4F41C1B98F8013063437B436422A2
:10AF5800022D93FBF2F34FEAE31308EE103A09D1FE
:10AF6800B8EEC80A04301E21DFED400A00F0BAFE30
:10AF7800BDEEC08A3E4B3F481B8898F80BE050F85E
:10AF8800251003FB04F6F6120EFB0616B6F5001F95
:10AF98003949A8BF4FF4001600F10C0E8E42B8BF15
:10AFA8000E465EF825104EF82540611A1B094FF62B
:10AFB800FF74B4FBF3F34B439BF84D1040F8256046
:10AFC8004FEA850976139B1171B107EE903A183054
:10AFD800B8EEE70A00EBC500DFED240A00F082FEB8
:10AFE800FDEEC07A17EE903A98F8151003EB43037C
:10AFF8004B435F43642397FBF3F718EE103A3F1275
:10B0080033441E493B4421F80A30114B1B881A056A
:10B0180006D51B4B1B785B0702D5E8B2FFF7E8F9AA
:10B02800184B18EE102A03F10C0149F803200135DA
:10B038001833032D49F8016049F8037008F1010835
:10B048007FF436AF05B0BDEC028BBDE8F08F00BFD2
:10B05800B4200020F6310020CC1700202A3400202C
:10B06800C0170020FC160020802400206F12833AAD
:10B07800401700208C2400200000E0FFBC240020A2
:10B0880032340020C42400202D4B2E4A93ED1B5A45
:10B09800D3ED1C4AD3ED1A5AD2ED003A25EE452AD3
:10B0A800F7EE007AB0EE004AB0EE673AA2EE043A44
:10B0B80064EEE41A25EE856AA1EE843AF1EE632A7D
:10B0C80083ED1D3AB0EE463AA3EEA46AA2EEA43A86
:10B0D80036EE066A65EEA46A83ED206A25EEE56A17
:10B0E80025EE247AE6EE047A33EE033AB0EE676A88
:10B0F800A1EE846A83ED1E3A83ED216AB0EE663ACA
:10B10800B0EE476AA3EE853AA2EEA56AE2EE856A3A
:10B11800A3EEA57AE2EE047A33EE033A36EE066A37
:10B1280076EEA66A37EE077A83ED1F3A83ED226A38
:10B13800C3ED236A83ED247AC3ED257A704700BFF7
:10B14800802400205C0000202DE9F04F2DED0C8BB1
:10B1580089B011F0FD0F06460191B24C06D0B24DF0
:10B168002B689F0700F1E78000F019BDD4F89C30E8
:10B17800AE48AE4F98470028F1D094F8AC20384636
:10B188003946FEF7A1FBAA4B04AA03F1080C1546A1
:10B19800186859689646AEE8030008336345724656
:10B1A800F6D118689B88CEF80000AEF80430BDF8D8
:10B1B8001CC0A048002100220346964633F8028F9F
:10B1C80035F8029023F8028C02320C2A18FB09EE9B
:10B1D800F4D137F8113083814FF4807213FB0CE3FC
:10B1E80093FBF2F327F811300131032900F10E0027
:10B1F800E1D1914BDFF85CA21A889846002A72D0F8
:10B20800D4F8D8301B7808EE103AAAF14809AAF108
:10B218003C054FF0000BB8F8000037F91B10B0F5EB
:10B228007A7F02BF0023C9F800302B61D9F80030BB
:10B238000B44C9F800302B6907EE901A0133012B33
:10B248004FEA4B02F8EEE77A2B6106D10023C5EDF1
:10B25800017AC5ED007AAB601BE0D5ED006A07EE18
:10B26800103A37EEE66AB8EEC77A86EE077A36EE17
:10B27800877AD5ED026A85ED017A77EEC77A85ED92
:10B28800007AE6EE276AF0EE667AC5ED036AC5ED48
:10B29800026A00230128BB522AF802302FD12B69F9
:10B2A8000392012BC3BF03F1FF3300EE103AD5ED33
:10B2B800037A9FED620A0290C4BFB8EEC00A87EE17
:10B2C800800A0AF0A3FD0298039A18EE103A63B1B7
:10B2D800F8EEC87AB4EEE70AF1EE10FA05DD4FF49D
:10B2E8007A73A8F8003000231AE0D9F800304FF438
:10B2F8007A7103F5FA7393FBF1F32AF802300BF134
:10B30800010BBBF1030F09F1040905F1140582D102
:10B31800012801D105F0D4FFB8F80030013BE0E77F
:10B3280037F813203AF81310521A27F8132001336C
:10B33800032BF5D113E7019B002B00F03084394F24
:10B348003F4B07F595705B68984707F59579002896
:10B3580000F0F8803B4B48461A784946FEF7B4FAA5
:10B36800B7F83031002B41D0D7F834010023B4F8B6
:10B378003021354939F913E02A4FB2F5C87F04BFA7
:10B38800002241F823204FEA830C51F80C20724424
:10B3980041F80C20002129F8131020F8131001336C
:10B3A800032BE4D1B7F83031012B1AD1D7F8383153
:10B3B8004FF4C87EC83393FBFEF20280D7F83C21D5
:10B3C800C83292FBFEF24280204AD7F840311288F8
:10B3D800C83393FBFEF39B1A83803180718001F0A0
:10B3E80029FAB4F83031013BA4F83031184B1B6806
:10B3F800580740F19380B4F844210A4B322A2BD1E4
:10B40800D3F834211188A3F8461151889288A3F8FB
:10B418004A213288A3F84C217288A3F84811A3F86E
:10B428004E211BE080240020EC1F0020FC16002089
:10B43800AC7A01082E2500202E34002000000000E0
:10B44800F82C002033340020B82500201C000020F0
:10B45800D41F0020A4250020002A3ED0D4F834C1EF
:10B468000023B4F8442139F91300A84F322AA84A16
:10B4780004BF002142F823104FEA830E52F80E1041
:10B48800014442F80E10002229F813202CF813204A
:10B498000133032B1146E4D1B7F84431012B17D1FE
:10B4A8000C2087F85C2187F85D3105F009FFD7F893
:10B4B8003431B7F846211A80B7F848215A80B7F8CE
:10B4C8004A219A80B7F84C313380B7F84E317380EF
:10B4D800B4F84431013BA4F8443194F85E318B4A06
:10B4E800E3B1D2F83401D2F85071002182F85E112C
:10B4F8004FF0320E97FBFEF70780D2F8547197FB96
:10B50800FEF74780D2F85831824A93FBFEF312883F
:10B518009B1A83803180718001F08CF9D4F8342132
:10B52800B4F82A3111885B1AA4F82A315188B4F882
:10B538002C315B1AA4F82C319288B4F82E319B1A5E
:10B54800A4F82E3105F054FED4F86031B4F82C215B
:10B55800C4F86001C31A08EE903AB4F82A316E4F65
:10B5680012FB02F213FB0322B4F82E31642113FB01
:10B57800032301FB03F267490B885B4392FBF3F358
:10B58800493B3B2B884624D80026D4F864311978E7
:10B59800A9B139F91630DFED617A614800EE103A49
:10B5A800F8EE680AB8EEC00A60EEA70A00EBC6001B
:10B5B80000F098FBFDEEC07A17EE903A01E039F8FA
:10B5C800163027F816300136032EDED14FF0010968
:10B5D80001E04FF000092A68524912F0080F08D01C
:10B5E800B1F900302BB1B1F9023013B1B1F904301F
:10B5F8008BBB4D4B187800F0100505F0FF0375B3B1
:10B6080012F020032BD000F0020202F0FF0332B345
:10B61800464B1B78042B21D9454B1B88B3F5967FE5
:10B628001CD3444B1B8807EE903A434BB3F90430C4
:10B63800B8EEE77A07EE903AF8EEE77AB2EE040A47
:10B64800C7EE807A012300209FED3C0A77EE677AE7
:10B6580067EE807A06E00023012001E00023184607
:10B66800DFED3B7A364A9FED2D7AB2F9005094ED22
:10B67800605AB1F802B07E88B7F804A0B8EE689AAC
:10B6880029EE079A07EE105AB2F90250B2F90420CF
:10B698000BEE105A06EE102AB8EEC77AB8EECBBAFF
:10B6A800B8EEC66A0A883D88898827EE05CA2BEE57
:10B6B80005BA26EE05AA002B4ED09FED227AF4EEAD
:10B6C800C77AF1EE10FA04DD9FED1F7A77EEC77A9C
:10B6D800F3E79FED1E7AF4EEC77AF1EE10FA04D57F
:10B6E8009FED197A77EE877AF3E7B6EE000A27EE30
:10B6F800800A03900291019200F057FDDFED14BA21
:10B70800019A0299039870EE2BBA27E08024002052
:10B71800D02500201C000020B2170020BD37863538
:10B72800E825002002170020F01F0020F61F002047
:10B73800F21F002048170020C017002035FA8E3C61
:10B74800FC160020DB0F4940DB0FC940DB0F49C066
:10B75800000000000AD7233C5FED03BA5FED049AAE
:10B76800F7EE00AA002857D013B207EE103A0FFAE6
:10B778008BF308EE103A0BB200EE103AB8EEC7DAC7
:10B78800F8EEC0CAB8EEC88A2DEE0D0A5FED0F7A42
:10B79800A8EE080AACEEAC0AB4EEE70AF1EE10FA2D
:10B7A8003ADD0AF033FB8AEE800AD4ED1E7AD4ED36
:10B7B8001D6A28EE008A2DEE007A68EE277A2CEEB4
:10B7C800800AE6EE877AD4ED1F6AE6EE807AD4ED39
:10B7D800216A28EE268AD4ED206AA6EE878A94ED9F
:10B7E800227AA7EE008AF0EE69CA28EE080AA7EEC8
:10B7F800A70A0AF00BFBD4ED237A20EE480AB0EE34
:10B80800698AE7EE80CAD4ED247AA7EE808AD4ED5F
:10B81800257AE7EE80BA03E0B0EE698AF0EE69CAED
:10B82800B9F1000F3ED02BB207EE103A33B206EE54
:10B83800903A0FFA8AF300EE103AF8EEC79AB8EE8B
:10B84800C0DAF8EEE6DA29EEA90A5FED3E7AADEE47
:10B85800AD0AADEE0D0AB4EEE70AF1EE10FA21DDFD
:10B868000AF0D4FA8AEE800AD4ED245A94ED256AB7
:10B8780029EE807A6DEE806A2DEE000A65EEC07AB8
:10B88800E6EE867A26EE476A7CEEA7CAD4ED237ADE
:10B89800A0EE276A67EEE67A38EE068AE7EE257AA2
:10B8A8007BEEA7BAD4F86491C34BD9ED017AF5EED3
:10B8B800C07AF1EE10FA4FF000021ADD67EEAC6ABA
:10B8C80093ED617AA6EE897A67EE886A83ED617AEC
:10B8D80093ED627AA6EE897A67EEAB7A83ED627AA7
:10B8E80093ED637AA7EE897AF0EE477A83ED637A6F
:10B8F80005E0C3F88421C3F88821C3F88C21AF4D33
:10B9080099ED025A2B78590709D4AD4B1A6844F6B9
:10B918001F639A429CBFF2EE047A25EE275AD4EDB3
:10B92800636A94ED617AD4ED627AA64EE5EE2B6AED
:10B93800E5EE087AA5EE2C7A3AEE266AF6EE006A6B
:10B948007BEE277A69EE266A3CEE077A67EEA65AFE
:10B9580027EE267A66EE266A94ED1B6A96ED005A63
:10B96800D4ED1A7A94ED1CBA66EE269A25EEC6AA8C
:10B97800E5EE079AA7EEC7AAF1EE4B4A26EEE78A4C
:10B98800E4EEA59AA4EEA6AAA5EE258A77EEA99AD2
:10B9980067EEA57AABEE078A35EE0AAAE5EE267AB7
:10B9A80029EEA90AE6EE477AAAEE0A0A36EE088ACE
:10B9B8003BEE27BAA8EE080AABEE0B0A0AF026FA05
:10B9C8008AEE800A6BEE007A2AEE00AA69EE809A67
:10B9D80028EE008AC4ED1C7A86ED00AAC4ED1A9AF6
:10B9E80084ED1B8AFFF750FBD4ED259AD4ED24AAE9
:10B9F8009FED75BA754EF0EE690AB0EE6A0A0AF064
:10BA08005FF820EE0B0A09F0B3FF94ED23AA30800B
:10BA1800B1EE4A0A09F0F6FFDFED6D7A37EEC00A9B
:10BA280020EE0B0A09F0A4FF94ED208AD4ED1DBA8C
:10BA38007080F0EE6B0AB0EE480A0AF041F8D4EDD7
:10BA4800647AE0EE4B7AB0EE670A09F091FF83B2B0
:10BA58001A0458BFB380D4ED657A5E4B94ED1E0A84
:10BA68001A78D4ED215A5449F4EEE79A44BF00F508
:10BA78006160B080F1EE10FACCBF42F0080222F00B
:10BA880008021A70B7F90030D4ED1F7A06EE103AA2
:10BA9800B7F9023007EE103AB8EEC77AB8EEC66AC0
:10BAA800B7F9043027EE000A06EE903AABEE860AA4
:10BAB80099F80130F8EEE66A012BA7EEA60A6AEEBD
:10BAC800877A27EE257AEAEE067AA8EE067A94EDCA
:10BAD800226AA6EE267AE9EEA67AF1EE479A18D1FE
:10BAE8002B785B070FD4D1F89831402293FBF2F200
:10BAF8009B1A07EE103AB8EEC77A37EE277ABDEEF2
:10BB0800C77A81ED667AD4F89831402293FBF2F334
:10BB180001E0B8F8003094ED678A07EE103AB8EE05
:10BB2800C77A77EEC77A94ED687A39EE077A77EEB6
:10BB3800C87A89EE079AA9EE278A84ED678A09F000
:10BB480017FFD4F8A451297800F020FBD4F8A831C5
:10BB5800B0EE690A1844C4F8A80109F009FF297869
:10BB680000F014FBD4F8AC31B0EE480A1844C4F81D
:10BB7800AC0109F0FDFE697800F008FBD4F8B0319B
:10BB8800154A184418EE901A1368C4F8B0011944FD
:10BB9800D4F8B43111600133C4F8B43106E000239D
:10BBA800A4F82A31A4F82C31A4F82E3109B0BDEC40
:10BBB8000C8BBDE8F08F00BF8024002032340020B9
:10BBC800A81700205C0000204C3D0F44C01700203F
:10BBD800DB0FC93FF01F002014340020F0B501240A
:10BBE800B0FBF4F58D4201D34C43F9E70026D4B1FC
:10BBF800B0FBF4F504FB1500B4FBF1F41EB9002DFD
:10BC080001DC002CF3D1092D03F1010EEFB204DDA4
:10BC1800002A14BF3725572500E030253D441D7004
:10BC280001367346E3E71C70F0BDF0B50124B0FBA4
:10BC3800F4F58D4201D34C43F9E70026D4B1B0FBAB
:10BC4800F4F504FB1500B4FBF1F41EB9002D01DC7A
:10BC5800002CF3D1092D03F1010EEFB204DD002A07
:10BC680014BF3725572500E030253D441D700136A7
:10BC78007346E3E71C70F0BD03685A1C0260197034
:10BC880070472DE9F843089E002B0746884614465E
:10BC980014BF4FF030094FF02009334613F8012B39
:10BCA8000AB9254603E0002CFBDD013CF6E7002D30
:10BCB80004DD38464946C047013DF8E724EAE47404
:10BCC8003546A01B284415F8011B11B13846C0475A
:10BCD800F7E7BDE8F883024B186805F096BB00BF8C
:10BCE800E80F002090ED017A07EE901AB5EE407A41
:10BCF800F1EE10FA01BFF8EEE77A9FED0E7A67EEE3
:10BD0800877AB7EE007A04BFC7EE277AC0ED017ACA
:10BD180090ED017AD0ED007A30EE877A30EE670A3E
:10BD2800C0EE870AE0EE807AB0EE670AC0ED007ACE
:10BD3800704700BFDB0FC94010B50278202A0346C0
:10BD480000F10100F9D0092AF7D02D2A03D10346C2
:10BD5800BFEE000A04E02B2A08BF0346B7EE000A2C
:10BD6800DFED387A1A46134612F8010BA0F13001BC
:10BD7800CCB2092C0AD807EE101AB8EEC77AF2EE40
:10BD8800046AA7EEA67AF0EE477AECE72E2816D1D9
:10BD9800F2EE046A1146B0EE666A0B4611F8012B02
:10BDA800303AD0B209280AD807EE102AB8EEC77A76
:10BDB80087EE267A66EE866A77EE877AEDE71A7856
:10BDC80002F0DF02452A35D15A782D2A02D10233F2
:10BDD800012004E02B2A14BF013302330020013B69
:10BDE800002213F8011F3039CCB2092C03D80A24D9
:10BDF80004FB0212F5E7B2F59A7F28BF4FF49A7256
:10BE08001346B7EE007A072B05D9DFED0F6A083B1A
:10BE180027EE267AF7E702F007032BB1F2EE046A61
:10BE280027EE267A013BF8E7F0EE476A20B1C7EE25
:10BE3800877A03E0F7EE006A67EEA67A20EE270A13
:10BE480010BD00BF0000000020BCBE4C30B52DED79
:10BE5800028B87B0B0EE408A0C220021054603A869
:10BE68000AF07CFFB5EEC08ADFED2A7AF1EE10FA0F
:10BE7800CCBF38EE278A38EE678ADFED277A28EEBE
:10BE8800278A6946FDEEC87A17EE904A84EAE4707C
:10BE9800A0EBE470FDF756F9002CACBF20232D234E
:10BEA80068468DF80C300AF099FF012807D1302335
:10BEB8008DF80D308DF80E308DF80F300CE002281B
:10BEC80005D130238DF80D308DF80E3004E00328AD
:10BED80004BF30238DF80D30694603A80AF064FFCB
:10BEE80003A80AF07BFF0338C4B2224603A92846F8
:10BEF8000AF09EFF00232B55284608490AF054FFF4
:10BF080003AB284619190AF04FFF284607B0BDECC5
:10BF1800028B30BD6F12033A00007A44C3990108BE
:10BF280070B5064615460846B6FBF2F414B120462D
:10BF3800FFF7F6FF05FB1464024B1B5D00F8013B9D
:10BF480070BD00BFC59901082DE9F04F814689B041
:10BF58008A4616461C4600253178002900F0DD8007
:10BF6800252902D00136484675E07278302A08BF84
:10BF7800B278A2F1300319BFB71C4FF0000BF71CC1
:10BF88004FF0010B092B4FF0000819D8A2F130032C
:10BF9800D9B2092905D80A2202FB083817F8012B5B
:10BFA800F4E7A2F16103052B02D8A2F1570305E0DB
:10BFB800A2F14103052B03D8A2F137030A2BEADDCE
:10BFC8006C2A31D13A78642A07F1010600F083809F
:10BFD8000BD8252A3DD003D8002A00F09E80BBE765
:10BFE800582A0CD0632A19D0B6E7732A22D002D86F
:10BFF8006E2A37D0B0E7752A5CD0782AACD1271DD5
:10C008002068A2F1580462424FF01001624155E0E5
:10C018002CD9582A32D0632A2AD13E46484621785C
:10C02800271DD04701350FE0642A64D00ED9732A42
:10C0380014D13E46236800934846514642460023A1
:10C04800FFF71FFE271D05443C4685E7252ADFD15B
:10C058003E4648462521D04701357DE70AD86E2A55
:10C0680006D13E46236804341D6075E7002A54D083
:10C078003E4671E7752A26D0782AF9D1A2F15803ED
:10C0880004F1040C5A422068CDF80CC04FF010019E
:10C098005A4105ABFFF7A2FDDDF80CC03E466446E9
:10C0A80005AB00934846514642465B46FFF7E9FD1B
:10C0B800054451E72068271D0A21002205ABFFF738
:10C0C800B4FD3C46ECE704F1040CCDF80CC0206844
:10C0D8000A210022DDE72068002804F1040708DAB5
:10C0E8002D238DF8143040420DF115030A2100224A
:10C0F800E5E705ABFAE72068002804F1040C0ADA42
:10C108002D238DF8143040420DF11503CDF80CC0E5
:10C118000A210022BEE705ABF8E7284609B0BDE8CA
:10C12800F08F0EB40FB505AB019053F8042B0649F8
:10C13800039301A8FFF708FF019B00221A7004B0BF
:10C148005DF804EB03B0704781BC00080FB413B569
:10C158000B4904AB08680B4953F8042B0968019391
:10C16800FFF7F2FE0446084B186805F042F900286C
:10C17800F9D0204602B0BDE8104004B0704700BFB7
:10C18800F4000020F0000020E80F002080EAE073AF
:10C19800A3EBE0738B4206DB002801DD401A7047F1
:10C1A80002D00844704700207047FDEEC07A17EEB1
:10C1B800903A2033402B43D8DFED237AB4EEE70AD8
:10C1C800F1EE10FA04DDDFED217A30EE670AF3E7CD
:10C1D800DFED1F7AB4EEE70AF1EE10FA04D5DFEDD1
:10C1E8001B7A30EE270AF3E7DFED1A7AB4EEE70A96
:10C1F800F1EE10FA04DD30EE670A37EEC00A0AE005
:10C208009FED157AB4EEC70AF1EE10FA44BF30EE8E
:10C21800270A37EE400A60EE007ADFED106A9FEDDC
:10C22800107AA7EEA67ADFED0F6AE7EE876A9FED30
:10C238000E7AA7EEA67A20EE276AA6EE070A7047BE
:10C248009FED060A704700BFDB0F4940DB0FC9406E
:10C25800DB0F49C0DB0FC93FDB0FC9BF000000007F
:10C2680092E741B99730083C15A82ABEDFED027A5B
:10C2780030EE270A99E700BFDB0FC93F064B1A8843
:10C2880022EA0000904210B518801C4602D0012016
:10C2980005F038F8208810BDB4200020064B1A8815
:10C2A8001043904210B518801C4602D0012005F0BA
:10C2B80029F8208810BD00BFB4200020024A9368E6
:10C2C80023EA000090607047D4170020024A936860
:10C2D80018439060704700BFD417002008B5104B72
:10C2E8001A780023D9B2914207D20E4951F8231087
:10C2F8000968002008600133F4E7322004F09FFF4A
:10C30800094B1B685A0309D5084B9B685B0305D486
:10C3180040F2DC50BDE8084004F091BF08BD00BF02
:10C328007C2E00204C2E0020D41F0020D417002083
:10C338002DE9F34105F07EFF454A702313704FF451
:10C3480000635380BE231371EF2382F8FC37002368
:10C3580082F8FD3719461646F25C0133B3F5006FD3
:10C3680081EA0201F8D13A4B83F8FD17394B1A6973
:10C37800120604D5384A5A6002F188325A600427F6
:10C388000020013F17F0FF074FD0324B3422DA600C
:10C39800002444B1002356F804800193FCF7A2FE60
:10C3A8000428EED117E0FCF79DFE0428E9D1294DB9
:10C3B8002B6943F002032B61284B6B612B6943F017
:10C3C80040032B61FCF78EFE2B69042823F002033F
:10C3D8002B61DFD0D5E71F4D2B6943F001032B619B
:10C3E80004F1006303F57C331FFA88F21A80FCF726
:10C3F80079FE042810D11A4B23440193019B4FEA7C
:10C408001848A3F80080FCF76DFE2B69042823F078
:10C4180001032B6105D0B4E72B6923F001032B61DD
:10C42800AFE70434B4F5006FB3D10A4A136904289E
:10C4380043F08003136102D102F095FE10B9052084
:10C4480004F078FF05F0E0FE02B0BDE8F08100BF1F
:10C45800D4170020002002402301674500F003089C
:10C4680002F0030810B50E4C206804F02BFE20687B
:10C47800047A002202FB02F3193B634303F6C41358
:10C488005343192193FBF1F3064921F81230013285
:10C49800072AEFD10449BDE81040FBF751BF00BFA0
:10C4A80044170020900F0020141900202DE9F041B6
:10C4B80002F059FE10B9042004F03CFFB34CB44D0F
:10C4C80005F0B8FEB3494FF4006220460AF03DFC7F
:10C4D80094F8CC37022B84BF002384F8CC3794F827
:10C4E800CC274FF4D07101FB02F3E018234400F588
:10C4F8003B70286093F8480303F55073022801FB4A
:10C50800024284BF0020187292F84833A24A13707E
:10C518000C2202FB0343A14A03F2CE731360A26804
:10C5280046F2090313401BB94FF40050FFF7CEFE43
:10C53800A368D80703D54FF40050FFF7BFFEA368E0
:10C54800590409D50820FFF7B9FE4FF40050FFF74A
:10C55800B5FE0120FFF7B2FEA3681A0706D54FF40F
:10C568000050FFF7ABFE0120FFF7A8FEA3689B046D
:10C5780002D54020FFF7A2FE012284F81D2294F87C
:10C58800DE21824B2AB193F8E22112B1002283F80E
:10C59800E221834B834E1E604FF0000C674604EB8C
:10C5A8000C03B3F8F6E14FEA5E0101F077314FEA88
:10C5B8009E0303F03333C1EB0E00C11A4FEADE03CA
:10C5C80003F01133CB1A03EB23131EF0010803F019
:10C5D8000F324FF0FF0392FBF3F3C3EB032318BFB3
:10C5E8000137A2EB030318BFFFB2012B0ADD022BB0
:10C5F80040F0C980B8F1000F00F0C5801EF0BC0FF4
:10C6080000F0C1800CF1080CBCF1280FC7D1013F24
:10C61800012F00F2B880FFF725FF30220021624881
:10C62800624F0AF09BFB624BD5F800801F60614B9C
:10C63800002108F18100C3F8008004F083FD5E4BFF
:10C6480080F0010018705D4B07F128021A605C4BFE
:10C6580007F1DC021A6098F80030022B594B14BF1E
:10C66800594A5A4A1A605A4B08F5C97240461A6024
:10C67800FDF732FE574B584994F8D6E1196064200B
:10C68800564BDFED576AC82210FB0E225A60002273
:10C698009A60DA601A615A619A61DA6183F8202037
:10C6A80083F821204F4BA1F168021A602B684E4A8B
:10C6B80003F2211010604D4A03F2911010604C4AA9
:10C6C800A1F18E0010604B4A17604B4A01F10C0033
:10C6D80010604A4A1631116049490E60B4F8641175
:10C6E80007EE101AB8EEC77AB4F8661187EE267A04
:10C6F800101D07EE901AF8EEE77A82ED037AC7EE7E
:10C70800A67A93F86410117193F88010517194F817
:10C71800E1111174B3F81E1193ED1A7ADFED396A3D
:10C72800C2ED027A67EE266AB6EE007A87EE267ABE
:10C7380007EE901A344908605361344A03F16C01DA
:10C748001160334A334982ED007AF8EEE77A9FEDBB
:10C75800327A324A0B60C7EE277A31499FED317A37
:10C7680067EE877AC2ED007A03F170020A602E49FB
:10C7780003F219130B602D4B1F602D4BBDE8F041E0
:10C788001A6005F041BDFCF781FC44E7D41700208E
:10C798001817002000F00308D82C002044170020A8
:10C7A800A43300205C190020C00E002014190020BA
:10C7B800F40E0020F80E00200A0000205825002062
:10C7C8000C0600207400002025AE0008B5220108E0
:10C7D800040F002004340020AA190020B0330020E0
:10C7E80000401C46B425002098260020F4080020AC
:10C7F800982F00209C2F00200808002038260020B1
:10C80800CC080020DB0F4940E42500202426002026
:10C8180020260020A407002000006144040800200E
:10C82800980700204C3D0F44F4070020FC07002027
:10C83800A006002008B5FFF77BFDFFF737FE0120B3
:10C84800BDE8084004F05EBD38B500240B4D6059C2
:10C85800254403F0C7FF696811B10948FFF776FC62
:10C86800A96811B10748FFF771FC0748103403F0B5
:10C87800B9FFB4F5F07FE9D138BD00BFC07A01082F
:10C88800EA990108F09901084CA5010870B5054618
:10C8980028460AF0A3FA064658B91A4B1A485A7994
:10C8A8001A4B03EB8203BDE87040D3F8DC11FFF7A5
:10C8B8004DBC2846164932460AF098FA60B9154820
:10C8C800154C03F08FFF54F8041F19B11348FFF7F4
:10C8D8003DFCF8E7124805E00024124B53F82410F9
:10C8E80021B91148BDE8704003F07CBF28463246A4
:10C8F8000AF07CFA01340028EFD1024B0B4D5C7131
:10C90800C6E700BFD4170020F6990108C07A0108CD
:10C91800029A0108079A01089C7C01081A9A0108E2
:10C928004CA50108A07C0108C298010810960108CE
:10C93800F0B585B004460AF051FA082826D1621EDF
:10C94800E01D1F4912F8013F09681944497801F0B0
:10C958000301022908BF203B82421370F1D125460A
:10C9680004F1080715F8016B164831460AF029FA50
:10C9780020B1284631460AF024FA10B1FAF740FFF0
:10C988001CE0BD42EED12046FCF7BEFB0E4803F08A
:10C9980029FF00230D4A1A4404A992F888210A4461
:10C9A8000849595C02F80C1C0133082BF2D100230A
:10C9B80007488DF80C3001A9FFF7C8FB05B0F0BD9A
:10C9C800800000203BB001081E9A0108D4170020FF
:10C9D800F0A30108264B274C1D68206880B5FBF79B
:10C9E80061FB2846FBF75EFB206841798A0703D480
:10C9F80041F0020104F0FAFC1F4B08229A611F4B18
:10CA08001A6812F4003F1F461FBF06236371E379BB
:10CA180023F001031CBF43F00203E371206804F014
:10CA2800F1FC90B1144E08233385124B186804F0BA
:10CA3800E6FC8046FDF760F808B103F02DF92846BA
:10CA4800414604F0E2FC0823B361284604F0DAFC0E
:10CA580038B12846266804F0D2FC0146304604F076
:10CA6800D4FC3B689B03D9D500F067FFD6E700BF2D
:10CA7800F42C00205026002000040048D41F002079
:10CA88002DE9F04105460AF0A9F92C4B04469E68A9
:10CA980088B92B4803F0A6FE2A4B53F8241041B15D
:10CAA8000123A340334202D02748FFF74FFB01344C
:10CAB800F2E7264821E02846254922460AF096F959
:10CAC80058B92448244C03F08DFE54F8041F00295B
:10CAD800EFD01D48FFF73AFBF7E72B782D2B03BF64
:10CAE800013504F1FF344FF001084FF0000800262B
:10CAF800144B53F8267027B91848BDE8F04103F0E5
:10CB080071BE2846394622460AF070F998B90120C4
:10CB1800B040B8F1000F03D0FFF7D0FB104802E097
:10CB2800FFF7D4FB0F4803F05DFE39460E48BDE819
:10CB3800F041FFF70BBB0136DAE700BFD41700203E
:10CB4800249A0108087D01081A9A01084CA50108D1
:10CB5800029A01082E9A0108047D0108C29801086A
:10CB68003A9A0108439A0108EFA3010810B508484A
:10CB780003F038FE074B00241C741C64064B1C7021
:10CB880004F0D2FD04F036F8044B1C6010BD00BF61
:10CB98004B9A01085026002034340020F42C002041
:10CBA800F8B5124C074604F60C56A3881F4219D054
:10CBB80025680F482946FFF7C9FA0E4928460AF0A2
:10CBC80049F9014640B1A3680B4A1B78013B52F86A
:10CBD800230003F007FE02E0204603F090FD07481B
:10CBE80003F000FE1434B442DFD1F8BD54840108C8
:10CBF800779A0108819A0108609101084CA50108FB
:10CC080008B50848FFF7A2FA02F0A6F902F06FF992
:10CC180018B9642004F013FBF8E70348BDE808409E
:10CC2800FFF794BA909A01089D9A01082DE9FF41EF
:10CC38000A48068885684488B0F80480C768FDF704
:10CC48000BFDCDF800800290019731462A46234615
:10CC58000348FFF77BFA04B0BDE8F0810C00002020
:10CC6800A59A0108F0B504788BB005460CB10024EC
:10CC780036E04B4B19680E2303FB041101F5907045
:10CC8800B1F92551B1F92121B1F92331009591F874
:10CC98002851019591F82951029590F907000390C0
:10CCA80001F594713F4891F902100491214601342D
:10CCB800FFF74CFA082CDCD170E02D2B14D1072C8F
:10CCC8001BDC284608F0E4FC0AAB661C03EB4404B2
:10CCD80024F8100C15F8013F303B092BFAD93446DB
:10CCE8002B78002BE9D104E0A3F13002092A09D8F6
:10CCF800E5E7082CBDF8182009D00BB0BDE8F040D6
:10CD0800FAF77EBD202BF8D101352646E7E7072A3A
:10CD1800F3D8BDF81A00224BA0F2EE2189B240F2F6
:10CD2800DC55A9421B68E8D8BDF81C10A1F2EE2416
:10CD3800A4B2AC42E1D8BDF81E6004B237B2A74233
:10CD4800DBDB0DB2AF42D8DCA542D6DBBDF82470E0
:10CD580007F16404A4B2C82CCFD8BDF826E00FFAB6
:10CD68008EF4112CC9DCBDF82050B42DC5D8BDF8FF
:10CD78002240B42CC1D812B24FF00E0C0CFB023377
:10CD8800A3F82101A3F82311A3F8256183F82851FA
:10CD980083F8294183F8277183F82AE10BB0F0BDA5
:10CDA80018170020029B0108F0B504468FB02046F2
:10CDB8000AF014F8C5B225BBAF48B04C03F012FD19
:10CDC80094F8D21009B9AE4854E049B294F8D0208A
:10CDD80094F8D130009194F8D310019194F9D410BB
:10CDE800029194F9D510039194F8D6100491A548AE
:10CDF80029460135FFF7AAF9102D04F10704DFD100
:10CE0800E1E72046A049052209F0F0FF0546B8B938
:10CE180029469E48702209F0A1FF9D4B19682846B3
:10CE28000E2303FB001301300022082883F82B216E
:10CE380083F82C2183F82D2183F82E21F0D119E1D4
:10CE480020469449042209F0D1FF05462046002DCA
:10CE58004AD1202109F0B5FF002800F00B81461CBB
:10CE6800304609F0BBFF2C4607468B4B53F824503D
:10CE78002DB98A480FB0BDE8F040FFF767B93046D2
:10CE88002946FAB209F0B2FF01340028EDD17B4AF5
:10CE980002F170011646002382F8D63082F8D230AB
:10CEA80082F8D13082F8D03007328A42F3D17C49F7
:10CEB80001EBC40191F8A022934210DAD1F8A472D0
:10CEC800C3EBC302B0183A4400F1D0011768C0F8A8
:10CED800D0709088888092798A710133E7E7294673
:10CEE8007048FFF733F996E06F49072209F07EFF93
:10CEF80005462046002D4AD1202109F062FF06464A
:10CF080009F06CFFC4B274BB6848FFF71FF92146EB
:10CF180067480134FFF71AF90E2CF8D15848FFF783
:10CF280015F9002463482146FFF710F90025584AEF
:10CF3800614811680E2202FB04120123D2F82B214A
:10CF48005E49AB4013425E4B05F1010508BF194627
:10CF5800FFF7FCF80E2DEAD149480134FFF7F6F83F
:10CF6800082CDFD186E03046564908F095FB2C4660
:10CF7800002852D0022C55D008F08AFB06AB514944
:10CF880043F82400002008F087FB0134F0E74D49FE
:10CF980008F082FB002460B1082C3ED008F078FB32
:10CFA80006AB484943F82400002008F075FB01341B
:10CFB800F1E7082C31D1069B0F2B2ED8DDF81CE0A9
:10CFC800BEF1070F29D8089F0D2F26D8099E06F114
:10CFD8006402C82A21D80A9DFF2D1ED80B98642800
:10CFE8001BD80C99642918D8884216DA0D9C032C92
:10CFF80013D8224AC3EBC303134483F8D0E083F861
:10D00800D17083F8D26083F8D35083F8D40083F8C2
:10D01800D51083F8D6402C4CC9E60FB0BDE8F040D7
:10D02800FAF7EEBB069B072B20D807990D291DD8C8
:10D038000278722A0DD06E2A18D1154A12680E206D
:10D0480000FB032301228A40D3F82B1121EA0202B4
:10D0580009E00F4A12680E2000FB032301228A40D0
:10D06800D3F82B110A43C3F82B2101E0FAF7C8FBC8
:10D078000D4C9CE60FB0F0BD2A9B0108D417002088
:10D088004CA50108559B010892980108A418002096
:10D0980018170020BD980108A07C0108C298010853
:10D0A800C07A0108D1980108229B0108F499010867
:10D0B800719B010827A30108769B0108FCA70108BA
:10D0C800B6A801087A9B0108109601082DE9F743D4
:10D0D800047805468CB9324D95F8AF12B5F8AC22F4
:10D0E80095F8AE322F48009121460134FFF72EF80B
:10D0F800102C05F10405EFD14EE008F0C9FA0F280D
:10D10800044636DC2846202109F05BFE264EE4B2B0
:10D11800D6F84480451CA4000027284608F0B8FA31
:10D128005FFA87F9B9F1010F83B208D0B9F1020F9C
:10D138000BD0B3F5B47F24D2726C13530AE0FF2BE3
:10D148001FD8736C2344987004E0FF2B19D8736CB4
:10D158002344D87028462C2109F033FE054608B12F
:10D16800013502E0B9F1020F0BD10137032FD4D1F9
:10D1780012E00E4800210F2203B0BDE8F043FAF791
:10D18800BCBA08EB04000021042209F0E7FD03B053
:10D19800BDE8F043FAF734BB03B0BDE8F08300BF45
:10D1A800D41700207C9B01085026002050980108C5
:10D1B8002DE9F0412DED048BB1498AB0044609F000
:10D1C800D5FDB049002820460CBF0126072609F0E6
:10D1D800CDFDAD490028204608BF022609F0C6FD4E
:10D1E800002808BF0426F10740F1F080A748A84CA2
:10D1F80003F0F8FA002003F0FBF8A64803F0F2FA6F
:10D20800A54803F0EFFA6279A44BA54803EB820323
:10D218002546D3F8DC11FEF799FFA248FEF796FFE2
:10D228004FF00008274695ED048AB5EE408AF1EEE6
:10D2380010FA04D19C48FEF789FF002570E09B484E
:10D24800D5ED059A95ED069AD5ED078A4146FEF784
:10D258007DFFB5EEC08AF1EE10FA02D5202003F06A
:10D26800B9FAB0EE480A06A8FEF7F0FD0146904864
:10D27800FEF76CFFF5EEC09AF1EE10FA02D5202009
:10D2880003F0A8FAB0EE690A06A8FEF7DFFD01462A
:10D298008748FEF75BFFB5EEC09AF1EE10FA02D5AB
:10D2A800202003F097FAB0EE490A06A8FEF7CEFD53
:10D2B80001467F48FEF74AFFF5EEC08AF1EE10FA04
:10D2C80002D5202003F086FAB0EE680A06A8FEF719
:10D2D800BDFD08F1010801467648FEF737FFB8F1B1
:10D2E8000C0F05F110059ED1A4E749B294F8D0209F
:10D2F80094F8D130009194F8D310019194F9D41096
:10D30800029194F9D510039194F8D61004916A48C3
:10D3180029460135FEF71AFF102D04F1070403D042
:10D3280094F8D2100029E0D16448654C03F05AFA09
:10D33800D7F8088054F8041F19B16248FEF706FFB1
:10D34800F8E70D46604B53F8254054B10123AB4034
:10D3580013EA080F03D05D482146FEF7F7FE0135B2
:10D36800F0E75B4803F03EFA21467B180AAA93F8D7
:10D3780088311344574A8A5C03F8102C0131082974
:10D38800F3D1002306A954488DF82030FEF7DEFEBD
:10D39800524803F027FA5248FAF706FF514803F0BB
:10D3A80021FA4F48FAF732FA4F4803F01BFA4C4873
:10D3B800FFF78CFE4D48FEF7C9FE4020FFF7F0FB53
:10D3C8004B4803F00FFA4648FAF750FDB20739D533
:10D3D800484803F007FA484803F004FA404803F0C5
:10D3E80047F8464803F0FEF93D48FAF793F94448F0
:10D3F80003F0F8F93A48FAF78BFC4248FEF7A6FE24
:10D408003748FAF70FFB404803F0ECF93448FFF7C8
:10D4180029FC00270E257D4300243C4A926C2A44AF
:10D428000123D2F80A20A34013421ED101340E2C46
:10D43800F3D10137082FEDD12C48FEF787FE802065
:10D44800FFF7AEFB730716D5314803F0CBF9314827
:10D4580003F0C8F9224802F0E5FF2448FEF776FEFB
:10D468004FF48070FFF79CFB05E0394622462A48B6
:10D47800FEF76CFEDAE70AB0BDEC048BBDE8F0817C
:10D48800909B010808A00108979B01089D9B010833
:10D49800D4170020AB9B0108BD9B0108C07A010886
:10D4A800C99B0108D49B0108E19B0108EE9B010878
:10D4B800F3990108F0A30108069C0108F69B0108EE
:10D4C800047D0108259C0108087D0108339C01089A
:10D4D800409C01083BB001084C9C0108559C010880
:10D4E80010960108649C0108709C01084CA501086D
:10D4F8007E9C01088B9C01089E9C0108AC9C01083D
:10D50800B69C0108C59C0108D39C01085026002040
:10D51800DF9C0108F09C0108029D010830B5002835
:10D52800104C114AB8BF40423C2590FBF2F304FB73
:10D53800030068430D4D90FBF2F22D682D7B25B951
:10D5480003EB830303EB830301E0C3EB031302EB59
:10D5580083030B8004FB02024FF47A7392FBF3F20D
:10D568004A8030BD806967FF80969800E01F0020E0
:10D57800022803D0431E584258417047064B1B6887
:10D588001B7823B1054B1868C0F3C0407047044BA3
:10D598001878C0F3800070470C060020DC160020C5
:10D5A8003234002010B50A4C5E280146206805D1A7
:10D5B8005D2103F02AFF20683E2105E05D2903D1A3
:10D5C80003F023FF20683D21BDE8104003F01DBF94
:10D5D8009C260020A0F17D03012B70B504460D4662
:10D5E8000A4E05D830687D2103F00FFF84F020042F
:10D5F8003068214603F009FF35B12B881C4404EB41
:10D60800142404F0FF042C8070BD00BFA420002067
:10D6180010B5054C206803F0F5FE18B1206803F03A
:10D62800EEFEF6E710BD00BF7420002010B50446DA
:10D63800C0B2FFF7B7FFC4F30720BDE81040B1E759
:10D64800024B5E21186803F0E0BE00BF9C26002054
:10D6580038B5064C05465E21206803F0D6FE2068E2
:10D668002946BDE8384003F0D0BE00BF9C26002004
:10D6780013B5044601A90068FFF750FF1320FFF710
:10D68800E7FFBDF90400FFF7D1FF1B20FFF7E0FF1C
:10D69800BDF90600FFF7CAFF2320FFF7D9FF23686B
:10D6A800002BB4BF53204E20FFF7C0FF01A96068CC
:10D6B800FFF734FF1220FFF7CBFFBDF90400FFF797
:10D6C800B5FF1A20FFF7C4FFBDF90600FFF7AEFF4C
:10D6D8002220FFF7BDFF6368002BB4BF5720452009
:10D6E800FFF7A4FF02B010BD674B73B51878674DFC
:10D6F800FFF73EFF2B788342044620D0C8B1644B25
:10D708001B68E3B193F9000002230093614B1B6887
:10D718005B78003318BF0123019304214FF416539B
:10D728000022FAF7DDFC5C4B186040B101232B7036
:10D7380005E0594E3068FAF7C0FC34602C70574B3E
:10D74800574D1878FFF714FF2B788342044618D0FA
:10D7580088B1544B1B68A3B10022012493F900003F
:10D7680000944FF4964301920821FAF7B9FC4E4B06
:10D77800186028B905E04C4E3068FAF79EFC346012
:10D788002C704A4B4A4D1878FFF7F2FE2B788342EB
:10D7980004462E4642D0002837D0464B1A68002A45
:10D7A8003CD0D37992F90000434C002B08BF0223E8
:10D7B80002220092002254F8233001921021FAF735
:10D7C8008FFC3E4B0546186040B33D4C94F84A30F8
:10D7D800022B0BD094F89620022A01D14C3405E094
:10D7E80023B1002A04F14C0418BF0024354B1C60F7
:10D7F80044B1204600214C2209F0B0FA02232560EA
:10D8080084F84A300123337008E02C4E306802F067
:10D81800EFFE3068FAF751FC34602C702A4B2B4D20
:10D828001878FFF7A5FE2B788342044629D000B369
:10D83800274B1B682BB3274A93F9000012685278CC
:10D84800002A0CBF082209220323009301924FF4F7
:10D85800614320210022FAF743FC1F4B186080B176
:10D868001E4A012313702B701D4B1A681D4B1A603A
:10D8780007E0194E3068FAF720FC184B34601C702A
:10D888002C7002B070BD00BF14060020A417002041
:10D8980010060020E01F00209C260020150600200E
:10D8A8000020002084200020742000202006002072
:10D8B8008A2000201C060020687A01088C2000209D
:10D8C80028210020902000202C060020A0200020E5
:10D8D8002806002024060020A4200020A8200020DC
:10D8E800A8170020AC200020642928BF6421F8B5BF
:10D8F80010FB01F56424064695FBF4F40027E4B216
:10D90800FBB2A34204D29F2001F0E3FB0137F7E703
:10D91800B4420BD2C4EB84101421C4EB800095FBF5
:10D92800F1F5663D2844C0B201F0D3FB0134E4B2FE
:10D93800B44201D29A20F7E7F8BD2DE9F743934C9A
:10D9480003F056FC6368C31A002BC0F23B8300F552
:10D95800433303F5A07363608D4B1D78237AC5F3B9
:10D968008005EB1A18BF012325724DB1002B00F07A
:10D978002983884B5A789A7001225A701A702BE0C2
:10D98800844A2BB1D37843F00203D3709378537051
:10D99800D67806F0020101F0FF0339B97D4989689C
:10D9A800411A002903DB06F0010300E0012303F01C
:10D9B8000107784917707BB1F2070DD50A79013252
:10D9C800D2B20523B2FBF3F303EB8303D31ADBB222
:10D9D800714A0B71D35C4B706E4EDFF80882337856
:10D9E8007BB3F37823F00203F3706C4B0344AE204F
:10D9F800B36000F0F4FF08B101F0FCFA88F8000009
:10DA0800002800F0DF82B02000F0E9FF402000F09D
:10DA1800E6FF002000F0E3FF102000F0E0FF4FF4E5
:10DA28008067013F0020BFB200F0D4FF002FF8D17B
:10DA3800384601F072FB7278594B53F8220001F016
:10DA480063FB98F80030002B00F0BC827378062B3B
:10DA580000F28682DFE813F00700840218007800DD
:10DA68001C0139017A014F494F4A504B5048FEF783
:10DA780058FB012001F051FB4D4801F045FB022005
:10DA880001F04BFB4B485EE14B4F3B689B0735D59C
:10DA9800DFF85481DFF85491B8F8001044480A239D
:10DAA800B1FBF3F203FB121399F80010009192B244
:10DAB80042499BB2FEF735FBFCF7E8FE012001F076
:10DAC8002CFB3B4801F020FB3D4B99F800201868DF
:10DAD800B8F80030067906FB123164234B43C1784D
:10DAE8008E1B56430220B3FBF6F6F6B201F015FB87
:10DAF80031461520FFF7F8FE032600E001263B68B3
:10DB08001F0540F12D822F4B2F491F68096800918E
:10DB180064232E4997FBF3F2254803FB1273FEF7A3
:10DB280000FBFCF7B3FE304601F0F7FA204801F09D
:10DB3800EBFAFBF765FF0746701C01F0EEFA1520BB
:10DB48003946FFF7D1FE0BE20120214F01F0E5FA3B
:10DB5800204801F0D9FA3B68980749D51E4A14486D
:10DB6800B2F90210B2F900300091B2F904201B4951
:10DB780001921B4AFEF7D5FAFCF788FE022001F055
:10DB8800CCFA0B4801F0C0FA032632E09C260020AC
:10DB980032340020542600203AA20108404B4C00A1
:10DBA800F07E01083FA2010848A201080F9301086E
:10DBB800A52600204EA20108D41F00205AA2010861
:10DBC800D81F0020E41F0020E81F002072A20108CF
:10DBD800EC1F002087A20108B21700209DA20108AF
:10DBE800ACA2010869020020DC1F00207800002098
:10DBF80002263B68D9071AD5B44AB548B2F90210CB
:10DC0800B2F900300091B2F90420B2490192B24A47
:10DC1800FEF787FAFCF73AFE304601F07EFAAC4888
:10DC280006F1010801F070FA5FFA88F846463B6889
:10DC38001A0718D5A94AA648B2F90210B2F9003055
:10DC48000091B2F90420A3490192A54AFEF769FAA6
:10DC5800FCF71CFE304601F060FA9D48771C01F085
:10DC680053FAFFB23E469F4A9948B2F90210B2F9F8
:10DC780000300091B2F904200A2192FBF1F2954993
:10DC88000192994AFEF74DFAFCF700FE304657E03C
:10DC98000026964F3B78B34240F262810E2E00F088
:10DCA8005F817008013001F038FA304604F0EAF874
:10DCB8003B78B34206D9202001F00BFA701CC0B2A1
:10DCC80004F0E0F80236F6B2E3E7894E894996F89F
:10DCD800CC277F48FEF725FA012001F01EFA7C4880
:10DCE80001F012FA844B85491F7879483A46FEF7C5
:10DCF80018FA022001F011FA754801F005FA0C2310
:10DD080003FB07667E4996F8CF2796F8CE3770480A
:10DD1800FEF707FAFCF7BAFD032001F0FEF96C489C
:10DD280001F0F2F996F8D41796F8D22796F8D33777
:10DD3800674800917349FEF7F4F9FCF7A7FD042042
:10DD480001F0EBF9624801F0DFF909E16E4B1B685D
:10DD58001B0640F10181236A616A6C4A8B421FBF2E
:10DD6800536292F82830013303F003034FF00101A6
:10DD78004FF0000018BF82F8283001F0DBF994F862
:10DD88002830634AD05C01F0A4F90220012101F097
:10DD9800D1F900265F4B9B5D3620C3EBC30393FB91
:10DDA800F0F0C0B2062828BF06206038C0B201369D
:10DDB80001F08FF9102EEDD1574B58491B78444884
:10DDC80013F0020F564B1A7814BF59234E23FEF74F
:10DDD800A8F9FCF75BFD022001F09FF93C4801F02F
:10DDE80093F95049504B4E680A68394892FBF3F250
:10DDF8004E4996FBF3F3FEF794F9FCF747FD032031
:10DE080001F08BF932484A4E01F07EF9494B4A49F4
:10DE18001A882F48FEF785F9FCF724FD042001F045
:10DE28007CF92B4801F070F9444B45491A88284879
:10DE3800FEF777F9FCF716FD04210A2001F07AF9BC
:10DE4800234801F061F93F49E26A2148FEF769F980
:10DE5800FCF708FD052001F060F91D4801F054F9B0
:10DE68007268B36838491A48FEF75BF9FCF7FAFCA0
:10DE780005210A2001F05EF9154801F045F93369DA
:10DE8800F26832491248D21AFEF74BF9FCF7EAFC5D
:10DE9800062001F042F90E4801F036F9B2682C4923
:10DEA8000B48FEF73EF9FCF7DDFC06210A2001F0DD
:10DEB80041F9074801F028F926490548152208F0D4
:10DEC800B7FFFCF7CFFC07203AE700BFFC1600209D
:10DED800A52600209DA20108B0A201080217002073
:10DEE80037B00108C0170020B4A20108C4210020DF
:10DEF800D4170020B8A20108D82C0020C4A2010819
:10DF0800D5A20108E6A20108D41F00209C26002003
:10DF1800F8A2010891170020F01F0020FDA20108B7
:10DF2800F61F0020F81F0020809698000EA3010815
:10DF3800B0070020F21F00201BA30108481700208B
:10DF480023A301082AA3010831A301083AA3010861
:10DF580041A30108CC020020F37843F00203F370D8
:10DF6800002D2FD1194B93F82030052B9BBF184A51
:10DF78009B183F251D7F0021122001F0DBF8284661
:10DF880001F0A7F81320002101F0D4F8114B1B78F9
:10DF9800002B114B1B7814BF72202120002B18BFB7
:10DFA800522001F096F81420002101F0C3F894F8EB
:10DFB80030500A4B585D013505F0030501F089F82A
:10DFC80084F8305003B0BDE8F08300BFB0330020C0
:10DFD800F07E0108E80D0020960E0020F8A2010846
:10DFE8002DE9F043324A334F13887D89B7F90490FD
:10DFF800B7F90E80B7F800E0B7F920C05D1B3B8980
:10E008005D43EC13B7F91230B7F91450DB0225441D
:10E018000A2693FBF5F52544B7F90240FD616E43E6
:10E02800A5F57A6505FB05F36C4305FB09F5B7F91A
:10E038000C90FF881B1308FB03F8E41203FB09F399
:10E0480004EBE8281B14042403EB65331EFB04844B
:10E058005568023304FA0CF49B1002344CF2503227
:10E06800A5EBA40403F5004342FA0CF27B43624398
:10E078004FEAD33747BFB2FBF7F35B005400B4FB5A
:10E08800F7F31A1240F6DE34524362430A4C5C43FB
:10E09800241404EB2242083602F6CF62361103EB51
:10E0A800221300B1036001B10E60BDE8F08300BF28
:10E0B800D02600209802002043E3FFFF6C4B6D4AF6
:10E0C8002DE9F04F5E8994684FEA062AB4EB0A0AF4
:10E0D8009C884FEA04481C894FF000054FF0000B5C
:10E0E80065EB0B0BA4FB0A6704FB0B77F40944EA06
:10E0F800476418EB04065C884FF000094FEAE715FF
:10E108004FEAC438DC8849EB050787B0CDE90467D6
:10E11800A4FB0A6704FB0B77340A44EA076418EB8C
:10E1280004064FEA27259C894FF0000949EB0507AB
:10E13800CDE90067AAFB046704FB0B77F40D44EAFA
:10E14800472414F5FA664FEAE75545F10007B6F596
:10E15800FA6F77F10003CDE90267964667DAA4FB08
:10E16800046704FB05F34FF0050C07EB4307DDE9F3
:10E178000489A6FB0C230CFB07335F104FEA320619
:10E18800B8EB06084FEA920669EB070946EA837678
:10E198009F10DDE90023921B63EB0703DDE90267AB
:10E1A800CDE90023344A4FF0FF33964277EB03035F
:10E1B800CDE9048928DA40F6AC52A4184FF00003E0
:10E1C8005D4104FB05F3A4FB044505EB43056FF033
:10E1D8000602664202FB0566A4FB0223334418EBE1
:10E1E800020649EB0307CDE904670B26A4FB0623C7
:10E1F80006FB0533DDE900455B104FEA3202A41A3D
:10E2080065EB0305CDE900450AFB0BF3DDE90245A3
:10E21800AAFB0AAB0BEB430B4FEADA7242EA4B025A
:10E22800A41A4FEAEB7365EB0305CDE90245DEF866
:10E238000C40009B019DA4FB032304FB05334FEA1C
:10E2480052584FEA635948EAC328DDE90423B8EB7A
:10E25800020269EB03039946D30B43EA494300B131
:10E26800036009B1029B0B6007B0BDE8F08F00BFE7
:10E2780084020020D026002024FAFFFF054B1A7CD8
:10E2880002F0FF0122B10122027000221A747047C5
:10E2980001707047D026002037B5104B04465D68E2
:10E2A800187806216A46A847A8B19DF800209DF86D
:10E2B800013043EA022323809DF802209DF80330B1
:10E2C80043EA022363809DF804209DF8053043EA61
:10E2D8000223A380012003B030BD00BF74020020D8
:10E2E80013B5104B04465B683B2006216A469847E5
:10E2F800A8B19DF800209DF8013043EA022323804D
:10E308009DF802209DF8033043EA022363809DF8BC
:10E3180004209DF8053043EA0223A380012002B0BF
:10E3280010BD00BF74020020054B93F82020920115
:10E3380034327720F42102F0FC02F7F755BC00BF15
:10E34800980200207720F4212E22F7F74DBC772081
:10E3580048210122F7F748BC772058210122F7F716
:10E3680043BC03460A4668201946F7F73DBC13B577
:10E378000622044603211E206B46F7F7B9FB002846
:10E388003DD09DF800209DF801309DF8021043EA29
:10E3980002231BB21B4A07EE903A92ED007AF8EE80
:10E3A800E77A012067EE877A92ED027AFDEEE77A46
:10E3B80017EE903A23809DF8033043EA01231BB2FD
:10E3C80007EE903AF8EEE77A9DF8041067EE877A40
:10E3D80092ED017AFDEEE77A17EE903AA3809DF868
:10E3E800053043EA01231BB207EE903AF8EEE77ACC
:10E3F80067EE877AFDEEE77A17EE903A638002B00F
:10E4080010BD00BF6000002007B5F62101AB032254
:10E418007720F7F76DFB9DF805309DF804201B0267
:10E4280043EA02439DF806201343054AB2F9202027
:10E43800C2F10802D340034A536003B05DF804FBFD
:10E4480098020020D026002007B5F62101AB022251
:10E458007720F7F74DFB9DF804209DF8053043EA37
:10E468000223024A138003B05DF804FBD026002083
:10E478001FB5044602210C2001220DF10703F7F70E
:10E4880037FB08B900203BE09DF80730DB07F9D5DA
:10E498000321062202AB0C20F7F72AFB0C200921E6
:10E4A80001220DF10703F7F723FB0028EAD09DF8B6
:10E4B800073013F00C0FE5D19DF809209DF80830BE
:10E4C80043EA0223C3EB83339B009DF80B20238090
:10E4D8009DF80A3043EA0223C3EB83339B009DF87F
:10E4E8000D2063809DF80C3043EA0223C3EB83338D
:10E4F8009B00A3800C200A210122F7F775FB01205D
:10E5080004B010BD07B5002101AB03227720F7F74F
:10E51800EFFA9DF805309DF804001B0243EA00431A
:10E528009DF80600184303B05DF804FB08B5FFF733
:10E53800E9FF014BD86008BDD026002008B5FFF7D9
:10E54800E1FF014B986008BDD026002030B5054694
:10E558000C461346294622466820BDE83040F7F7A6
:10E56800C7BA07B50A2100220C20F7F73DFB142093
:10E5780002F065FE0A210F220C20F7F735FB0A206E
:10E5880002F05DFE01AB102103220C20F7F7B0FA70
:10E598000A2002F054FE0A2100220C20F7F724FB7F
:10E5A8000A2002F04CFE0DF10303022101220C2087
:10E5B800F7F79EFA0DF10303092101220C20F7F762
:10E5C80097FA0A2101220C20F7F70EFB03B05DF839
:10E5D80004FB084B1B681869074B20F01F0200F06A
:10E5E8001F01D25801238B401A4201D0FAF7B2BF5B
:10E5F800704700BFC002002014040140094B1B688B
:10E608001869094B20F01F0210B5D258012400F0F8
:10E618001F0304FA03F31A4203D0FAF79BFF034BD4
:10E628001C7410BD8002002014040140D026002074
:10E638002DE9F0437D4A136887B0904693B11A6874
:10E648001AB17B49486902434A619A88ADF80020AB
:10E6580002228DF803209868002269468DF802206E
:10E66800F7F72CF9322002F0EAFD002111221E20D2
:10E67800F7F7BAFA012160221E20F7F7B5FA6420ED
:10E6880002F0DDFD02A8FFF772FE00240A272646E5
:10E698002546022101221E20F7F7A6FA322002F0B1
:10E6A800CEFD02A8FFF763FEBDF90820BDF90A10E8
:10E6B800BDF90C308A421444A8BF0A4693421D444F
:10E6C800A8BF134613F5805F0E4404DD013FE0D177
:10E6D8004FF0010901E04FF000091E20002112222D
:10E6E800F7F782FA0A27022101221E20F7F77CFA9F
:10E6F800322002F0A4FD02A8FFF739FEBDF9082078
:10E70800BDF90A10BDF90C308A42A4EB0204A8BF77
:10E718000A469342A5EB0305A8BF134613F5805F8D
:10E72800A6EB010602DD013FDDD101E04FF0000953
:10E7380007EE904A9FED3F7A3F4FF8EEE77A0021C7
:10E74800C7EE277A70221E20F0EEE77AC7ED007A2E
:10E7580007EE906AF8EEE77AC7EE277A9FED377AE8
:10E76800F0EEE77AC7ED017A07EE905AF8EEE77A0D
:10E77800C7EE277AF0EEE77AC7ED027AF7F734FAB0
:10E78800012120221E20F7F72FFA1E200221002245
:10E79800F7F72AFA642002F052FDB9F1000F04D10C
:10E7A8004FF07E533B607B60BB60D8F800301F4C55
:10E7B8001A7B002A37D01A7D002A34D01C498A696E
:10E7C80042F001028A61197D187BFAF70BFE236873
:10E7D8009A689988128A114225D093F91500184928
:10E7E80002F0F0FD23681869FAF7B4FE23681B6984
:10E7F800049300260C23012504A88DF815308DF804
:10E8080014608DF8165003F04BFA23688DF80660F3
:10E818005B7D8DF8043001A803238DF805308DF851
:10E82800075003F01FFA07B0BDE8F083C0020020CC
:10E838000010024000406F466000002001C05E46A4
:10E84800DBE50008F0B52C4D6B7C85B0002B50D172
:10E858002A4C2368002B4CD01A68294E12B17169D2
:10E868000A4372619A88ADF80020022298688DF8F0
:10E878000320694600228DF80220F7F71FF8B369D4
:10E888001E4F43F00103B3612368187B197DFAF723
:10E89800A9FD23689A689C88128A144002D0012333
:10E8A8006B7426E0174993F9150002F08BFD3B685D
:10E8B8001869FAF74FFE3B688DF80C401B69029304
:10E8C80008230DEB030001268DF80D308DF80E603E
:10E8D80003F0E6F93B688DF806405B7D8DF804305F
:10E8E80001A803238DF805308DF8076003F0BAF905
:10E8F800D5E705B0F0BD00BFD0260020800200207B
:10E908000010024005E6000870B50446FFF79AFFBC
:10E91800B4F5807F0ED0BB2C0ED8612C0ED8292CD4
:10E928000ED8132C0ED8092C0ED8002C14BF06258F
:10E9380000250AE0002508E0012506E0022504E09C
:10E94800032502E0042500E00525154C8021A36875
:10E958006B209847642002F072FCA36803216B20A7
:10E968009847104AA3681178192098470F2002F099
:10E9780066FCA36829461A209847A36818211B201B
:10E988009847A36810211C209847A36802213720C4
:10E998009847A36838200121BDE87040184700BF98
:10E9A80074020020BC02002008B5FFF74BFF074B9C
:10E9B8005B7813B1012B03D008BD4FF4006201E06E
:10E9C8004FF48052024B1A8008BD00BF700200202D
:10E9D8001C000020024640213C20F7F705B90246FA
:10E9E80080213C20F7F700B90148024902F0E7B955
:10E9F80000480140702F00200148024902F0DFB9A9
:10EA080000400140202F00200148024902F0D7B9F8
:10EA180000080040F82E00200148024902F0CFB952
:10EA280000040040D02E00204FF08040014902F041
:10EA3800C6B900BFA82E002010B5064C06482146CE
:10EA480002F0BDF904F1C8010448BDE8104002F025
:10EA5800B6B900BF802E0020002C014000440140C0
:10EA68000148024902F0ABB9002C0140802E002079
:10EA7800426A806A131A5842584170474171704778
:10EA880043799B070AD5436A8269D154436A01696D
:10EA98000133B3FBF1F201FB123343627047427951
:10EAA80002F0020202F0FF0342B10369426A806A7F
:10EAB800013BDBB2101A23EA000070471846704782
:10EAC800437913F001031FBFC36803F1FF32C36921
:10EAD800006A1DBF181A1040C0B218467047437923
:10EAE80013F0010310B504460DD0FFF7E9FF58B144
:10EAF800236A6269E168D05C0133B3FBF1F201FB80
:10EB08001233236210BD184610BD90F83B3210B581
:10EB18007BB990F83A3290F83942A34209D2B0F85A
:10EB2800401201229A400A430133A0F84022DBB286
:10EB3800F3E710BD8379DB07D0F8343144BFB1FA6D
:10EB480081F149095A681B8909B193617047138596
:10EB5800704738B50D4B0E4D1A8A0E4B1968498807
:10EB680011421C4603D002F043FB286007E002F084
:10EB78003FFB2B68984282BFC01A074B1860236876
:10EB88005868BDE83840FAF7E5BC00BF0004004803
:10EB9800E4260020AC070020000000201FB5012358
:10EBA800ADF80830ADF80410002301A9ADF80A301B
:10EBB800ADF80C30ADF80620FAF752FB05B05DF859
:10EBC80004FB38B5A0F513746379A579DB0744D540
:10EBD80094F8383205F00105EBB1226B1068C36A6E
:10EBE8005B08436294F83C3223B1B4F842320133F3
:10EBF800A4F84232917A6A00FFF7D0FF012384F823
:10EC08003B32002384F8393284F83A3284F83832B7
:10EC1800A4F8403238BD94F83B32012B04BF94F875
:10EC2800393284F83A322046FFF76FFF94F83B22D6
:10EC3800236B3AB9012284F83B221868997A05FABD
:10EC480002F207E0002284F83B2295421868997A7C
:10EC580008BF0222BDE83840A0E738BD10B5A0F5CE
:10EC6800127494F83C22BAB9A36A616A994228D00E
:10EC7800591CA069A162C35C2069DBB25B0043F444
:10EC880000738142A4F83E324FF00A0384F83D3203
:10EC980028BFA262012312E094F93D327BB1B4F897
:10ECA8003E124B08A4F83E32204601F00101FFF75E
:10ECB80041FF94F83D32013B84F83D3201E084F88D
:10ECC8003C3294F83832002B4ED194F83932013363
:10ECD800DBB2092B84F8393203D12046BDE8104055
:10ECE80013E70A2B40D194F83B322BB9B4F84032E1
:10ECF80043F00103A4F840326379D9071CD5B4F86E
:10ED08004002820501D4C30705D4B4F84432013364
:10ED1800A4F8443210E0E36AC0F347000BB1984707
:10ED28000AE0E3696269D054E369E1680133B3FB3F
:10ED3800F1F201FB1233E361012284F8382294F8DE
:10ED48003B220023012A84F839320DD1A27984F8B4
:10ED58003B32236B12F0010F1868997A0CBF02221C
:10ED68000022BDE8104019E710BDF2E6F1E6F0E632
:10ED78002DE9F04F534D1E464FF414732C1D434399
:10ED880085B080469146E718A24610B92B444E4AF2
:10ED980003E0012805D14D4A2B445A631032C3F8C9
:10EDA80038214FF4147303FB08F3EC180AEB030241
:10EDB80003F59C7346486060343253442163A26172
:10EDC800E36100224FF0010B4FF48071D4F8383121
:10EDD80021610320626222626161E262A26284F8B8
:10EDE800402284F83CB284F83D22A4F84622A4F8D4
:10EDF8004822C4F80C906072A67284F84A8204F51E
:10EE08009A7258681B8901924FF0020C03A9ADF859
:10EE18000C308DF80EB08DF80FC0CDF800C0F6F7A5
:10EE28004DFD636BDDF800C0597B58681B898DF870
:10EE38000E1003A9ADF80C308DF80FC0F6F73EFDA3
:10EE480059463846FFF776FE322002F0F8F9019A63
:10EE5800204BD2F804B0B3FBF9F1B1F5803F03D3EE
:10EE6800012BF8D95B08F6E74FF4147404FB08F893
:10EE780005EB0809584689B2482208F5127802F0CD
:10EE88002DF80AEB0804144BC9F84C3200225846F6
:10EE9800214602F079F8D9F8345016F0010F0CBF6A
:10EEA800022200222868A97AFFF778FE0B4BC9F8DE
:10EEB80050322846211D002202F066F8384605B077
:10EEC800BDE8F08FE42600200C9201082C9201087E
:10EED800147F010800A24A0465EC0008CBEB000887
:10EEE80003460A4690F84602D96A9B7940E7104BD8
:10EEF80073B518781C4698B105230E4D8DF800306F
:10EF08004FF4805600238DF8013001A82E856946FC
:10EF1800022202F071FEAE619DF8050000F00100CA
:10EF280000F00100207080F0010002B070BD00BF49
:10EF38002D06002000040048064B70B51D680646E3
:10EF48001C46FFF7D4FF18B923685B1BB342F8D9F6
:10EF580070BD00BFA817002038B50E4C4FF480557F
:10EF680045F20820FFF7E8FF2585062002F01CFE81
:10EF7800094BA56101221A70C720258502F014FEED
:10EF8800064AA56100231370054A1370054A1360E9
:10EF980038BD00BF000400482D060020882B002043
:10EFA800892B002030060020F7B503238DF80430A4
:10EFB800030C8DF805308DF80700030A06200F466C
:10EFC80014468DF80630FFF7B7FF78B1084D4FF4B7
:10EFD800805601A904222E85002002F00DFE384635
:10EFE8000021224602F008FEAE61204603B0F0BDC3
:10EFF8000004004810B5D420FFF7F1FC8020FFF78B
:10F00800EEFCA820FFF7EBFC3F20FFF7E8FCD3203D
:10F01800FFF7E5FC0020FFF7E2FC4020FFF7DFFCEC
:10F028008D20FFF7DCFC1420FFF7D9FCA120FFF7A7
:10F03800D6FCC820FFF7D3FCDA20FFF7D0FC12205B
:10F04800FFF7CDFC8120FFF7CAFCCF20FFF7C7FCF4
:10F05800D920FFF7C4FCF120FFF7C1FCDB20FFF744
:10F06800BEFC4020FFF7BBFCA420FFF7B8FCA6209D
:10F07800FFF7B5FCAF20FFF7B2FCA620FFF7AFFC07
:10F08800AE20FFF7ACFC2020FFF7A9FC0020FFF71B
:10F09800A6FCB020FFF7A3FC4020FFF7A0FC00204F
:10F0A800FFF79DFC1020FFF79AFC4FF48064013CA9
:10F0B8000020A4B2FFF78EFC002CF8D18120FFF7C6
:10F0C8008EFCC820FFF78BFCAF20FFF788FC0120DF
:10F0D80010BD70B500EB8000094CA0F1A1059C386B
:10F0E80025440444074B15F8010F1E787040FFF7BC
:10F0F80071FCA542F6D13046BDE87040FFF76ABC06
:10F10800387F01083534002010B5441E14F8010F6B
:10F1180010B1FFF7DEFFF9E710BD08B55038C0B2EF
:10F12800FFF75DFC0020FFF75AFC1020BDE80840FF
:10F13800FFF755BC503910B50446C8B2FFF74FFC6D
:10F1480004EB4400400004EB440400F00E00FFF719
:10F1580046FCC4F3C3001030BDE81040FFF73FBCC5
:10F168000846F9F7E5B90F4B1A78702A16D15A886C
:10F17800B2F5006F12D11A79BE2A0FD193F8FC2785
:10F18800EF2A4FF000000BD113F8012B5040064A2C
:10F198009342F9D1B0FA80F04009704700207047D7
:10F1A800704700BF00F0030800F803082DE9F04F8E
:10F1B8002DED028BEF4C85B000214FF40062204604
:10F1C80007F0CCFDEC4B04F53B721A60EB4B0026C4
:10F1D8001E70EB4B04F2CE721A607023237002206B
:10F1E80003236371FDF772F84FF48070FDF76EF832
:10F1F800202242F2107384F868216E22A4F8643148
:10F2080084F87A211E230A22A4F8663184F87B2127
:10F218004FF416732B22A4F86C3184F87D21012356
:10F22800212284F85E3184F8693184F86A3184F8DF
:10F238007C3184F87E2184F884312322002384F8E9
:10F248007F21C4F82032C4F824324FF4C872052351
:10F2580084F8CC67A4F87061A4F86E61A4F87261B0
:10F2680084F8556184F8566184F85761A4F85861A8
:10F27800A4F85A61A4F85C6184F85F61A4F882611B
:10F28800A4F88021A4F8866184F81D6284F81C62C1
:10F2980084F8286284F8296284F82B3240F2DC531F
:10F2A800A4F8963140F24C43A4F8983140F26C73BC
:10F2B800A4F89A3140F27533A4F89C3140F6430320
:10F2C800A4F89E3184F82A6284F8906184F89161E8
:10F2D800254623463746032FCCBF0122002207F1DB
:10F2E800010783F8A02114BF1E220522122F83F8DC
:10F2F800A12103F10203EED140F27E41A4F84011AE
:10F3080040F23A714FF4FA63A4F8421140F27E5188
:10F31800A4F8C631A4F8CA31A4F8CE31A4F8D23181
:10F32800A4F84811052340F2EA5184F8E031A4F822
:10F338004A11C82340F2B451DFF83CB2A4F8E431D2
:10F3480000264FF001084FF47A724FF01E0C4FF46C
:10F35800C87340F2DC504FF0190AA4F84C1132215E
:10F36800A4F8C421A4F8C821A4F8CC21A4F8D02179
:10F37800A4F84421029284F893C1CDF80CC0A4F8F3
:10F38800E831A4F84601019084F8E1A184F892617B
:10F3980084F8946184F8D46184F8DE6184F8DF81AC
:10F3A80084F8E28184F8E38184F8E68184F8EA61EC
:10F3B80084F8EC81A4F84E11A4F85031A4F8521145
:10F3C800009184F8546184F8ED6184F8EE6184F862
:10F3D800EF8184F8F061F9F759FEDBF80030DDF8C9
:10F3E8000CC0267383F80BC083F80CC04FF0220CB6
:10F3F80083F806C04FF00E0C83F810C04FF0350CA0
:10F4080083F81AC04FF0210C83F811C04FF0530C49
:10F4180083F81BC04FF05A0C83F808C04FF0780CE3
:10F428005F759F7583F80AC05F274FF02D0C4FF06A
:10F4380028090099DF704FF00F0E0A2783F807A0FC
:10F4480083F814C04FF0640ADFF854C15973197176
:10F4580083F8008083F8019083F80290DF759E732B
:10F468001E7683F805E0DE735E769F7483F81CA031
:10F4780083F8099083F81E8083F84D90C3F838C04C
:10F48800C3F83CC0DFF81CC1C3F828C0DFF818C1B6
:10F49800C3F834C0DFF814C1C3F844C0C3F848C087
:10F4A8004FF04B0C83F84CC0DFED367A9FED368A6F
:10F4B800C3ED0B7A4FF4E17CA3F856C0B7EE087A97
:10F4C8004FF0100C83F858C083ED087A83ED097A61
:10F4D800C3ED0C7A83ED108A83F84E7083F84F7071
:10F4E80083F8507083F851A083F852A083F853A092
:10F4F80083F8546084F8D017142184F8D61701983B
:10F508002249A4F8D8074FF0460C84F8CFC784F8EE
:10F51800CEA784F8D16784F8D56784F8D26784F8D1
:10F52800D36784F8D467A3F86060A3F8626099662B
:10F53800152183F8701016495967164999671649B5
:10F54800D967A3F85E6083F864E083F86C9083F869
:10F558006D9083F880801148F9F7D6FDDBF800300C
:10F56800029A83F819614FF44871A3F81E1183F8C1
:10F578001A611DE0D417002018170020D82C00208D
:10F5880044170020CDCCCC3E000000000000A04075
:10F598009A99193FF6287C3F3D0A773F76A30108E0
:10F5A8000AD7A33C9A9979406666663F0000C04036
:10F5B80083F81B9183F81C8183F82061194684F82D
:10F5C800D67184F8D771A4F8D82184F8DA61A4F840
:10F5D800DCA10E2202FB06326FF0170082F821012F
:10F5E800032082F822016FF02F0082F82301072000
:10F5F80082F824016FF0230082F82501052082F8A3
:10F60800260101365A2081F8280181F8290164224F
:10F61800FF20082E81F8272181F82A0101F10E0127
:10F62800D7D1002183F89111C821A3F89211142190
:10F6380083F89411A3F898211E214FF4967283F849
:10F648009511A3F89A210121282283F89611A3F88D
:10F658009C212F4B18EE102A45F8102F9D42F9D106
:10F668002C480021402207F079FB00232A4D2B4C1F
:10F6780059591A1904330868C2F8AC02382BF5D165
:10F6880004F50B700021802207F068FB05F13801B2
:10F69800702204F50B7007F058FB00F0A3FA4FF442
:10F6A8000020FCF713FEDBF800600125314604F268
:10F6B8008C404FF4D07284F8F45784F8F25784F8E9
:10F6C800F35707F042FB04F22C6031464FF4D07236
:10F6D80007F03BFB124B1B681A68C4F8DA275A6814
:10F6E800C4F8DE279A68C4F8E2271A68C4F8E6273F
:10F6F8005A68C4F8EA279A68C4F8EE27022384F8FF
:10F70800E85484F8883605B0BDEC028BBDE8F08F6C
:10F7180094180020801A0020DC810108D4170020EA
:10F72800441700201549D1F8883043F47003C1F814
:10F738008830134B1A6842F001021A605868114A5F
:10F7480002405A601A6822F0847222F480321A60E9
:10F758001A6822F480221A605A6822F4FE025A605B
:10F76800DA6A22F00F02DA62186B074A02401A635B
:10F7780000229A604FF000638B60704700ED00E054
:10F78800001002400CC07FF8CCFC00FF38B5144BC9
:10F798001B68984205461ADD124B93F8F44714B1DA
:10F7A800012C09D017E0104B1B68186988B1A842D2
:10F7B800CCBF0120022038BD7F280CDCFBF742F8C3
:10F7C800C0F17F00854208DDFBF71AF805E000204C
:10F7D80038BD012038BD022038BD204638BD00BFE5
:10F7E800D4310020D41700201C300020074B93F898
:10F7F800F437012B08D1064A064BD0681B688342B0
:10F8080034BF00200120704700207047D417002023
:10F818000C0000203006002038B5094B93F8F45747
:10F8280065B9084C2068F8F748FC074B25601B7839
:10F83800022B03D1BDE83840F9F7E7BB38BD00BF5C
:10F84800D41700201C30002019300020064B93F8F4
:10F85800F4371BB1012B05D1FAF7D2BF034B186857
:10F8680001F0C7BD00207047D41700201C300020CD
:10F87800F8B5011F06460023083051F8042F02F19D
:10F8880020043F2C3BD802F108040F2C06D8023282
:10F89800032A04D9002B08BF012300E00223814278
:10F8A800EBD1012B30680ED0022B1AD0736803F00D
:10F8B80003039B0000F0030043EA0010B36803F061
:10F8C8000303184317E000F00F0040F04000F8F77A
:10F8D8002FFEB068736800F00F0040EA0310C0B252
:10F8E80009E000F03F0040F08000F8F721FE307991
:10F8F800F8F71EFE307ABDE8F840F8F719BE06F1B1
:10F908000C0734463A46002552F8043D03F18001BD
:10F91800FF294FEA850510D903F50041B1F5803F6D
:10F9280002D245F0010508E003F50003B3F1807F3A
:10F9380034BF45F0020545F00305B242E4D165F055
:10F948003F00C0B2F8F7F4FD05F00303022B20785E
:10F9580007D0032B0CD0012B13D1F8F7E9FD607801
:10F968000FE0F8F7E5FD6078F8F7E2FDA07808E029
:10F97800F8F7DEFD6078F8F7DBFDA078F8F7D8FD3A
:10F98800E0780434F8F7D4FDBC424FEAA505DBD192
:10F99800F8BD10B504467F2C06D964F07F00C0B2CC
:10F9A800F8F7C6FDE409F6E7E0B2BDE81040F8F75D
:10F9B800BFBD430083EAE070EBE72DE9F047314B28
:10F9C80093F8F437012B86B0074601D004464AE085
:10F9D80007F004FA03A9054606466846FAF720FE2A
:10F9E800039B049A029713442B443F2B059519D97E
:10F9F8000023684603A90322FAF73EFE039B3BB99E
:10FA0800049B2BB9204A13705370059BABB301E0DC
:10FA1800FAF7EEFD039B049A059E134433447F2BAB
:10FA28002BD8029FDFF86090CA4639461AF8024B75
:10FA3800C4F18008B04528BFB0460AEB040044442E
:10FA4800E4B2424607F081F9802C89F8004014D1CD
:10FA5800C8EB0606504607EB0801324607F075F971
:10FA680089F8006009E0254614F8011B21B1074B0D
:10FA7800186801F0CAFCF6E7ED1B284606B0BDE899
:10FA8800F08700BFD4170020882B00201C300020EE
:10FA98000FB437B506AC482054F8045BF8F748FDB6
:10FAA8002020F8F745FD2A4623460B4901940020FB
:10FAB800FCF74AFA04460A20F8F73AFD074BC4F166
:10FAC800FF241A6804F57F04FD3414441C6003B055
:10FAD800BDE8304004B0704769F10008D431002017
:10FAE8000FB407B504AB064953F8042B0193002063
:10FAF800FCF72AFA03B05DF804EB04B0704700BFC6
:10FB080069F1000810B54B88DC0641BF2F4B14790A
:10FB18001B6853F8244044BF2D4B43F820404B88C2
:10FB28009B0641BF294B54791B6853F8244044BFB6
:10FB3800274B43F820404B881C070ED5254B0C78E3
:10FB48001B78B3EB141FA1BF204BD4781B6853F864
:10FB58002440A4BF1E4B43F820404B889B070ED57A
:10FB68001D4B0C781B78B3EB141FDFBF174B547871
:10FB78001B6853F82440DCBF154B43F820404B88E2
:10FB8800DC070FD5154C0B78247803F00F03A3423C
:10FB9800DFBF0E4B14781B6853F82440DCBF0C4BB6
:10FBA80043F820404B885B070FD50B780C49097840
:10FBB80003F00F038B42A1BF044B92781B6853F8E4
:10FBC8002220A4BF024B43F8202010BD9426002019
:10FBD8003A0D00207F2400207D2400207C24002072
:10FBE8007E240020254A264826490023F0B51468BB
:10FBF80003700B701D461A46661976884EB9675D04
:10FC08003FB9037000230A704B7007781D461A46E7
:10FC18000CE0360548BF013205F1040503F1010384
:10FC280048BFD2B2802DDBB2E6D1EAE7E8B2B842EB
:10FC38000CD214F8250006099E4200F00F00A8BF58
:10FC4800731C9042A8BF421C0135EFE74B708A70C5
:10FC5800C2F3470102F001020A444C1E0A490B484C
:10FC68000A70C3F3470203F0010313440470084900
:10FC7800501E084A08701370F0BD00BFB82000205D
:10FC8800742400200C2C00207E2400207C240020DA
:10FC98007F2400207D2400202DE9F04FC24BDA6834
:10FCA8002DED028B1A61C14A1168D960C0490B68F1
:10FCB80043F020030B60BF4B1978012990460CBF15
:10FCC800002201221A70BC4B1A78910789B040F1C2
:10FCD8003D83BA490978042940F23883B84909783C
:10FCE80001F0040101F0FF0011B922F001021A70BD
:10FCF8001B78DB0702D408B1FAF750FBB149CA7880
:10FD0800531C052293FBF2F202EB82029A1AAE4BC5
:10FD1800CA701B78039392000023AC4CDFF8CCC266
:10FD2800DFF8D8925CF8231091FBF9F504F108008C
:10FD380004F1100640F82350A54844F8231000FBAE
:10FD4800051142F2107091FBF0F080B226F8130012
:10FD58004FF0140E04F1140604F13C0A0EFB036E76
:10FD68005AF823605EF802704EF80210F61B314410
:10FD780044344AF82310052691FBF6F109FB0511D6
:10FD880044F82310039C012C4FEA830BE24605D16B
:10FD98000238B0F5797F98BF4BF80C100BB90123E6
:10FDA800BBE7884CD8F80030226D9FED8A7A8A4EDE
:10FDB8008A4D9B1A07EE903AF8EE677AD8F8003029
:10FDC8002365C7EE877A7C4B1B78B7EE008AF4EE82
:10FDD800C87AF1EE10FA58BFF0EE487A13F0010332
:10FDE800C4ED157A12D005AA00927D4B06AA01929D
:10FDF8000CCB9AE80300FAF765F96421059A069B8B
:10FE0800B2FBF1F293FBF1F3328000E033802B80F8
:10FE180094F858306B48002B3BD0D0ED157AC26D62
:10FE2800DAF80030C8EE276A9B1A026E022507EE40
:10FE3800103AB8EEC77ADAF8043027EE267A9B1A19
:10FE4800FDEEC77AB0F9662017EE901A07EE903AE1
:10FE5800644BB8EEE77AD3ED007A67EE277A67EE5F
:10FE6800A67AFDEEE77A17EE903A02FA83F3B0F934
:10FE7800642093FBF5F302FA81F29BB292FBF5F250
:10FE880092B2A0F86A30A0F86820A0F86630A0F80E
:10FE98006420012384F85830534BDAF804101B8887
:10FEA800DAF80000474D514E216603F03003E06553
:10FEB800002B00F04B8205F17403009305F17803E1
:10FEC8000193EA6E2B6FFAF7FDF872682B6F9B1A95
:10FED80007EE903A434B326893ED007AEB6EF8EEFA
:10FEE800E77A9B1AEB67384B67EE877A1B78FDEE4B
:10FEF800E77A012BC5ED207A03D0022B00F0DF80D2
:10FF080024E2D5ED287A3A4BD5ED215A95ED255ABC
:10FF180095ED156A95ED264AD5ED274A35491D68B0
:10FF2800B1EE677ABDEEC77AFDEEE77A17EE10EA12
:10FF380017EE90CA0020304A91ED007A52F82070EE
:10FF480007EE907AF8EEE77AA2F1140367EEA57A45
:10FF580033F81060FDEEE77A283217EE903A9B1BD3
:10FF68009BB222F810301BB207EE903AF8EEE77A0F
:10FF78003B4467EE857A4400FDEEE77ACDED037ADF
:10FF880007EE903AF8EEE77ABDF80C8067EE847ACF
:10FF9800A7EE867AFDEEC77A17EE902A724531DB16
:10FFA8006245A8BF62462EE0B0070020A8170020CF
:10FFB800EC1F00204A170020F01F0020F61F002029
:10FFC800323400200C2C0020000F0020102C0020C0
:10FFD800806967FF00007A446A2000206C200020B6
:10FFE8004C1700206C000020B4200020F81F0020CF
:08FFF800040F0020340F00206B
:020000040801F1
:10000000882C002080969800DB0FC940724607EECE
:10001000902AF8EEE77A5FED046AC1ED007AFDEE12
:10002000E77A313617EE903A43449AB2AB78D1ED85
:10003000027A07EE103AB8EE477A4B684F6027EE27
:10004000267AFB1A88EE077AB6B2622E06EE903A4E
:10005000F8EEE66A37EE067AC6EE866A86EE077A2C
:1000600076EEE76AE7EE267AC1ED047AC1ED027A10
:100070000FD964EEA77ABA4EFDEEE77A17EE903A02
:10008000B3F5FA6FA8BF4FF4FA63B342B8BF334673
:1000900000E0002313441BB240F6B8329342A8BFDD
:1000A0001346B04A9342B8BF1346AF4AA352AF4A71
:1000B000142303FB002351F8142B1A60002840F08E
:1000C000498101203BE7AA4BD5F874801F68D4F81A
:1000D00078903E89DFEDA78A4FEA58039E4228BFF9
:1000E0001E46B5F8A8301AB29642C3BFD5ED157AB0
:1000F0009FEDA17A67EE877AB6B2C1BFFDEEE77ACF
:1001000017EE906AF618B6B2C8BFA5F8A860D4F882
:10011000AC50C5EB09052846FAF786F80028D8BF89
:10012000404241F293129042CCBF0020012088B39C
:1001300007EE905AB8EEE70A20EE280AFCF739F8E5
:1001400007EE908AF8EE677A40F6B83320EE270A79
:10015000FDEEC07ACDED037ABDF80C20A4F8B020F6
:1001600012B29A42A8BF1A467E4B9A42ACBF09EB24
:1001700002034B4448F6A042934203DDA3F50C432F
:10018000A03B04E0002BBCBF03F50C43A033C4F834
:10019000B43001E0C4F8B490D4F8B450C5F50C53B1
:1001A000283307EE903AF8EEE77A67EEA88AB0EEC9
:1001B000680AFCF75FF88DED070AB0EE680AFBF7F6
:1001C000F8FFD4ED317AD4ED2E4AD4ED155A94EDE2
:1001D0002F4A94ED305A65498DED060AB1EE677AE3
:1001E000BDEEC77AFDEEE77A0DF1180E17EE10AAF4
:1001F00017EE90BA0020614AFEEC016A32F9103025
:10020000DFF88C9107EE903A07EE106AF8EEE77A85
:10021000B8EEC77A3C32D6EE877A4FEA400CFDEE54
:10022000E77ACDED037ABDF90C30B3F57A7FA8BF3C
:100230004FF47A734B45B8BF4B461FFA83F922F847
:1002400010900FFA89F207EE902AF8EEE77A27EE7F
:10025000A47ABDEEC77A8DED037A27EE847AD1EDCC
:10026000007ABDF80C90E7EE257AFDEEE77A17EEFE
:10027000902A524503DB5A45A8BF5A4600E0524631
:1002800007EE902AF8EEE77A9FED3D6AC1ED007A1D
:10029000BA7891ED027A06EE902AF8EE666A4A681C
:1002A0004B6066EE866A9A1AC8EE266A143106EE2C
:1002B000102AB8EEC66A76EEA56A86EE256AC5EE05
:1002C000A66A36EE476AA6EE867A01ED017A01ED5E
:1002D000037A25EE077ABDEEC77A17EE103ABDEE27
:1002E000E77A4B4417EE102A13441BB240F6B8329B
:1002F0009342A8BF13461B4A9342B8BF13461A4AFB
:100300002CF802301F4A142303FB0023C3ED007AAC
:1003100008B901206FE73B7923B1642395FBF3F51E
:10032000194B1D803B8898450DD9D4F8AC30A06F8F
:10033000C01AF9F779FF80EAE072A2EBE07242F2AC
:1003400010739A4206DD114B01221A700E4BB4F85D
:10035000C8201A8009B0BDEC028BBDE8F08F00BF49
:1003600030F8FFFF48F4FFFF880F00205C0F0020EB
:10037000040F0020D30237390000C842742C00203B
:10038000DB0FC940340F0020FC0E0020000F0020BE
:1003900018FCFFFF8388826810B51C0641BF144813
:1003A00090F8CC074FF4D07404FB0022D80544BF6A
:1003B0001048007803F03F0344BF00EB400002EB1D
:1003C0008002042B0DD003D8013B012B07D910BDAF
:1003D000102B08D0202B08D0082B07D101E011707A
:1003E00010BD118010BD116010BD116010BD00BFA7
:1003F000D4170020D82C002007B5064B0093064BDD
:1004000001930649064A074B0748FBF7A3FE03B0D2
:100410005DF804FB379301080F9301084EA2010811
:1004200048A201082B9301087FA3010808B50378AF
:1004300033B90C4B0C481978BDE80840FBF78ABE6D
:1004400005F02AF902280CD8064B1870074B0C222D
:1004500002FB0030064B06301860FCF707F8054831
:10046000E5E708BDD82C00209FA301089C1F0020B1
:10047000441700201096010808B503783BB90B4BD0
:100480000B4893F8CC17BDE80840FBF763BE05F0B6
:1004900003F9022808D8054B83F8CC07FBF74CFF7B
:1004A000FCF708F80348E8E708BD00BFD4170020B0
:1004B000A3A301081096010838B5037803BB214BAC
:1004C0001B6801330F2B07D81F490C2202FB0312B4
:1004D0001C4695682DBB00E01C4601340F2C01DD45
:1004E000002400E005D818490C2202FB041295688C
:1004F000BDB99C42F1D11548BDE83840FBF72ABE92
:1005000005F0CAF80F28044605D80F4A0C2303FB50
:1005100000239D682DB921460D48BDE83840FBF702
:1005200019BE084B1C6000F0BBFE21462A46094854
:10053000FBF710FE0C235C43034B185DBDE838400D
:1005400000F0C2BE70000020B4820108B0A3010810
:10055000C6A30108DEA3010873B5037813B9F7F742
:1005600053F93DE01F4901AA05F0F7F800240146C0
:100570002646254699B134B1012C08D1084605F02C
:100580008BF8064603E0084605F086F8054615494F
:10059000002001AA05F0E1F801340146EAE70B2D3D
:1005A00002D911480C220BE0022C10D1A6F57A7367
:1005B000B3F57A7F07D90D484FF47A714FF4FA6298
:1005C000F7F79FF80CE00A4B03EB45035E80084BFE
:1005D000084803EB45032946B3F90220FBF7BAFDAF
:1005E00002B070BD7A9B0108509801082A9F01084B
:1005F000D82C0020F5A3010838B50D4C23688342A0
:10060000054606D1F7F75DFD204600214C2206F095
:10061000A9FBE36CAB4209D12846F7F752FD054828
:1006200000214C22BDE8384006F09CBB38BD00BF1D
:100630002821002074210020034B1A68D379591C0B
:100640001344D171187A70479420002010B5FFF739
:10065000F3FF84B2FFF7F0FF04EB002080B210BD7F
:1006600010B5FFF7F3FF0446FFF7F0FF04EB00407F
:1006700010BD064B10B504462146186800F0C9FEAF
:10068000034B1B6898796040987110BD982000203A
:1006900094200020014B1B689879EAE79420002001
:1006A00038B5044624200D46FFF7E3FF4D20FFF741
:1006B000E0FF002C084C14BF21203E20FFF7D9FF9B
:1006C0002368002228469A71FFF7D3FF236893F826
:1006D0004900BDE83840CCE79420002001460020C6
:1006E000DEE710B50446C0B2FFF7C3FF200ABDE83D
:1006F0001040BEE710B5044680B2FFF7F2FF200CB1
:10070000BDE81040EDE737B58288836804461006DF
:100710000D4641BF2B4991F8CC174FF4D07000FB28
:100720000133D10544BF2849097802F03F0244BF94
:1007300001EB410103EB8103042A12D006D8012A00
:100740000DD0022A32D193F9001030E0102A0AD0DD
:10075000202A0AD0082A29D1B3F9001027E01978F5
:1007600025E0198823E0196821E093ED000A684626
:10077000FBF770FB01461548FBF7ECFC05B3D4ED25
:10078000037A6846B8EEE70AFBF764FB01461048B7
:10079000FBF7E0FC94ED040A6846B8EEC00AFBF7EC
:1007A00059FB01460A48FBF7D5FC09E0002109483E
:1007B000FBF7D0FC25B10848E1682269FBF7CAFCC9
:1007C00003B030BDD4170020D82C0020F3990108C5
:1007D000EC99010827A3010804A40108024B014673
:1007E000D86900F016BE00BFD82C002010B5441EFA
:1007F00014F8011F21B1034BD86900F00AFEF7E796
:1008000010BD00BFD82C002010B503781BB90A48D2
:10081000BDE81040EAE704F03FFF0446082899BF0E
:100820002146064806480821FBF794FC601EC0B22A
:10083000BDE81040F7F7C8BB0BA4010852A401089B
:100840007EA40108F7B52B492B4B08782B4D1C686B
:100850002B4B05EB80001A882A4BD0F8C0101B7870
:10086000294800914FF47A71B4FBF1F1FBF772FC67
:1008700026484821FBF76EFC254B1F680026F3B283
:1008800005EB8302D2F8D010E9B101249C403C4230
:1008900017D0220715D01F4AD25C0B2000FB032380
:1008A000164A1D4802EB8303D3F8F020FBF752FCF5
:1008B000022C06D1194B93F8281011B11848FBF7F8
:1008C00049FC0136DBE71748FFF790FF164B174846
:1008D0001A68174B9A420CBF164B174B1A88174BC6
:1008E000198892B24FF4006303B0BDE8F040FBF703
:1008F00031BC00BF3C200020A8170020B4820108B2
:10090000DC1F002078000020A9A40108ECA4010845
:10091000EC1F00207C000020FCA40108D82C002043
:1009200004A501084CA50108D416002008A501085B
:1009300000540040D8160020DA160020D0160020FF
:100940002DE9F843002481462746184E06F5D07558
:10095000494654F80580404606F080FAC8B1414641
:100960001348FBF7F7FB1349404606F077FA0146B8
:10097000281941B183681B7806EB8306D6F8A80EC8
:10098000FFF734FF01E0FFF7BEFE0B48FFF72EFF35
:100990000137143440F60C539C42D6D11FB9074896
:1009A000BDE8F84322E7BDE8F88300BFB482010840
:1009B0007B9A0108819A01084CA50108C298010898
:1009C0002DE9F04F2DED028B83B0824606F00AFA36
:1009D000054628B1012819D19AF800302A2B15D1E3
:1009E0007748FFF703FF0024764E7748A159FBF7BD
:1009F000B1FB30192946FFF786FE7448FFF7F6FE73
:100A0000143440F60C539C42EED1D3E050463D21C5
:100A100006F0DBF9002800F0C68003461F4613F8F5
:100A2000012D202AFAD0461C304604F035FE05463A
:100A30003046FBF785F9CAEB0707B0EE408A4FF066
:100A4000000BDFF8B491142409F5D07304FB0BF408
:100A5000019354F80380404606F0C4F98446624688
:100A600050464146CDF800C006F0C4F9DDF800C09C
:100A7000019B002840F08A80FAB2624540F08680EF
:100A8000404653491F1906F0E9F98246002851D023
:100A9000E5B930464F4906F0E1F948B13846012141
:100AA000FFF778FC4C484B4A4146FBF753FB0125C6
:100AB00030464A4906F0D2F9002838D0384602219B
:100AC000FFF768FC4448454A414629E04C44D4F8C5
:100AD000AC319D4216DA4248FBF73CFB3D48FBF740
:100AE00039FB4048FBF736FB3C48FBF733FB3D48FE
:100AF000FBF730FB3C4803B0BDEC028BBDE8F04F88
:100B0000FBF728BBD4F8B0319D42E4DC09EB850447
:100B100038462946FFF73EFC2F48D4F8A82E414618
:100B200003B0BDEC028BBDE8F04FFBF713BB002D0B
:100B300040D1D0E74C44D4ED6B7AF8EEE77AB4EECE
:100B4000E78AF1EE10FA1FDBD4ED6C7AF8EEE77A63
:100B5000B4EEE78AF1EE10FA16D8B4F8A43113F027
:100B6000200F18EE101A384608BF2946FFF712FC6E
:100B700041461E48FBF7EEFA3846514603B0BDEC3D
:100B8000028BBDE8F04FBEE5194806E00BF1010B02
:100B9000BBF1A70F7FF455AF164803B0BDEC028B35
:100BA000BDE8F04F22E6504603B0BDEC028BBDE835
:100BB000F04FC5E603B0BDEC028BBDE8F08F00BF7F
:100BC0003AA50108548401087B9A01084CA5010844
:100BD000819A01084FA5010857A5010867A50108DA
:100BE00070A501087A9B0108E8A401089CA50108EA
:100BF000A7A50108C2980108B482010808B50748F2
:100C0000FFF7F4FD064BD869F7F750FA00F06CFDDA
:100C1000FBF768FB034B044ADA6008BDC7A501086F
:100C2000D82C002000ED00E00400FA0508B50548C6
:100C3000FFF7DCFDFEF7BEFAFBF77EFBBDE80840E0
:100C4000DCE700BFD3A5010808B50448FFF7CEFDD7
:100C5000FBF772FBBDE80840D0E700BFE9A501083B
:100C6000026D036B70B50446D5699BB9A90611D511
:100C7000C36A1BB1908C80B298470BE0E169928CFB
:100C800040694E1CD2B2E6614254E169E268914289
:100C900028BFE361616BA1B92A0612D5636AA26A13
:100CA0009A42236D09D0501CA669A062B25C1A85D5
:100CB0002369984205D3A16203E01A6822F08002FA
:100CC0001A602B0742BF236D08221A6270BD026BA7
:100CD000C168034610B5406942B11A6C8C1A013ADA
:100CE000005D08BF0A46C0B21A6410BD1A6A805C73
:100CF00001328A4228BF0022C0B21A6210BD436B83
:100D000013B190F844007047836A406A1B1A584236
:100D100058417047426A816A03698A4238BFD218D3
:100D2000521A416B21B149680A44591E8A4203D2C2
:100D3000013B981AC0B2704700207047036B13B193
:100D40005B68016C01E0C369016A8B423CBFC26809
:100D50009B18581AC0B27047836A8169426B194464
:100D6000D160416A99429DBF0169CB1A5360CB1A89
:100D700096BF0023536083624FF0000380F8443035
:100D8000136888BF816243F0010313607047436AB0
:100D90008269D154436A02690133934228BF002318
:100DA0004362436B1BB11B68DB0705D4D4E7026DBC
:100DB000136843F08003136070474171F4F774B90E
:100DC0008160F4F771B92DE9F0410369C768054600
:100DD0000E461F40002F35D0B7FA87F24FF0004380
:100DE000D340DB432B611F40A2F11B03042BF1D83E
:100DF000DFE803F0221F1C190300746A24B1013CD0
:100E00000023A4B2736201E0EC6AA4B2D6F8208099
:100E1000B8F1000FDED0D8F80030404621469847A0
:100E2000D8F80480F4E73068696B07E07068A96B54
:100E300004E0B068E96B01E0F068296C036889B2EE
:100E40009847C7E7BDE8F081224B10B5224C5A43C2
:100E5000224BB3FBF2F203880139013AA04289B276
:100E600092B29BB20ED004F50064A0420AD0B0F159
:100E7000804F07D0A4F59834A04203D004F58064D5
:100E8000A04202D123F070039BB2154CA04206D0C1
:100E900004F58064A0421CBF23F440739BB203801E
:100EA0000D4BC162984202850FD003F50063984252
:100EB0000BD003F54063984207D003F58063984256
:100EC00003D003F58063984201D1002303860123F8
:100ED000436110BD40420F00002C014000A24A04B3
:100EE0000010004073B505460068FFF7ADFF2A68A3
:100EF00013889BB243F001031380EB7A8DF8043022
:100F00000124002601A88DF805408DF806608DF8B3
:100F1000074000F0ABFEEB7A1B2B0BD1192301A885
:100F20008DF804308DF805408DF806608DF8074087
:100F300000F09CFE02B070BD134B800A984220D096
:100F40000AD84A3B984212D00133984211D0B0F5EA
:100F5000801F14D1012070470C4B98420BD00133F5
:100F600098420AD0023B984209D1042070470220DF
:100F70007047032070470520704706207047FE2009
:100F800070470020704700BF4B0010005100100058
:100F9000F8B50468064620460F461546FFF7CCFF15
:100FA00006284BD8B27A910847B902238B40D4F86F
:100FB0000CE0DB439BB203EA0E03E3600A23204A02
:100FC00003FB001342F82370043342F82350154604
:100FD0003FB1B17AE268890802238B409BB2134388
:100FE000E360282202FB00522032EFF312865023E6
:100FF00083F3128803B203EB8303DB0003F10C01DC
:101000001C3329442B4451F8047F17B117600A6838
:1010100004329942F7D100231360F3B283F31188AD
:10102000282303FB0050036A1BB1E36843F001036C
:1010300003E0E2684FF6FE731340E360F8BD00BFC3
:10104000802E002000480BE61C2D0020004807E6FB
:10105000702D0020004803E6C42D00200E4B0F48E1
:101060004FF400525A600E4A11684FF6FE730B405F
:101070001360D0F8DC2011684FF6FE730B4013604C
:10108000D0F8CC20D0F8D0309A4201D0A83063E616
:10109000012380F8EC307047000002401C2D002036
:1010A00044000240034B4FF4004208B19A6170477C
:1010B0001A85704700080048034B4FF4004208B1FE
:1010C0001A8570479A6170470008004810B5447847
:1010D0000078002202FB02F3193B634303F6C413BA
:1010E000534340F6C411434393FBF1F3034921F802
:1010F00012300132072AEDD110BD00BF182E00209A
:101100000430114B33F91000B0F5617F10B506DBE8
:1011100040F6330398420246A8BF1A4601E04FF456
:1011200061720C78192340F2833013FB040494425B
:1011300007DA497813FB01039342B4BF0020012072
:1011400010BD002010BD00BFF631002010B500F129
:10115000500302788A4203D18478C278944204D33F
:1011600004309842F5D1002010BD012010BD0B4B7A
:101170001B6813F4805F0A4BB3F9063005D0C089B1
:10118000421A934207DD084400E0008A8342B4BF5C
:101190000020012070470120704700BFD41F0020AD
:1011A000F63100201FB5094B1B681B030AD58DF8CB
:1011B000040001230D2001A98DED030A8DF80530EF
:1011C000F7F7A4FA05B05DF804FB00BFD41F0020B8
:1011D0001FB5084B1B681B0309D58DF8040002914D
:1011E00000230D2001A98DF80530F7F78FFA05B01F
:1011F0005DF804FBD41F002010B50A4A0A4B1168A1
:101200009B6800BF12689142F7D1084A14694FF4F5
:101210007A7000FB04F2D31AB3FBF4F300FB013045
:1012200010BD00BFA817002010E000E0182E00201D
:1012300038B50446FFF7E0FF0546FFF7DDFF401B2A
:10124000A042FAD338BD10B504462CB14FF47A70E1
:10125000FFF7EEFF013CF8E710BD024A13680133C7
:1012600013607047A817002010B5094CA36923B17B
:1012700094F91420282A00D19847236A3BB1044AE4
:1012800092F91C20282A02D1BDE81040184710BD51
:10129000182E0020014B1B68184700BF183400208F
:1012A00010B50020FFF7F6FF054B00241C7000F07E
:1012B000DBFF044B83F824409C629C851C6310BDBB
:1012C000D4330020182E002010B510B9BDE810400E
:1012D000E6E700230C225A430A4C1119125D8242A0
:1012E00003D00133102BF5D110BD074B186B18B18B
:1012F0004A784078824203D2002219639A859A6222
:1013000010BD00BFB4820108182E002010B54000A7
:101310001428A8BF14200023074A022199540B4423
:1013200099181424834201F8014CF5DBFF21D154B4
:101330000F20BDE81040C7E7042D00202DE9F84339
:1013400007460B24013C35D01D4B08229A617D1CB9
:1013500032264FF00508DFF86890B9F814309BB2D8
:1013600083F00803A9F814300120FFF793FF3046FB
:10137000FFF769FFB9F814309BB283F0080300202F
:10138000A9F81430FFF786FF3046FFF75CFFB8F18D
:10139000000F08D0B8F10108DDD14FF4FA70FFF763
:1013A00052FFFA26D7E7013DD5D14FF47A70FFF707
:1013B0004AFFC7E7034B044ADA60BDE8F88300BF81
:1013C0000004004800ED00E00400FA0510B5084CE8
:1013D000A369224633B1236A1BB10020BDE8104047
:1013E000ACE7012302EBC3039961187510BD00BF80
:1013F000182E002003689B69184703685B6918472B
:1014000003681B6918470368DB68184703685B6853
:10141000184703681B6818472DE9F84FB0F90230E8
:10142000934218BF00232DED048B18BF037005787D
:1014300004460E469146002D40F0978007EE902A14
:10144000DFED7D8AF8EEE77AB6EE009A67EEA88ABD
:10145000DFED7A7A68EEA78AA04668EE898A274689
:10146000B0EE680AFAF7A5FEB0EE408AB0EE680A60
:10147000FAF700FF88EE000A40F2DC5363651023A0
:10148000A4F852301823A4F85030DFED6D6A60EEF6
:10149000266AB7EE006AB0EE667AA0EE007AD0EE69
:1014A000006A37EE067A76EE866AC6EE077A84ED33
:1014B000046A27EE807AB0EE498A27EE007A77EE4A
:1014C000075A84ED017AC4ED025A70EE005A84ED99
:1014D000037AB8EE007AA5EE807A27EE877A67EE77
:1014E000A67A84ED057AC4ED067ADFED567A98ED9A
:1014F000047A27EE277AF0EE678AB5EEC07AF1EE2D
:1015000010FA4CBF77EE487A77EE087A013517EE7D
:10151000900A01F0A7FDD8ED017A67EEA87AC7E935
:101520000E01F5EEC07AF1EE10FA4CBF77EEC87AF4
:1015300077EE887A08F1040817EE900A01F092FD20
:10154000032DC7E9080107F10807CED1A6F2DC5345
:101550001B042367E3676367C4F88030A367C4F89C
:1015600084300123A4F802902370D4F85490B4F985
:101570005280636A276A206FE26FD4F840C0D4F8C3
:101580008010C4F88020C9EB060606FA08F64FEA78
:10159000E67B734307FB0B332667A7FB06671F44F5
:1015A000636C656F60674FEAE27B53430CFB0B3E55
:1015B000ACFB02237344B61A67EB0307E36AA26A23
:1015C000C4F884104FEAE07B434302FB0B3EA2FBCE
:1015D00000237344B6185F41E36CA06CB4F950204B
:1015E000A5674FEAE17B4B4300FB0B33A0FB0101F6
:1015F0001944636B361A206B4FEAE57B05FB03F356
:1016000000FB0B3367EB0107A0FB050119448019B0
:10161000794101F05BF808F1FF3201239340E06764
:10162000C01841EBE371424601F050F8BDEC048B69
:101630004844BDE8F88F00BF6F12833ADB0F494082
:10164000F404B53F0000804B2DE9F8430024234B00
:1016500093F86460E0B2B0420CD203EB8003204AFE
:101660005B6B32F810101BB10B2801D8DB68984770
:101670000134ECE71B4B1B685B032DD5002423468C
:10168000E2B2B24228D2DFF8549009F134074FEAAF
:10169000840857F8242055689D4215D02846FFF746
:1016A0004BFCEFF31283502282F3128828216A6ADE
:1016B00001FB00900132C0F88C206A6942F00102FF
:1016C0006A61DBB283F3118857F808301B68002287
:1016D0001A6001342B46D3E7BDE8F883182E0020AA
:1016E0001C170020D41F002008B50E4B1B6813F4F4
:1016F000805F0D4B14BFD3F88021D3F8842193F879
:10170000641092880023D8B2884204D2074820F897
:1017100013200133F7E7FFF797FF3220BDE80840B9
:1017200091E500BFD41F0020182E00201C170020B8
:101730000A4B1A680A4B30B502F48052D3F8804144
:10174000D3F8845100230AB1A18800E0A988054894
:1017500020F8131001330C2BF5D130BDD41F00201D
:10176000182E0020DA2C002070B5124D00242146DE
:1017700005F28910702285F8884105F0F3FA2146B8
:10178000D5F8FC310B4A0B4493F9020080B102F208
:1017900089141E680E5108199C8884809B79837176
:1017A00092F8883107310133702982F88831E7D106
:1017B00070BD00BF182E0020094B1A680E2303FBD2
:1017C0000020437AFF2B07D0064A12789A4203D9A9
:1017D000054A32F8130000E0808800B2704700BF6D
:1017E00098260020C4210020F63100202DE9F04F7A
:1017F00095490B7813F0010F87B003F0040200F055
:101800008481002A40F08E819048056815F080653B
:1018100040F08881980700F1788143F004030B7051
:101820008B4B8C4FB3F904300A2293FBF2F38A4AB4
:1018300013803B681B0340F14981884B80201D7059
:10184000F7F7DEFC08B1FEF7D7FE854E3478012CA1
:1018500040F03C81834B93F8F21721B193F8F327C2
:101860000AB1914203D3012283F8F22711E0964690
:101870000846BEF1000F06D090FBFEFC0EFB1C0CD0
:101880007046E646F5E791FBF0F183F8F21792FB1C
:10189000F0F283F8F32793F8F427012A82BF714A04
:1018A000002182F8F41793F8F497B9F1000F03D0F0
:1018B000B9F1010F2ED036E08020F6F73FFD8046CB
:1018C00088B38021F6F716FD98F80620664B7070F5
:1018D00053F8223098F90000B3F5613F0CBF0222A3
:1018E000002202218DE806004A468021F6F7FCFB23
:1018F0005E4B70601B684FF4FA7203EB4303B3FB5B
:10190000F2F31BB1402BA8BF402300E00123337248
:1019100060B908E0564BDB682BB1FDF76BFF10B9DF
:101920004023337202E000233370CFE00021142201
:10193000504805F017FA504B336203F17C02F8333C
:10194000B3624E4B7262474A1B88A6F8A03192F8E8
:101950009231396892F8F2C792F88491002B484B83
:1019600018685379A3F11907C1F3C03E18BF4FF0AF
:10197000010E7E427E41012B14BF334601230493A6
:1019800092F8F3373F4E05969C453F4B37681B78DE
:101990000393C1F3402B01F40068C0F3800AC1F344
:1019A0004001C0F3C0002CBF4FF0000C4FF0010C01
:1019B000621ED2B2531E132B3DD8DFE803F00C0C8D
:1019C0000C0C0C0C0C0C0AADAF2729353712121277
:1019D000393F049BA3E0039B9342B4BF0023012340
:1019E00028E03B78022B0BD107EB820353ED027A00
:1019F000F5EE407AF1EE10FA14BF0123002319E04E
:101A0000BB185B79003318BF012313E00B4686E057
:101A1000B8F1000F04D009F1FF367342734100E0C2
:101A2000434603F001037AE05B4678E0734676E0D4
:101A3000634674E013B1012393401D43142C25D851
:101A40000134E4B2B4E700BF32340020DC160020D9
:101A5000C0170020D41F0020FE0E0020D02100203F
:101A600018300020D4170020687A010840170020A1
:101A70000C0000202430002044300020542200209C
:101A8000EC1F0020181700207C2E0020059B274CFF
:101A90001868C4F8A45181301921FFF757FB0023BF
:101AA000C4F8AC31A4F8B031A4F8B231C4F8BC31F8
:101AB000C4F8C0311E4BD4F8B8211B68C4F8C43137
:101AC000022384F8A801C4F8B4212370184B194AE2
:101AD0001B6892F8E0214FF47A7101FB0233164A39
:101AE0001360164B1B681A0609D5154B1B789B070C
:101AF00005D5144B1B78042B01D9062000E00520E6
:101B000007B0BDE8F04FFFF7DFBB5AB9012007B0BF
:101B1000BDE8F04FFFF7FABB034600E05346002B49
:101B200089D18DE707B0BDE8F08F00BF18300020E5
:101B3000A8170020D4170020B80E0020D41F0020C2
:101B4000F01F0020F61F002010B5154A1378590722
:101B500025D523F004031370124B1B681B0319D502
:101B6000114C2378A3F10802012A0BD8FF20002191
:101B7000F6F7CCFD0D4B1B68C4F8C431FDF76AFEC7
:101B80000A2306E0012B05D90A2B03D0FDF748FEF6
:101B9000012323700420BDE81040FFF795BB10BD62
:101BA00032340020D41F002018300020A817002055
:101BB00040F2E9330F4A1289920704D4013B9BB2E9
:101BC000002BF7D10BE00C4A40F2E93310700949C1
:101BD0000989C9070AD4013B9BB2002BF7D1074AF8
:101BE000138801339BB21380FF2070471078C0B276
:101BF000704700BF003800400C380040E43100203E
